:020000040000fa
:08000000540704000000000099
:020000040000fa
:10020000003b88004200f800000e20004220b700aa
:1002100050052000303b8800a00a2000303b8800b9
:1002200061e7a80000000000000000004200f900a3
:1002300061c7bf000078a300fdff3a000000060080
:10024000801f780002d0bf0064e7b7004f0078003d
:10025000103b880010042400e9ff070061c7a900d3
:100260000000060000037800810278004200f800d8
:10027000000e20004220b70002d0bf0032e0b700dd
:100280008001eb000201d100820378000e003200f1
:100290000300d000000043001002ba006418b80048
:1002a000843278000300d000000043001082ba00be
:1002b0006418b80000804200140098008301e80030
:1002c000878f5100f2ff39004200f900000006005c
:1002d0008000fa00889fbe008a9fbe008c1f7800b5
:1002e000010578000206780001fc2f0081046000ff
:1002f00080057800fb03b2000004eb00e00f110062
:100300003d0031000204200061f72f008f80400083
:1003100009007800d3ff07000800e00018003a0049
:100320000b00e00016003200000420000b0050001b
:10033000800078008c0f5000010039008c0078009c
:10034000810178000001eb00e08f10000a0031000d
:100350000b0041000000d0008200d000e1027d00cf
:1003600064f72f000002420005b27f000201e8009e
:10037000830f5100f6ff39000304440015003700d5
:10038000080056000204200080007800820f500010
:100390000100390082007800810178000001eb0043
:1003a000e08f10000a0031008200d00002004400fb
:1003b0000000d000e0027d0064f72f00010242003f
:1003c00005b27f000201e800830f5100f6ff3900fb
:1003d0000804b0000900780099ff070061f72f00ba
:1003e0008f80400009007800080007000904b00071
:1003f0008c0f5400c3ff39004f0678004f05be0034
:100400004f04be000080fa000000060000017800e2
:10041000010278004200f800000e20004220b700e0
:1004200002d0bf0032e0b7008001eb006418b800d2
:10043000640078000009bb006418b80000004200a6
:10044000100090000089bb000281e8008301e800f1
:10045000ff8f5100f5ff36004200f9001000240024
:1004600067ff070061c7a9000000060002e2b700ad
:100470000782a8000000060008c2bf000018a30001
:10048000fdff320008c2a90000c2bf000080fb00cf
:10049000000006000ec2bf00610060000080fb008b
:1004a000000006000cc2bf000000d1006300600025
:1004b000e30f500002003a00901080000200370065
:1004c000901080000080fb00000006008000780093
:1004d0000cc2bf000000d10063006000e30f5000b9
:1004e00002003a0081108800020037000180fb0002
:1004f00080108800000006000a10e20009003200a7
:1005000010042000f1ff070030062000efff070075
:10051000b0062000edff0700a0002000ebff070061
:100520000400370010c4b30010f0b7001000200022
:10053000608088000000060000808000e50f500009
:100540000f003e000a10e20009003200e004200023
:10055000deff070030062000dcff0700b0062000a9
:10056000daff0700a0002000d8ff070004003700d2
:10057000e0c4b30010f0b7001000200060808800d5
:10058000000006000a10e2000900320050042000ba
:10059000ceff070020072000ccff07002007200027
:1005a000caff0700a0002000c8ff070004003700b2
:1005b00050c4b30010f0b700100020006080880025
:1005c000000006003600f800809fbe00829fbe003b
:1005d000849fbe00869fbe00802020004200f8005d
:1005e00042a0a80042c0a80042e0a800900f7800f6
:1005f000100078004200f900e74060000002b200fd
:100600004200de0080c07000eacf500022003a00b5
:1006100099ff07000041780031808000200121000f
:10062000827078000100e00002003a000280fb00c6
:10063000408088003180800020062000808f50009c
:1006400003003e000100e80030808800030037000e
:100650000630ef000030ec00b7ff0700418080005b
:1006600030808000810f50002100360020012100e1
:1006700061407800ea4f500003003a00100020006b
:10068000208088001a0037000630ef000030ec00b0
:10069000a9ff070016003700e2cf500002003a0021
:1006a00075ff070011003700e6cf500010003a0038
:1006b0000e10e2000b003a000c10e20004003200c1
:1006c00010d0bf0069ff07000c30ef0002003700b8
:1006d00070c5b30065ff070010002000708088001f
:1006e000030037000ed0bf0060ff07000e30ef00a0
:1006f0000782a80085a0a9004f03be004f02be00dc
:100700004f01be004f00be003600f9000040060059
:100710003600f800809fbe00829fbe00849fbe000e
:10072000869fbe00889fbe008520a9002901210068
:1007300012003700388080005aff070000f47c0068
:100740000610e20003003a0012d0bf000000fb00d8
:10075000408088003180800020062000808f50007b
:1007600003003e000100e8003080880003003700ed
:100770000630ef000030ec006fff070045ff070078
:100780000004e000ebff3a004180800030808000f0
:10079000810f50000a0036002001210061407800de
:1007a000ea4f500003003a0010002000208088002b
:1007b000030037000630ef000030ec005eff07005a
:1007c0004f04be004f03be004f02be004f01be00eb
:1007d0004f00be003600f90000400600000278001d
:1007e000824278000041eb008001eb00e08f1000b6
:1007f0000500310064c07900004141008301e80038
:10080000818f5100fbff390002c06a000080fb00ad
:100810000000e9004f00de00000006004f28b00095
:10082000889fbe008a9fbe008c9fbe008e1f7800ee
:100830006055b8008044eb00100020005080880014
:100840000c30ef00094678000430ef000030ef0074
:100850008001eb00f107200000df2f00008247003d
:10086000120120000300d00002307a008301e8006a
:10087000818f5100fbff3600c10820004200f800c4
:1008800042a0a80042c0a80042e0a800910f780052
:10089000910678004200f900e20820004200f800ca
:1008a00042a0a80042c0a80042e0a800920f780031
:1008b000120778004200f900030920004200f80006
:1008c00042a0a80042c0a80042e0a800930f780010
:1008d000130278004200f90084bf9f000000eb0083
:1008e0004200f80042a0a80042c0a80042e0a800d0
:1008f0008100780081007800800878004200f900cb
:100900004200f80042a0a80042c0a80042e0a800af
:100910000201780002017800000978004200f90025
:100920004200f80042a0a80042c0a80042e0a8008f
:100930008301780083017800800978004200f90083
:100940000208200000ef2f00808047000000eb002d
:1009500044fe07000a10e2000e0032006802200088
:1009600080382000cf80de00803f9d004008de0000
:1009700001002000903f9d002200200001d72f00a1
:100980008f8040000800780051fe07008d20a800ed
:100990000d003700e8022000202e2000cf80de006e
:1009a000803f9d004008de0001002000903f9d0038
:1009b0002200200001d72f008f804000080078001f
:1009c00043fe07008da0a800cbfe07000904e0004d
:1009d000fd003a000410e200aa00320021012100cb
:1009e000914078008100fb001001210061417800f6
:1009f0008180e9003001210078ff07000004e00059
:100a000003003a000030ec00cbfe070099003700ed
:100a10001350e20084003a0014d0bf000000fb0035
:100a200022002000110009000200d8000005fb0090
:100a300015d0bf004804dd0016d0bf000080fb00c9
:100a4000000444000804d1008001eb00e00f150011
:100a5000130031008701210006f02f0075012100ed
:100a6000f40f20000301d000070041009000fb00bc
:100a7000c808dd0086806000050041001000fb0012
:100a800004006000808040000bd72f008285450065
:100a900081b57f008301e8008a8f5100f1ff3900a2
:100aa0000210e20013003a00f0072000800f54000b
:100ab00010003e008001eb000a00e0006c003200f4
:100ac00001df2f0001814700030044000000d00037
:100ad0008300d00004d72f0001024200e4807f0091
:100ae000013079008301e8008a8f5100f6ff390058
:100af0005f0037000210e20025003a00f07320008a
:100b0000800f540022003600e0ff2a00800f5400be
:100b10001f003e000a01780001d72f008f8040009f
:100b200008007800eafd07000a0178000120210092
:100b300008007800cbfd0700160020008001eb00c4
:100b40000a00e0000d003200022021000300d00066
:100b50000bd72f008f8545008b004000020040001e
:100b600091007800908f5000010032000003eb00ec
:100b70008301e8008a8f5100f4ff39000600e0008d
:100b800026003a000030ec006bfe0700240037001e
:100b900011808000f0072000808f500005003a008f
:100ba000f0bf2f00800f540002003600e10f440018
:100bb00030003a0011808000800f2000808f5000ac
:100bc0002b003a00ee0f540029003e008001eb009c
:100bd0000a00d10000017800100032006418b8004b
:100be00004d72f000f024200e40078000300440005
:100bf0000108bb006418b8000bd72f008f85450093
:100c00000080450090009000030044000188bb0074
:100c10008301e800828f5100f0ff390036fe0700a3
:100c20001cc0b300130037003001210041c0b300e5
:100c300090cf100009003a0014d0bf004800dd003a
:100c400051012100914078008180fb0001004000ab
:100c50000000d1001080880005003700300121001d
:100c600014c0b300904f120002003a008444780090
:100c700021fe07000430ef000630ef006055b80099
:100c80000200370061054500e0854d00004828005e
:100c9000e1012000800f5500818f5d0006003600c5
:100ca0000030ec000610e2000100320022fe0700d6
:100cb0000630ef006055b80000808000e50f50005e
:100cc0003f0036002ffe07000c04e0003b003a0016
:100cd0008da0a9008d20a9000004eb0002082000cf
:100ce0000bef2f008b8047000800780078fd07008d
:100cf00002082000012021000800780059fd0700ab
:100d0000160020008001eb008b82470004202100a8
:100d1000f20720000300d0008500400004004000de
:100d200091007800908f5000010032000003eb002a
:100d30008301e800828f5100f6ff36000600e000d4
:100d4000e6ff3200c00820004200f80042a0a800e0
:100d500042c0a80042e0a80000007800000078002f
:100d60000d0878004200f900e00820004200f80079
:100d700042a0a80042c0a80042e0a80000007800fd
:100d8000000078000e0878004200f90000092000f9
:100d90008fb897004200f80042a0a80042c0a80007
:100da00042e0a80000007800000078000108780008
:100db0004200f90010002000290037000030ef0049
:100dc0000904e00003ff32000c10e200feff3a00cd
:100dd0008da0a9008d20a9000004eb0002082000ce
:100de00004df2f00848047000800780038fd0700ea
:100df00002082000012021000800780019fd0700ea
:100e0000160020008001eb000bdf2f008b824700d3
:100e100004202100f20720000300d00085004000dc
:100e20000400400091007800908f500001003200d3
:100e30000003eb008301e800828f5100f6ff3600cb
:100e40000600e000e5ff32000030ef000230ef0066
:100e50000430ef000630ef000000fe000000eb0061
:100e60004f0778004f06be004f05be004f04be007e
:0c0e7000ef1fb1006f08b1000000060089
:020000040000fa
:100e80000000000000000000000000000000000062
:100e90000000000000000000000000000000000052
:100ea00000000000000000000fe3200080ff200091
:100eb0000001880000000000050007000c0007008a
:100ec000d0620200000000000040da000000fe00d6
:100ed0004440a90000e220000000e00003003200ce
:100ee00000002000a00188004440a8000000060087
:100ef000c04d2700010020001600370062004000ae
:100f0000e0804800910188009001ba006200400032
:100f1000e0804800910188009002ba006200400021
:100f2000e08048000002eb006028e10005003a0084
:100f30008301e90007003300038009000059eb003a
:100f4000040037006128e100010032000082eb005c
:100f500005000700910188001001ba000200e000be
:100f6000e6ff3a0000000500910188008002780049
:100f700062004000e08048003559ba008301e90072
:100f8000080032002559ba008301e900050032004b
:100f90000400e000f4ff320015d9ba008301e90033
:100fa000f1ff3a0000000600817621000a010700e7
:100fb0000000e0000500350081762100a00020003f
:100fc0004f0107000000e00002003d000080eb0040
:100fd000000006000000050081762100480137006e
:100fe000889fbe0080047800010078000204780029
:100ff000890178001100200066010700890078004f
:10100000880f5000010032008000eb0001007800e2
:101010004f04be00000006000000fa004fb9970020
:10102000e881570081762100007f2000b101070090
:101030000080fa0000000600ea874700889fbe0093
:101040008a9fbe008c9fbe008e1f780080067800ad
:10105000010678008204780000047800010037005f
:101060000804e8001800fb00570207000000e00039
:10107000fbff3a0098407800d0c2b30080cf500008
:101080000400320000c0e900d0ef9f0080cf500084
:1010900002003a00d1ef9f000804e8000900e000d8
:1010a00046003500e18f5400440032004002200029
:1010b000808f540041003c000900e0000d00340026
:1010c000f08f54001a003a0000c3b300984f10008c
:1010d00017003a009840900080c7b30080cf5000be
:1010e0001200320080c5b30080cf500010003a00db
:1010f0000e00370000c3b300984f1000020032000a
:10110000a90020000a0037009840900080c7b30073
:1011100080cf5000040032008900200080c5b30059
:1011200080cf500002003a00090120000884e80046
:10113000d8b79f0000c3b300984f100002003a00d8
:10114000d84f1000feff32006055b8000807780045
:101150000e003700fab79f008bbf9f0020142100bc
:1011600000425200c4ef9f006149b9000a00be006e
:101170009d1107004fea97000401fb00cf91de00ac
:1011800000054100818549000804e8001800fb00c3
:101190001502070080007800090178002014210062
:1011a00018020700000278000000e000e9ff3a00a2
:1011b0005fb09700880f500005003a000c00e00077
:1011c000010032000d0e78006000b80027003700e3
:1011d0008e00540070162100694078000000fb006a
:1011e00000805000170033004240a9000f003c006f
:1011f0004fe997000200fb00cf80de0000005500a1
:1012000081805d00800f5500818f5d0007003900ef
:101210006149b900641107007fb197008fb9970049
:10122000820f5000838f58000600320020022000f9
:10123000704688000085eb008085eb00b3c2b300e8
:10124000d3ef9f00d0c2b3005fea9700804f5200f7
:1012500002003a0060051500e0851d000c00e0006a
:1012600001003200080e78000a00be004f07780027
:101270004f06be004f05be004f04be00af00b100d8
:10128000000006000e00fa00889fbe008a9fbe0084
:101290008c1f7800c0b79f00010478000205be00d3
:1012a0008004780078805700e50107006806600038
:1012b0000030a100e10f500014003a00f8815700ff
:1012c000b300780000027800080178000900780077
:1012d0005d0207000000e00002003a006000b80074
:1012e000030037007fb097008fb89700710f070099
:1012f00090bf9f00a1bf9f005fb19700efb1970023
:101300000a0141008b81490016003700e20f5000ae
:1013100018003a00f8815700b3007800140020004c
:1013200008017800090078002d0307000000e000a4
:1013300002003a006000b800030037007fb0970059
:101340008fb897005b0f070090bf9f00a1bf9f0061
:101350005fb19700efb197006e8057001804070047
:101360000a01be001fb89700afb8970081040700bc
:101370000d003700e30f500003003a00000020008a
:1013800001f8270004003700e40f500005003a0080
:10139000f0ff2f00f1ff270090bf9f00a1bf9f002b
:1013a000030037006000b80090bf9f00a1bf9f00fe
:1013b0001fb89700afb897000c00e00001003200a2
:1013c00001f0a2004f0678004f05be004f04be009a
:1013d0000080fa0000000600889fbe008a9fbe00c1
:1013e00000057800810478001004e000300032002d
:1013f000c900900069009000808f500004003900ff
:1014000009007800d80407000000e0003000350033
:1014100019a8a30005003200a10020000a007800ee
:101420001605070080057800010037008005eb00f5
:101430000b00e000030032000a8055000004e800c1
:10144000030037000a007800160507000004780042
:1014500069009000c901900003005000880f5000ff
:10146000020031008005eb000004780008017800dc
:101470008a00780003007800110507000805450080
:101480004900900008004000c00498000b00e000f4
:101490000500320009007800100507008080eb008d
:1014a0000000e00012003a001a04e000d0ff3a0009
:1014b00019b8a300080032000900780007050700ea
:1014c0008080eb000000e00009003a0002003700d5
:1014d0008080eb000600370000c02000190060008b
:1014e0000200320049009000e00498008000eb0008
:1014f000010078004f05be004f04be00000006004a
:10150000889fbe000104780080447800c1009000ec
:1015100068009000808f50000500390008007800b6
:10152000910407008080eb000000e0001600350009
:10153000e80044001100780009587800800878001d
:101540001800780000b8a30004003a0000a8a30027
:1015500007003200eacf540005003a000800780086
:10156000de0407008080eb000000e00006003a0087
:1015700000c0200018006000020032004800900007
:10158000600498008980fb00010078004f04be00d1
:1015900000000600e4874700889fbe008a9fbe00c7
:1015a0008c9fbe008e1f780081bf9f008200780054
:1015b00083047800000778000fb997000116b8007f
:1015c0008c0578000001eb000c00e00042003200c6
:1015d000010178008fb997000300e0003e0032005f
:1015e0000c00e0002e003200c9009000690090005d
:1015f000808f500004003900090078005a04070069
:101600000000e0002600350019a8a3000600320003
:101610000b017800a10020000e007800f9000700ff
:1016200000057800010037000005eb000b0478008e
:101630000a00e000020032000e0055000004e8003d
:1016400069009000c901900003005000880f50000d
:10165000020031000005eb0000047800080178006a
:101660008e00780003007800950407000807470003
:10167000888555004900900008004000c00498008b
:101680000a00e0000400320009007800930407001b
:101690000000e00002003a000b00e000d2ff3a0038
:1016a00019b8a30002003200090078008b0407007b
:1016b00000c02000190060000200320049009000c4
:1016c000e00498000b0056008fb997001100090044
:1016d0000380d80000017800020078004f077800ee
:1016e0004f06be004f05be004f04be004f00b100c4
:1016f000000006006200fa00889fbe008a9fbe00bc
:101700000004be0002057800830078006a8057005c
:10171000ae040700f88f9f0089979f000000eb0040
:10172000909f9f001a80fb008005fb000000ea00ec
:10173000cf04de000904780050022000808f55009d
:1017400001003a000904e9000800e0000c00340040
:101750000f909700080178008a007800ff899700b1
:101760000300010080979f008080eb000000e000f4
:10177000900032001f98970008004000909f9f0043
:101780000905450050022000808f550004003200fa
:101790000b00e000e3ff3a009f98970085003700b8
:1017a0000000eb00f0979f00e0979f00d0979f000c
:1017b000c0979f00b0979f00a0979f00b09f9f0089
:1017c00009003700a0882000008050000000d000f1
:1017d0000189200001004000bf98970090807000b0
:1017e000b19f9f000a05e8009a00fb00a088200036
:1017f00078040700800078000000e000f1ff3a0064
:10180000a0c2b3009a4f10000e003a003fb89700f4
:101810000080e900b0bf9f0010007800a09f9f00eb
:101820000000e00005003d000000ea00a09f9f00ce
:101830003f9897000020a000b09f9f000a05e80095
:1018400011003700a19f9f000b003700af98970051
:10185000f0ff2700808f5000060032006a09b900af
:101860001a00fb000200400001fd2f0001004000b3
:10187000a09f9f000a05e8001a00fb005d04070016
:101880000000e000f1ff3a00e0c2b3009a4f100000
:10189000030032000080eb00809f9f001c00370097
:1018a000a0c2b300da4f100007003a003fb897001b
:1018b0000080e900b0bf9f0010007800809f9f006b
:1018c0000a05e800120037000000eb00809f9f002f
:1018d0000b0037008f989700f0ff2700808f500093
:1018e000060032006a09b9001a00fb00020040003d
:1018f00001fd2f0001004000809f9f000a05e800c5
:101900001a00fb003b0407000000e000f1ff3a0072
:101910009a00fb00a0a320002e0407008040eb00eb
:101920000000e00001003200ba407800817f9f0093
:1019300080c6b30080cf500004003a009acf100058
:1019400002003a0066405000070037008f78970089
:10195000c0c6b30080cf500005003a009acf1000f7
:1019600003003a0065404000807f9f000a05e800c0
:10197000a0fb2f00008447003a41780088017800de
:10198000ea80570060f92f000f0040001f04070095
:101990000000e00006003a008800780060f92f009f
:1019a0000f004000c90507000000e0005dff3d009a
:1019b0008080eb00010078004f05be004f04be00a0
:1019c0000080fa00000006006900e1000400350014
:1019d0006d00e100030034000002b100010032009c
:1019e0000000050010000500800078001104b1001f
:1019f000030035009101b10001003c000050a0003f
:101a0000000006000200e0000500320090cf100048
:101a1000040032000000e8000201e900fbff3a0088
:101a20000000eb0000000600804680000000e0009f
:101a30000100320000000100e08c200000000600e0
:101a4000889fbe008a9fbe008c1f78000006780029
:101a500081057800100478000005eb0001003700d4
:101a60000804e8001800fb00d7ff07000000e000b2
:101a7000fbff3a0098407800d0c2b30080cf5000fe
:101a800002003a008a00200003003700b0c2b30011
:101a900080cf500001003a000804e8009840780028
:101aa000e2c6b30082cf500003003200e3c4b300ab
:101ab00083cf50001f003a00d840780010c6b30012
:101ac00080cf50000300320010c4b30080cf50001c
:101ad0002a003a00d840780082cf5000030032003c
:101ae000e0c4b30080cf500024003a000804e800ae
:101af000880478004a00200080c2b300984f10008c
:101b000007003a005900fb003e0607000000e00015
:101b1000fcff3a00f0c5b300994f1000f9ff320006
:101b200090c2b300994f10003c003a000904e8004d
:101b30003a00370090c6b30080cf50000300320057
:101b400090c4b30080cf500038003a00584078006d
:101b5000824f500002003200834f500007003a00cd
:101b6000d840780060c6b30080cf50000600320035
:101b700060c4b30080cf5000030032001c04780022
:101b80000005eb00250037003a00b300d84078008c
:101b900093c6b30083cf50000300320090c4b3005b
:101ba00080cf50001d003a008800e8001141780005
:101bb000e0c6b300804f510003003200e0c4b30020
:101bc000804f510015003a0051417800834f510079
:101bd0000300320090c4b300804f51000f003a0060
:101be0005141780040c7b300804f510003003200dc
:101bf00040c5b300804f510008003a0051417800c1
:101c000090c7b300804f51000300320090c5b3006d
:101c1000804f510001003a000104e8000b00e00091
:101c200003003200880d7800010037000a00a00090
:101c3000080e78000a0078004f0678004f05be00b5
:101c40004f04be0000000600e6874700889fbe00e4
:101c50008a9fbe008c9fbe008e1f7800f0b79f0049
:101c60000105780082bf9f00030678008304780096
:101c70006920b900000478008006eb0000c3b300bf
:101c80009a4f100003003a001d002000da4f1000a8
:101c9000fdff32008005eb00000eeb003c167800e3
:101ca00028003700888f550016003d009200200064
:101cb000110009008205d800010078000000e00052
:101cc00003003a00e4844400800ceb00b91478006f
:101cd0001900be00a200200003002000c20e070071
:101ce0001a4178000201fb00cf91de0000004100a4
:101cf000818049000003b1000180b100808cbe00ea
:101d00000d00370010002000010020001c0e4000d4
:101d10005c964800888f550008003a0040c3b30025
:101d20009a4f10000500340012002000030020002c
:101d3000990c4100d99449008b05e8000a05e80098
:101d40001d0020001a00fb002a0307000000e0002d
:101d5000d4ff3a008b0f540001003d008805780045
:101d6000e0c2b3009a4f100001003a000a05e800f3
:101d70000b00e00029003a0000c3b3009a4f1000a6
:101d800026003a000081eb008081eb001c0e410030
:101d90005c9649001d002000da4f1000f9ff320068
:101da0001e003700888f55001a003d009200200069
:101db000110009008205d800010078000000e00051
:101dc00003003a00e4844400800ceb00b91478006e
:101dd0001900be00a200200003002000820e0700b0
:101de0001a4178000201fb00cf91de0000004100a3
:101df000818049000003b1000180b100808cbe00e9
:101e00008b05e8000080eb008080eb001c0e40009a
:101e10005c9648000a05e8001d0020001a00fb003f
:101e2000f40207000000e000deff3a00920020000c
:101e3000110009008205d800010478000800e000c4
:101e400010003200690414001902be00e00f5200b5
:101e5000e08f5a00070032006440b800c2842000be
:101e6000020040001001be000400be005e0e07002c
:101e7000808cbe00888545006140b9001c1e1000a2
:101e80001c961800e88f5500100034001900be00a1
:101e9000e00f5000e08f58000c003a00e985550033
:101ea00090002000010020001c0e40005c964800bd
:101eb000e4845400e88f5500040034001900be008b
:101ec000e00f5000e08f5800f4ff32000d00e000fa
:101ed000310032009a40780050c6b30080cf5000e5
:101ee0000300320050c4b30080cf50002a003a00f3
:101ef000da407800b0c2b30080cf50000400320056
:101f00000047780000c0e80080cf500002003a008f
:101f1000014778000a05e8006044b8008006eb003d
:101f200012003700f00f2e00515f2000800f540088
:101f3000818f5c000b003c00a20020000300200009
:101f40000800be00280e07001a4178000201fb00bd
:101f5000cf91de0000044100818449000803b100f4
:101f60000980b1000a05e8001d0020001a00fb00ee
:101f7000a00207000000e000eaff3a00d0c2b30070
:101f8000804f570002003a0060041400e0841c00f7
:101f90001c0e44005c964c008fb897000100e000d6
:101fa00006003200ffb097000d00e0000100320093
:101fb0008a0078000fb9970001097800920020008c
:101fc000110009008205d8004f0778004f06be00b7
:101fd0004f05be004f04be006f00b10000000600b8
:101fe000e6874700889fbe008a9fbe008c9fbe0088
:101ff0008e1f7800f0b79f000105780082bf9f0018
:1020000083057800030478006720b9008004780015
:102010008006eb0000c3b3009a4f100003003a00a3
:102020001d002000da4f1000fdff32000006eb001b
:10203000800deb00bb1578002e003700890f56008d
:1020400019003d0072002000811f78001100090076
:102050000206d80001007800cf0078000000e00000
:1020600003003a0064044400000ceb0038147800cc
:102070001801be004418dd00cc11de0083017000a1
:102080004411dd000080200000805000718120009c
:1020900060c078000000fb00cf80de00001c410023
:1020a00001944900100037001200200003002000b6
:1020b0009b0d4100db954900890f56000b003a004b
:1020c00000802000008050007181200060c07800f6
:1020d000e74f5000050034001000200001002000f0
:1020e000180c4000589448000c06e8000a05e80067
:1020f0001d0020009a00fb006201200000802000eb
:1021000040fe0700800078000000e000cbff3a00ae
:102110008c8f540001003d0009067800e0c2b30036
:102120009a4f100001003a000a05e8000c00e00098
:102130002c003a0000c3b3009a4f100029003a0067
:102140000081eb008081eb009b0d4100db95490095
:102150001d002000da4f1000f9ff32002100370087
:10216000890f56001d003d0072002000811f78007d
:10217000110009000206d80001007800cf007800a5
:102180000000e00003003a0064044400000ceb008f
:10219000381478001801be004418dd00cc11de00b0
:1021a000830170004411dd00008020000080500099
:1021b0007181200060c078000000fb00cf80de004d
:1021c000001c4100019449000c06e8000081eb006e
:1021d0008081eb009b0d4100db9549000a05e8007a
:1021e0001d0020009a00fb006201200000802000fa
:1021f00004fe0700800078000000e000d8ff3a00ed
:1022000072002000110009000206d80001007800c9
:102210000000e0000d003200670010006402b90009
:102220001801be000402e90003003300020141006e
:1022300083814900fbff3700028cbe000006460088
:10224000cf80de009b1d10009b951800e60f560006
:10225000100034001800be00e00f5000e08f58005e
:102260000c003a00670656007000200001002000b4
:102270009b0d4000db95480064045400e60f5600b7
:10228000040034001800be00e00f5000e08f58003a
:10229000f4ff32001b00be004209dd00ce00de006c
:1022a000810071004200dd00808dbe000d00e00065
:1022b000310032009a40780000c7b30080cf500050
:1022c0000300320000c5b30080cf50002a003a005e
:1022d000da407800b0c2b30080cf50000400320072
:1022e0000047780000c0e80080cf500002003a00ac
:1022f000014778000a05e8006044b8008006eb005a
:1023000012003700f00f2e00515f2000800f5400a4
:10231000818f5c000b003c00a20020000300200025
:102320000800be00300d07001a4178000201fb00d2
:10233000cf91de0000044100818449000803b10010
:102340000980b1000a05e8001d0020001a00fb000a
:10235000a80107000000e000eaff3a00d0c2b30085
:10236000804f570002003a0060041400e0841c0013
:102370009b0d4400db954c008fb997000300e000f3
:1023800006003200ffb097000d00e00001003200af
:102390008a0078000fb897000108780072002000ca
:1023a000110009000206d8004f0778004f06be0052
:1023b0004f05be004f04be006f00b10000000600d4
:1023c000889fbe008a1f7800000578000204be00c6
:1023d000100190004710de0080007800f10fb2007d
:1023e000e14f400006003a00f207b20002003a0056
:1023f0001a00e000190032002000200046003700db
:102400000100e00006003a000a0078000b04070013
:10241000800078000000eb000100e0003e003c007e
:102420006108b9000804400089844800e00f2000da
:10243000800f5400e08f5c000a0034001a00900006
:102440000200200003f82f000000e0000200350029
:102450000200200003f82700028dbe0010002000bb
:102460002d0037009a009000e00f5400e08f5c00d0
:1024700005003400f007280000806000c740dd0040
:102480000100700022003700000028000082600078
:1024900001007800f007b2000070a000100598005d
:1024a00061045400e0845c00f70f4400e08f4c00ae
:1024b00004003d0014059800000deb000000eb0047
:1024c0001500370088017800f00f440004003c003c
:1024d000000d78000000eb0010059800f0014400aa
:1024e0008301ea00080032001a0078000300de00d1
:1024f000f08011001a0190008110dd00010d7000c4
:102500000311de00120598001a009000040070000c
:10251000100598000080eb004f0578004f04be00c6
:10252000000006000200fa00889fbe008a1f7800a3
:10253000000578000204be00800078006880570023
:10254000f20307001a00be000801be00040b0700da
:10255000008dbe004fb99700cf91de000a007800d1
:1025600097ff07004f0578004f04be000080fa0077
:10257000000006000400fa00889fbe008a1f780051
:102580008c9fbe0090bf9f00a1bf9f000204be00b1
:10259000e00f5100e08f59006c0032006011b8006c
:1025a000970c07000000e000680032000c002000db
:1025b0000df82300e00f5400e08f5c0032003d0076
:1025c00060041400e0841c000005eb0011003200e0
:1025d0000808a300070032006450b80002872000fa
:1025e000020040001001be000c00be00dc0a070023
:1025f0000006be008904d1000884d3000a05e80063
:10260000e00f5400e08f5c0002003200e40f550040
:10261000efff36000c01be000000200001f823008f
:10262000b10b07000001be006e805700bdff070020
:10263000000578000000e0003d003d00e00f540080
:10264000e08f5c003a003200224480003344800076
:102650000000200001f82300a30b07000006be00c5
:102660000c01be006e805700aeff07000005780029
:102670000000e0002e003d0061045400e0845c0096
:10268000f7ff3a002a003700e00f5400e08f5c00ab
:10269000270034000005eb000808a3000700320003
:1026a0006450b80002872000020040001001be0004
:1026b0000c00be00aa0a07000006be008984d100f3
:1026c0000884d3000a05e800e00f5400e08f5c00a6
:1026d00002003400e40f5500efff36000c01be008d
:1026e0006e8057008fff0700000578000000e000b3
:1026f0000f003d00e00f5400e08f5c000c00340040
:102700002c4480003d4480000c01be006e805700c8
:1027100084ff0700000578000000e00004003d0091
:1027200061045400e0845c004240a900f6ff3c00d4
:10273000000120000a00e00003003200e10f550014
:1027400002003a0080002000980307001fb897009d
:10275000afb897004f06be004f0578004f04be008b
:102760000080fa0000000600889fbe000004780088
:10277000c0019000600090008000eb00808f51004d
:102780003b0039001801780020002900000061009a
:10279000e20f500009003200020078000090a00013
:1027a0000200e0000200350000202400000071005b
:1027b000000c78008080eb002d003700010026001f
:1027c00001006100810f500008003a0038009000bd
:1027d000808f510005003900080078003f00070095
:1027e0008080eb000000e00021003a0000c02000e3
:1027f0001800600017003a00600220000800400046
:10280000a8049000808f540012003a00002020009d
:10281000aa03070080007800200498000000e00070
:1028200005003a0029049800490498000900e800ce
:1028300030049800060037001860a000400498009b
:102840000020b00030049800410c9800510c980012
:10285000d103070028009000500498003800900031
:102860006004980000002600180c70008000eb0047
:10287000010078004f04be00000006008001eb005c
:1028800010417800814f510001003a00800178002a
:102890000000e8000204e000f9ff3a0003007800bd
:1028a00000000600800078001004e0000200320002
:1028b0005104e000feff3a000080500000000600d6
:1028c000800178000200e00003003200b159780076
:1028d0000201e900fdff3a0000000600889fbe00eb
:1028e000000478000000e0000f003a006044b800e7
:1028f0000800d000817b2100608078000000e000ab
:1029000004003200f5ff07000000e00001003d0078
:102910008084eb000804e80009007800e70f540009
:1029200028003c00f2ff370010d8a300240032003a
:10293000a004900040009000808f54000b003100f4
:1029400009015000384090000000fb008900780029
:10295000730907000000e000110034008084440087
:1029600048009000808f5400f5ff39002800900047
:10297000400498009800780000c0200000806000ab
:1029800002003200a804900001003700b804900053
:1029900001e8a3000900320069049800080037002c
:1029a000a80090004104980061049800510c980020
:1029b0001890a0000080eb0002003700590c98002e
:1029c0000000eb004f04be00000006000108780084
:1029d0000000060090cf1000050032001004e00057
:1029e00001003a0000000500d0cf1000fbff3a00c4
:1029f000000006000003b100030035009000b100a4
:102a000001003c001000050000000500889fbe008a
:102a10008a1f7800000478000102780002457800df
:102a2000830478000200fb00cf80de005002b1007a
:102a30000180b10032052000820f5000e08f580065
:102a400095013e00006001008d01370092013700c2
:102a500091013700900137008f0137008e01370058
:102a60008d0137008c0137008b0137008a01370058
:102a70008901370088013700870137008601370058
:102a80008501370084013700830137008201370058
:102a900081013700800137007f0137007e01370058
:102aa0007d0137007c0137007b0137007a01370058
:102ab0007901370078013700ed00370076013700e3
:102ac0007501370074013700e9003700e80037006e
:102ad000e7003700700137006f0137006e013700e3
:102ae0006d0137006c0137006b0137006a01370058
:102af0006901370068013700670137006601370058
:102b00004b01370064013700630137006201370071
:102b100061013700800037005f0137005e01370038
:102b20005d0137005c0137005b0137005a01370057
:102b30005901370058013700cd00370056013700e2
:102b4000150037001c003700c9003700c8003700e7
:102b5000c700370050013700170037004e0137001b
:102b60004d0137004c0137004b013700ec003700b6
:102b7000690037001f013700470137004601370061
:102b80002b01370044013700630037004201370052
:102b900041013700600037006e01440012007800e8
:102ba000808141009480e900010a78000009e80072
:102bb0009149780041013700a8609000c0c6b30079
:102bc00080cf50000a003a009400780064805000e2
:102bd000000a78001000be004f89de00cf91de00b1
:102be0000002be000203780082037800150037005f
:102bf00010c7b30080cf500002003a0014017800e3
:102c00000400370014017800a0c6b30080cf500044
:102c100005003a0068005100000a78003002be004a
:102c20002003be00070037000280e900000a780098
:102c30001000780000027800cfa2de0005037800c3
:102c400086037800049cbe000694be00a860900035
:102c500080c6b30080cf50000f00320020c6b30002
:102c600080cf500006003a00184078000000fb00ba
:102c7000cf80de0001017800820178000a00370071
:102c800040c7b30080cf50000300320066404000d0
:102c900080cf500006003a0018007800cf80de0098
:102ca0000101780082017800009cbe000294be0001
:102cb0003800be002801be00e00f5000e08f580031
:102cc000e00f5900e08f590004003d006e01440000
:102cd00092007800d0c2b3000c00370008109000ba
:102ce0000018a300040032006e0144009200780036
:102cf000b0c2b300050037000008a300570032003f
:102d00006e0144009200780000c2b30080f47800a5
:102d10000109e80051003700a8609000c0c6b30068
:102d200080cf500006003a00940078006480500084
:102d3000000a78001002be006033b80015003700aa
:102d400010c7b30080cf500002003a001401780091
:102d50000400370014017800a0c6b30080cf5000f3
:102d600005003a0068005100000a78003002be00f9
:102d70002003be00070037000280e900000a780047
:102d800010007800000278000500200006002000f6
:102d900007002000049cbe000694be00a8609000be
:102da00080c6b30080cf50000f00320020c6b300b1
:102db00080cf500006003a00184078000080fb00e9
:102dc0000100200002002000030020000a0037005c
:102dd00040c7b30080cf500003003200664040007f
:102de00080cf500006003a00180078000100200053
:102df0000200200003002000009cbe000294be00e0
:102e0000081090000038a300140032003800be0003
:102e10002801be00e00f5000e08f5800e00f59007d
:102e2000e08f59000d00320080c7b300804f55007d
:102e30000300320080c5b300804f550007003a0000
:102e40006e0044009000780002c3b30082f4780062
:102e50008100e8008af478000108e800780090001a
:102e600000804400600498008a4078006d003700bc
:102e7000a860900014017800c0c4b30080cf500057
:102e800005003a0068005100000a78005001be00b9
:102e90004000be000400370064005100000a7800c2
:102ea0001000be00580a0700009cbe000294be003d
:102eb000380090000000e00004003d006e01440076
:102ec00092007800d0c2b3000c00370008109000c8
:102ed0000018a300040032006e0144009200780044
:102ee000b0c2b300050037000008a300050032009f
:102ef0006e0144009200780000c2b30080f47800b4
:102f00000109e80078009000008044006004980007
:102f10008a407800080078006302070067003700e5
:102f2000286090008000fb00c0062000808f5000c9
:102f3000230032000a003c0064005000808f5000e3
:102f40002600320004003c0066005000808f5000d4
:102f50000b00320021003700a006200005003700da
:102f600040072000808f50001c0032001b003c00f6
:102f700063005000808f50000700320017003700b8
:102f80001480e900000a780010007800485c900086
:102f900008487800490037001480e900000a7800ea
:102fa0001002780068089000cf80de0001017800f0
:102fb00082017800009abe000292be003f003700f6
:102fc0001480e900000a7800100178006808900079
:102fd000cf80de000089be00380037001480e90091
:102fe000000a780010007800680c9000080878004b
:102ff000320037001480e900000a780010007800e1
:10300000cf80de000101780082017800009cbe00c4
:103010000294be0078009000008044006004980094
:1030200081c7b3000800780076040700230037004a
:103030001480e900000a780010007800600498000d
:10304000580990000200e00002003d0015fe070054
:10305000090037008000eb006afa07008000780062
:103060000000e00003003200680090000080500083
:103070000100370058089000100c98000f0037002e
:103080006e0144009200780050c2b30080f17800d5
:103090000109e80009003700ee0044001100780043
:1030a000808144000a4278008008e8000a04e000b9
:1030b00001003a0054c2b300844978000000eb00dc
:1030c0004f0578004f04be00000006000400fa001f
:1030d000889fbe008a9fbe008c1f78000004780085
:1030e0000106780070089000f80090000100500080
:1030f00088089000010050009808900001005000de
:10310000a808900001005000b8089000010050008d
:10311000c8089000810550000002220090bf9f0067
:1031200000032300a0bf9f00081090000028a30008
:1031300018003a000b00e000160034000b05780080
:103140008a047800e20f55000100360029002000b3
:103150000900e0000c00340058009000c801900005
:1031600009017800ee805700030001005004980028
:103170008080eb000000e0009c00320068089000b6
:1031800009004000600c9800090555004240a90064
:10319000ebff3c00780190000200e0000c003400de
:1031a00058009000c80190008c00780003000100d6
:1031b000500498008080eb000000e0008b0032009b
:1031c00068089000f800900001004000600c980032
:1031d000080890000000e0001600340000057800a8
:1031e0008a047800e20f5500010036002900200013
:1031f0000900e0000c00340058009000c801900065
:1032000009017800ec805700030001005004980089
:103210008080eb000000e00074003200680890003d
:1032200009004000600c9800090555004240a900c3
:10323000ebff3c00180990000200e0000c00340095
:10324000e800900058009000c801900003000100c1
:10325000500498008080eb000000e0006300320022
:10326000680890009808900001004000600c9800e9
:10327000280890000000e0001600340000057800e7
:103280008a047800e20f5500010036002900200072
:103290000900e0000c00340058009000c8019000c4
:1032a00009017800ec8057000300010050049800e9
:1032b0008080eb000000e0004c00320068089000c5
:1032c00009004000600c9800090555004240a90023
:1032d000ebff3c00380990000200e0000e003400d3
:1032e000e80090001808900080804000580090008e
:1032f000c801900003000100500498008080eb009a
:103300000000e0003900320068089000b808900022
:1033100001004000600c9800480890000000e000a8
:1033200016003400000578008a047800e20f55008a
:1033300001003600290020000900e0000c003400e4
:1033400058009000c801900009017800ec805700f7
:1033500003000100500498008080eb000000e000b2
:10336000220032006808900009004000600c9800bc
:10337000090555004240a900ebff3c0008109000f1
:103380000028a300180032000b00e00016003400f3
:103390000b0578008a047800e20f55000100360022
:1033a000290020000900e0000c00340058009000c3
:1033b000c801900009017800ee8057000300010069
:1033c000500498008080eb000000e000070032000d
:1033d0006808900009004000600c9800090555003d
:1033e0004240a900ebff3c008000eb0001007800a8
:1033f0004f0678004f05be004f04be000080fa0063
:10340000000006000003b1000b0035009000b10081
:10341000080034008000b100070035009001b100c1
:10342000040034007000b100030035009001b100c9
:1034300001003c001000050000000500800178003c
:10344000900090000000280000836000140020001d
:1034500001007800f007b2009001980002003a00e5
:103460001300e000240032000000e00004003a00f5
:1034700013007800900198008009eb0014ff2f00e2
:1034800093009000f0072000808f50000a003e005b
:103490008100d000130178004f10de0080807000a2
:1034a000910198008209d0000402e900f007200091
:1034b000808f5000f6ff360013019000f50f2000ba
:1034c000850f5100090036001300d100cf10dd0038
:1034d000810970000200d100900198000402e80008
:1034e00000017800850f5000f7ff3e0013009000a8
:1034f000f007b200900198001300900006007000e1
:10350000900198000400780000000600889fbe002b
:103510008004780001047800110090004700de006c
:1035200000017800f20fb200e14f40000a003a00bb
:10353000800ceb0011009000f007b20002003a008e
:103540001100e000020032002000200015003700ca
:1035500010002000130037000200e00005003c00ce
:1035600001007800b5ff0700000178000000e000ce
:103570000a003c0018009000f107280001006000dc
:1035800001f02300010070001004980020f82f00c3
:10359000800c41000080eb0002003700800ceb0043
:1035a0000000eb004f04be00000006008000780021
:1035b00065006000030032001002200070468800a1
:1035c0000000060078806000020032002002200027
:1035d0007046880000000600889fbe0080047800c6
:1035e000d1bf8000010078000100e0000a003a002d
:1035f000c17f2100fc17e2001c003200110078009e
:10360000908f5400140036008080e8001100e00024
:10361000faff3a00150037001100e0000600320002
:1036200011017800928f54000b0036008280e80070
:103630001100e000faff3a0010017800c17f21007c
:10364000e0bf8000820f50000800320011007800b7
:10365000908f540002003e000100780015003700f2
:103660008080e800910f1100f8ff3a00f8bf800059
:10367000890f540001003100090478000800780027
:1036800092030700000178000000e00005003a0006
:103690000000eb00890f5400060032000804d1003e
:1036a000f3ff370008197800020078008e03070046
:1036b000cbff37004f04be0000000600881f7800d3
:1036c000630440000800a1000001eb00800f5400db
:1036d00022003600e30f540001003e0048002000a5
:1036e00008007800bcff0700800078000001eb00b4
:1036f0000000e0001900320010017800920178000b
:1037000064805100880f50000300310012009000c7
:103710008008780007003700080041008008780022
:1037200012029000140098001100780008885100df
:1037300008097800910078000100e00004003200e0
:10374000110090008180e8000000e00001003a00d4
:103750008000eb00d1bf88000281e8000200780001
:103760004f04780000000600881f780088002000c1
:103770000800d000817b2100608078000000e0001c
:10378000010032000a0007000804e900f8ff3700d2
:1037900040bb21008d033700d648e20003003a0009
:1037a000fbff070020c0b300d6e8b700000006000a
:1037b000889fbe000004780048fc07008004780061
:1037c0001868a3000200320028009000460307009a
:1037d0000000eb0020049800384090000004e00056
:1037e000050035000000fb00fb0507000000e000bd
:1037f000010032008084eb00181090000000e0000f
:1038000008003200fd0507000000e0000100320062
:103810008084eb0018109000330307000000eb00d9
:10382000101498001878a3000e0032008000eb00fe
:103830000100d000827b210002004000900f1400a4
:10384000060032008100e800e78f5000f8ff3600e4
:103850000800780024030700100037000008eb0080
:10386000fbff3700000ceb0000c0eb003044980079
:1038700060022000080040002004980040049800e6
:1038800050049800400c980060049800500c980078
:103890007004980076004400000c9800090078003d
:1038a0004f04be0000000600ef04b000889fbe0079
:1038b0008a9fbe008c9fbe008e1f7800c0af9f0005
:1038c000a1df9f0060fa2f000f004000e0af9f00d3
:1038d000cfaa97005503be004502be0084af9f00eb
:1038e00095af9f00a6af9f00b7af9f0010c6b30073
:1038f00080cf50001600320010c4b30080cf5000bb
:10390000130032004fab9700560890000000e00013
:1039100003003d0060002000500b98000c003700b1
:103920000000e0000a003a0070c6b300afdb970069
:1039300080cf53000300320070c4b30080cf530027
:1039400003003a0010002000cfa89700d00898008c
:10395000cfa89700e2fc2f00028047002803070051
:1039600080017800e20f500014003a00cfa99700c0
:10397000e3009000300020009009980010c6b300ca
:103980002fda9700804f52000a0032006440400056
:10399000804f5200070032000040e800804f520084
:1039a00004003200829a20000040e800804f52005c
:1039b00017003a00c29a2000150037000000e0000e
:1039c00018003400cfaa9700e500900030002000d6
:1039d000900a980010c6b3002fdb9700804f530069
:1039e0000a00320064404000804f5300070032005c
:1039f0000040e800804f530004003200029b20008a
:103a00000040e800804f530001003a00429b200034
:103a1000b258780002007800b058780090487800da
:103a2000f201370014c6b300afdb970084cf530018
:103a30000300320010c4b30080cf530010003a00de
:103a40004fa89700ec0040001101780000c3b300bc
:103a5000005978008208e80080c7b300afd897000b
:103a600084cf50000100320080c5b30000497800c7
:103a70004fa99700720090000080e8007001980044
:103a80000300e00003003a008006eb00fda79f0062
:103a9000d001370011c6b300afd9970081cf5100d4
:103aa0000300320010c4b30080cf5100ad003a00d3
:103ab0008e9b20002fda9700814f520001003200c8
:103ac0009e9c2000cfaa9700550890008006e80031
:103ad0000000e00001003d001d0220000d06e8008e
:103ae0004fab97003604be002605be006022b8002a
:103af0006033b8000fa897009fa897002fa99700e0
:103b0000bfa997005f0707000000e00001003d002b
:103b10000bf0a20088af9f0099af9f00aaaf9f0053
:103b2000bbaf9f007fa0970064005000f0a79f00ec
:103b3000efab9700805beb00e7af9f003f003700e3
:103b4000c20120000300200001fd2f00018047007a
:103b5000d90207000faa97009faa97002fab9700e2
:103b6000bfab9700f4af9f0085b79f0096b79f004b
:103b7000a7b79f000400be000601be00460707006d
:103b80000004be000005be00670656004240a900c2
:103b90000c0034006c0707000002be000203be00e8
:103ba0007fa897008fb097001fb19700afb1970023
:103bb0006807070080af9f0091af9f00a2af9f00f2
:103bc000b3af9f00efaa9700e7824200e5af9f00e6
:103bd00070002000e00f5400e08f5c000d00340006
:103be000600020006fab97006f636500e6af9f0039
:103bf000cc5bdd004455de000a857300c4ddde00c9
:103c0000e00f5500e08f5d00020034000000e90085
:103c1000f4ff3b000000e90005003300efa8970027
:103c20008060eb00e1af9f000000e900fbff3b007c
:103c30006fa9970067014100e2af9f000c00e00010
:103c4000090034006022b8006033b8000fa8970064
:103c50009fa897002fa99700bfa997003f070700cb
:103c60000000e000b6ff3c00efa9970064fa2f00c7
:103c70000f024200048051000006e90075fa2f008f
:103c800085824700e5af9f008d0f560001003d0083
:103c90008c0678000d00e0002b0035008c8f56005c
:103ca00005003d006fab970066c07e00f2c0b30018
:103cb000e74f500001003c000041eb008d00e9009f
:103cc000efab970067c07800824f500006003a00c3
:103cd0008d06e9008100e900efa9970063c0780034
:103ce000824f5000faff3200ef4f510004003a00bb
:103cf0006faa970064c078000040e80000f27800e6
:103d00000100e00007003d00efaa97008502e900ee
:103d1000e5af9f008d06e8007fa09700640040009b
:103d2000f0a79f008d00e900070033006fab9700fc
:103d300066c078000000fb006e40780000f3780059
:103d40008100e900f9ff3b00cfab970057089000d6
:103d50000000e0001f013d000d00e900d00b9800bd
:103d60001c0137000fac97009fac97002fad970058
:103d7000bfad97006022b8006033b8000800be00f5
:103d80000a01be00bf0607000000e00005003d007c
:103d90000bf0a20088af9f0099af9f00aaaf9f00d1
:103da000bbaf9f007fa09700725927000280b90027
:103db000026a280013002000b9050700e400500043
:103dc000f1a79f001d003b0063801000c1ff2f0082
:103dd000010460000800ea00f0a79f008004eb00e7
:103de0000800e000470034000808a3000e0032007d
:103df0006848b800c2182100020040003002be002e
:103e00002003be000fa897009fa897002fa9970036
:103e1000bfa99700d606070080af9f0091af9f0013
:103e2000a2af9f00b3af9f000884d1008904e800cf
:103e30000800e000ecff3c00320037000100e00029
:103e4000300034006022b8000600200007ff230085
:103e5000b4b79f00c5b79f00d6b79f00e7b79f00d4
:103e6000c0ff2f0000806000f0a79f0000047800d2
:103e70008004eb00160034000808a3001000320094
:103e80006848b800c5182100050040003002be0097
:103e90002003be003fb09700cfb097005fb19700fe
:103ea000efb19700b20607000002be000203be0099
:103eb000b4b79f00c5b79f00d6b79f00e7b79f0074
:103ec0000884d1008904e8000800e000eaff3c0013
:103ed0003fb29700cfb297005fb39700efb3970060
:103ee0000fa897009fa897002fa99700bfa9970038
:103ef0001407070080af9f0091af9f00a2af9f0003
:103f0000b3af9f004fab9700d608900060c6b300d8
:103f1000afdb970080cf530004003200668740007b
:103f200060c4b30080cf530003003a007fa0970025
:103f3000008040006a074000f30f57000100340082
:103f40003e01200000c3b300efa89700805878001e
:103f5000e1af9f003a0037000800be000a01be0032
:103f60004d0607000006be00f0b79f0081bf9f000e
:103f7000680757004240a9000e003400720607008f
:103f80000002be000203be000800be000a01be001f
:103f9000700607006022b80046782d0077192400cb
:103fa0007306070080af9f0091af9f00a2af9f00f4
:103fb000b3af9f00efa99700e8814100e3af9f00f6
:103fc00088002000e00f5600e08f5e0011003400f2
:103fd00078002000a2002000030020007fb097009e
:103fe0008fb897002a0207006faa970005c3b30095
:103ff00005624100e4af9f00f0b79f0081bf9f00c2
:10400000e00f5000e08f5800020034000804e9007f
:10401000f0ff3b000804e9000600330000c3b300d2
:10402000efab970080637800e7af9f000804e900da
:10403000faff3b006fa8970068004000e0af9f00c8
:104040000e00e0000b0034000fac97009fac97000f
:104050002fad9700bfad97006022b8006033b80065
:104060000800be000a01be003c0607000000e00098
:10407000b9ff3c00efa8970062fa2f000f01410042
:10408000028050000007e90073fa2f008381470087
:10409000e3af9f007fa0970067004000f0a79f005c
:1040a00001c3b30093cf10000a003a000e07e900e5
:1040b0007fa097000000e900f0a79f006faa97007b
:1040c0000402e800e4af9f0014427800814f5200e0
:1040d000f6ff3200cfaa9700d508900060c6b30063
:1040e0002fdb9700804f53000300320060c4b30001
:1040f000804f530004003a007fa0970000804000ea
:104100008006e8000a0037008001eb0050c6b300cb
:10411000afdb970080cf53000300320050c4b300e0
:1041200080cf530001003a00130020008386400036
:104130008d0f570001003d008e0678000d00e00055
:10414000240035008e8f560006003d006fa89700b2
:10415000e0c07e0092c3b30040c3b30080cf5000e4
:1041600001003c0002c3b3008d00e900efa99700f5
:1041700063c07800824f500006003a008d06e900c7
:104180008100e9006faa970064c07800824f500058
:10419000faff320090c3b300804f510004003a0090
:1041a000efaa970065c078000040e80080f2780030
:1041b0000100e00007003d006fab97000603e90037
:1041c000e6af9f008d06e8007fa097000000e800a2
:1041d000f0a79f007fa297008d0178006fa997003c
:1041e000afd897004fa89700c00107004f0778008d
:1041f0004f06be004f05be004f04be00ef04b100e5
:10420000000006006f02b000889fbe008a9fbe00bb
:104210008c9fbe008e1f780080067800f0832000ff
:10422000b0b79f0080c5b30080cf500002003200bd
:10423000e2822000b2b79f0083002000c3b79f0036
:10424000f0c6b30080cf50000a0032006940400041
:1042500080cf500005003200a4002000c4b79f00aa
:1042600080c5b30080cf500002003a00000120005a
:10427000c0b79f008e0120003d04be002d05be008a
:1042800040c6b30080cf50000300320065404000bc
:1042900080cf50000a003a00e00f5400e08f5c002d
:1042a000e00f5d00e08f5d0005003d000800be00ee
:1042b0000a01be007d0607000205be000004be0024
:1042c000e00f5400e08f5c00e00f5d00e08f5d00c8
:1042d00003003a005d0890000000e0000c0032008e
:1042e0007e012000cfb0970001027800cfa2de004f
:1042f00005037800860378000800be000a01be00ae
:10430000000707003fb2970064407800d0e79f00a5
:104310004fb09700cf80de00010178008201780065
:10432000d0b79f00e1b79f00f2b79f0083bf9f0007
:104330000203be000002be000800be000a01be006b
:10434000e9060700809ebe008296be00e00f500086
:10435000e08f5800e00f5900e08f59002200340030
:104360000e00e000200034003d00be002d01be0024
:104370005fb29700efb297007fb397008fbb9700b3
:10438000e40607000205be000004be000e07e900b7
:10439000e1fc2f008f804000010647005fb29700cc
:1043a000efb297007fb397008fbb97000800be0065
:1043b0000a01be00740707001d0010003fb19700fe
:1043c000624e7800889ebe008a96be00e00f5400c0
:1043d000e08f5c00e00f5d00e08f5d0002003400c4
:1043e0000e00e000e0ff3c00cfb19700e88f5100e5
:1043f00010003a000d1090000038a3000d003200ac
:10440000f70f570006003e00e4fc2f000e024200aa
:10441000e4c07f0000c3b30080cf5000050032002d
:104420000e07e90000c3b300e1fc2f008e804000be
:1044300080f07f0078011700920e98006d009000c8
:10444000e3fc2f008f8141008e8041001cf90700a2
:104450001d0e90005d089000800f560006003d0084
:104460000c005000800e98000d1090000040a1003c
:10447000801698000f0037000000e0000d003d009e
:104480000d10900074006000f00f500009003a0019
:104490007d089000fd009000010050008d08900004
:1044a000010050000c0750004240a90001003400f8
:1044b0008e0e98004f0778004f06be004f05be00d5
:1044c0004f04be006f02b100000006000000e000d3
:1044d00003003400d2020700e10f400001003a005f
:1044e0000000eb00000006000000e0003600320093
:1044f0000081e90012027800e30f5200320036001a
:104500000408a30030003a00e1bf80000100e00091
:1045100002003200810f51000300310001087800d1
:10452000e2bf88001d003700810178001100900073
:104530000000e00008003200820f50000600310049
:1045400080017800100090000000e00002003200be
:10455000820f5000faff390093007800018041007b
:10456000800f510018003900820f500003003a00fc
:104570008489400003017800080037009300900010
:104580000100e0000300320004004100808f500071
:104590000d003900110198009201980092009000de
:1045a0000100e000080032009201780003004100a1
:1045b000810f500004003a00fa37ef0010894100e3
:1045c0001000900010019800000006000001780023
:1045d000000020000000e000080032000000800021
:1045e0000000e000050032000000e9000000880043
:1045f0000000d0000100800002b07800000006003a
:10460000889fbe008004780001047800310090008b
:104610000000d0004501de00f07f2000800f510037
:1046200010003a00800ceb00310090006f00600039
:1046300008003a00210090000000e00005003a0068
:10464000110090000000e00002003a001100e000bc
:10465000020032002000200015003700100020006a
:10466000130037000200e00005003c000100780064
:10467000cf010700000178000000e0000a003c00c4
:1046800038009000f10028000100600001fe2300c6
:10469000010070003004980020c02f00800c410001
:1046a0000080eb0002003700800ceb000000eb0004
:1046b0004f04be0000000600881f78008a9fbe00dd
:1046c000000478000205be00300190000200d00016
:1046d000c500de00f07f2000808f50000c003a0003
:1046e0006f00610008003a00280090000000e00020
:1046f00005003a00180090000000e00002003a00b7
:104700001800e0001c003200200020005d0037008f
:104710000100e00006003a0008007800a40107004c
:10472000800078000000eb000100e00055003c0034
:104730006108b9000a0540008b854800e07f200031
:10474000800f5500e08f5d000d00340038009000b0
:104750006022b8000600200007ff2f000000e000e4
:10476000030035006022b8000600200007ff270084
:10477000049cbe000694be001000200041003700db
:10478000b8009000e00f5500e08f5d000500340098
:10479000f000280000806000c450dd0001007000bf
:1047a0003600370000002800808260006f806000c3
:1047b0000040a0003004980061055500e0855d00d0
:1047c000c0fc2f00f1ff2f00800f5500818f5d008e
:1047d00006003d00350498000000eb00200498001e
:1047e00010049800000ceb00260037000a02780045
:1047f000f00f45000b003c0018009000000c780002
:1048000028009000100498003800900020049800c0
:104810000000eb003004980070024200f00f4200ec
:10482000f5ff34000402ea0012003200180178009b
:104830000411de00f0011200180090008300dd007a
:10484000010c71000400de00280190008310dd00df
:1048500001007000100498000411de003800900080
:104860008301dd0003017100220498000400de00d2
:104870003004980038009000050070003004980063
:104880000080eb004f05be004f04780000000600da
:104890000400fa00889fbe008a9fbe008c9fbe0065
:1048a00080bf9f0091bf9f000206be00fc02070070
:1048b0000001be000004be000c00be00ca030700d9
:1048c0000fb997009fb997000005510081855900e5
:1048d0000800be000a01be004f06be004f05be0024
:1048e0004f04be000080fa00000006000a00fa0033
:1048f000889fbe008a9fbe008c9fbe000004780087
:104900000145780082057800830478000406780069
:104910000300e00002003c00190020006ba420000e
:1049200060c6b300804f55000e00320060c4b30073
:10493000804f55000b00320070c6b300804f550009
:104940000300320070c4b300804f550083003a006a
:10495000e40f46008100350058089000800f560093
:104960007e003d000c06e80060c6b300804f550095
:104970001000320060c4b300804f55000d003200bb
:10498000081090000038a30004003a005808900076
:10499000808f540001003d00590c98005808900089
:1049a0000c005000500c980002003b000000eb008f
:1049b000500c98000c00e00027003c00f20144007d
:1049c000130178006800900001c3b3000170790002
:1049d0000201e80082097800580890000000e00019
:1049e00003003c00081090000038a30004003200cf
:1049f000e8009000e0c2b300807079008209e8000e
:104a00000c00ea00d8089000808f500001003d00a3
:104a10000106ea000c00ea00200c98000c8040001f
:104a2000500c9800890f500001003d008004780070
:104a3000680090009808900001004000390c980030
:104a4000090178008b0078009df707005808900056
:104a5000090050001a003700e80090001808900084
:104a60008c8f540018003d00008040000901780040
:104a70008b00780092f707001808900009014000a9
:104a8000120c980009005600200c9800580890005d
:104a90000000e00003003c00081090000038a30074
:104aa00006003200e8009000e0c2b3008070790098
:104ab000380890000000e800300c9800580890007a
:104ac000400c9800a3003700008040000c017800e3
:104ad0008b0078007af70700180890000c0040005f
:104ae000100c98008c845400580890000000e000de
:104af00003003c00081090000038a30006003200bc
:104b0000f20144009300780068019000e0c2b30015
:104b100000f178008109e80058089000890f5000e2
:104b200001003d0080047800680090009808900023
:104b3000010040008c8045000901780060f7070003
:104b40001808900009004000100c980058089000c8
:104b500009005000200c98007e00370070c6b3009a
:104b6000804f55000300320070c4b300804f5500e1
:104b700014003a0058089000808f540004003d0053
:104b8000081090000038a30001003a00590c98006a
:104b9000580890000000e900500c980002003b000b
:104ba0000000eb00500c980051c6b30070c6b30073
:104bb000804f55000100320051c4b3000145780018
:104bc0000900370010c6b300804f550002003a00bc
:104bd0000ac7b3000400370010c4b300804f55006b
:104be00001003a000ac5b300f20144001301780045
:104bf000680090003b7079000201e80082097800ab
:104c0000580890000000e00003003c0008109000ed
:104c10000038a30004003200e8009000e0c2b300b6
:104c2000807079008209e800580890000000e000d8
:104c3000100034008904e900890f500001003d0094
:104c400080047800680090009808900001004000ff
:104c5000090178008b00780019f707001808900008
:104c600009004000100c98005808900009005000fe
:104c7000200c9800e8009000180890008085400003
:104c80008a5d78008b06e8000c00e0000400350027
:104c9000b0c2b300804d78008d0578000400370065
:104ca000d0c2b300804d78008d0578000c06ea0074
:104cb0008004eb000c00e00009003400a10020009b
:104cc0000c0078008d0007007681540001f17f0010
:104cd000000678008904e8000000e000f7ff3c00cf
:104ce000e18f540009003c0050c6b300804f5500ce
:104cf0000300320050c4b300804f550003003a0057
:104d000000c3b300805e78008d0578000900e000e4
:104d100002003a0000c3b300805d78000900e000a3
:104d2000070034008904e900f680540061c07f0068
:104d300002c3b300825d40000900e000f9ff3c00bf
:104d40006800900098089000010040000080550025
:104d5000300c98000810900074006000f00f5000b4
:104d60000e003a0078009000980890000100400082
:104d7000a808900001004000b80890000100400021
:104d8000c80890008100400078089000808f500093
:104d900002003d0001005000000c98004f06be00cc
:104da0004f05be004f04be000080fa000000060060
:104db000000278003000900001002800010360002c
:104dc000150020006f0060003002980008003a00d3
:104dd000240090000000e00005003a00140090005c
:104de0000000e00002003a001400e0003e00320043
:104df000340090000000e0000b003a002400900016
:104e000030029800140090002002980014007800ee
:104e100010029800000aeb00f0825200340090006b
:104e20000000e000f5ff320034009000ef0f50006a
:104e300014003e008001d000a40090004f08de0066
:104e400080817100330298008100d000140190002d
:104e50004f10de0080807000210298000201d00017
:104e6000940078004f08de000001710012029800e3
:104e7000010ad0008502e90003007800ef8f51009d
:104e8000ecff3600b4019000ff8f51001300360094
:104e90001401d10014009000cf00dd00010a710060
:104ea0000000d100a40090004f09dd000200700056
:104eb000100298008100d1004f18dd008080700042
:104ec000210298000300d100300298008502e8001a
:104ed00080017800ff0f5000edff3e00340090008d
:104ee0006f006000300298003400900006007000ef
:104ef00030029800050078000000060001017800eb
:104f000000027800110009000200d8000002fd0034
:104f10000491b900820250000400be0000000600a7
:104f20000a00fa0000027800c3202000e5202000db
:104f30000721200046212000e20f50001b003e0008
:104f4000e0468000e10f50000400320063212000a1
:104f500085212000a7212000e62120001340900099
:104f60000078a30002003a00000beb0013f0a00051
:104f7000154090000028a30001003a0015a0a000f1
:104f8000820178000200e00010003200154090001d
:104f90000008a300fdff32003100fb00800b780009
:104fa0008301e900f9ff3a000800370030002000d3
:104fb000b0bf9f00c4bf9f00d1bf9f00e2bf9f0052
:104fc0006a80570000c0da006fb9970002007800cd
:104fd0000080fa00000006000a00fa00110020001c
:104fe000b1bf9f00c0bf9f006a80570000c0da00b9
:104ff0004fb897000080fa00000006000a00fa008f
:1050000051002000b1bf9f00c0bf9f006a805700c1
:1050100000c0da005fb897000080fa0000000600c8
:10502000889fbe0080047800de08e20005003a0098
:105030000000eb00100007008080eb000000e000a3
:105040000a003500f8468000880078000900e0007a
:105050000600320009004400070007008080eb00d2
:105060000000e000010035008800780001007800b1
:105070004f04be0000000600800078000001eb0035
:105080000000e00003003a0080a42000f046880001
:105090000600370000e32000808f500002003e0031
:1050a000f1468800010037000081eb000200780023
:1050b00000000600889fbe008a9fbe0001057800a0
:1050c0000100e0000400350008003c000000e000a2
:1050d000200032000500370060001000e08018005a
:1050e00002003b0001f02c001a0037000004be0053
:1050f0006011b8006b0920000982cf00020039005e
:105100000882cf000441b000694252000e00320014
:1051100008003b0082817100610164008904d100b4
:105120000884d3008b05e8000442e800f9ff3a0048
:10513000050037000804440089844c008b05e90011
:105140000442e900fbff3a00290107000af0a7002a
:1051500001f0a0004f05be004f04be000000060095
:10516000889fbe008a9fbe008c1f78004601070002
:105170004d01330003866c006450e10024003200ce
:105180006420e100270032006150e100220032007b
:105190006120e100210032008b854200eb07b10065
:1051a0000134b800003ab8000804420089844a007b
:1051b000013ab8000030b8008880400009014a0078
:1051c00004003300000040008180480002014900d3
:1051d0008b05e900c909dd00830170000100320080
:1051e00013002000c814de004814dd004709de006b
:1051f0001200b200c808de0008847000fc0007003e
:1052000001f0a1000cf0a70001f0a0002f01370071
:105210006120e100310132000801be000200be0041
:10522000f7ff37006150e100fcff3a002b01370027
:1052300003f0a200889fbe008a9fbe008c1f7800ea
:1052400011010700180133006450e1004f003200e3
:105250006420e1005200320003826c0007003b0032
:105260000905d0000306d000820f54000c065d0033
:10527000020039000200320089017800030678003c
:105280008582550004003d000003fd008103fd0000
:105290008502ea008b854200840f720002003b0009
:1052a00060001000e08018006011b8000005eb00fd
:1052b0007a28e1000a00390006007800c75ddd00a9
:1052c000f707b200878075002d00370082817100da
:1052d0000a017800610560008180d1000080d30060
:1052e0008502e900f9ff3b0006044000878448007e
:1052f00002003b0060041400e0841c000988a30045
:10530000070032008a8171008281710061016400ae
:105310008904d1000884d3008b05e800170037000a
:105320000978a30013003a000b00e00013003400da
:105330008b05e9000804440089844c000a44740089
:105340000978a3000d003a000b00e00007003400cc
:105350008b05e9000804440089844c0001003a00f0
:105360000b0020000978a300f7ff32000001eb00da
:1053700002003700828171000a0178009c0007005a
:105380000cf0a70001f0a000d00037006420e1007d
:1053900002003a00838f6c00d00033000801be0089
:1053a0000200be00c90037000001be00ce000700a9
:1053b0000470a70003f0a1006509b10016003200d7
:1053c0000d0035006828e10006003500f0ff2f00d1
:1053d000f1ff27000300e00013003b00010028005c
:1053e0000000050000004000818048008502e900bf
:1053f000fcff3a0008003700f88f420002003c0032
:105400008000eb00000005008100d1000080d30087
:105410008502e800fcff3a000300e00002003b00c8
:1054200060001000e080180000000600f4ff2f006c
:10543000c20037000001be00ab0007000470a700e7
:1054400003f0a10003f8a30013003a006509b100be
:1054500010003200090035006928e1000200350023
:105460000100280000000500000040008180480085
:105470008502e900fcff3a0000000600f88f4200b8
:10548000050035008100d1000080d3008502e800ce
:10549000fcff3a00000006008000eb000000050061
:1054a000839f68000100e00002003d0060001000e2
:1054b000e08018000300e00002003d0060011100e0
:1054c000e0811900b80007004f00e00002003b0037
:1054d00060001000e080180000000600b200070025
:1054e0000400be0000000600889fbe008a9fbe0028
:1054f0008c1f7800640007006b00330003866c008b
:105500006450e1002e0032006420e10033003200dc
:105510006150e1002f0032006120e10031003200d3
:1055200085855500eb07b000090020000804200025
:10553000050037000804440089844c000a0031004b
:105540000603430087834b000001530081815b0009
:10555000f8ff33000203be000800a0000804440066
:1055600089844c00f6ff3900c639dd0083017300e1
:1055700001003200130020008904d1000884d30008
:105580000998a300050032000800a7000300a0004e
:105590008904d1000884d3008b05e8008904d10078
:1055a0000884d3000001eb000281d2001000070044
:1055b00001f0a1000cf0a70001f0a00043003700ab
:1055c0006420e100450032000801be000200be0078
:1055d000f7ff37006120e100400032006000b800b2
:1055e000f3ff37000000200001f82700f0ff37002c
:1055f00081002000618055000b003d000b00200061
:1056000061fe2f000100e1001d0034008281710065
:10561000610164008904d1000884d3000000e8001f
:10562000faff3a007100200061006400030070007e
:10563000020060000900320061044400e0844c0074
:105640000988a500050032008b05e8006808e10024
:1056500002003a008904d1000884d300f20f200030
:105660000258e10005003d00c75ddd00f907b2000a
:105670008980750008007800000006000bf82700fc
:105680008b007800000005000004be001600070033
:105690000003be000405be000200be0012000700a9
:1056a000844f7500000006000200be006450e10057
:1056b000050036006420e100020036000968a300fe
:1056c00001003a000800be000160a0004f0678000b
:1056d0004f05be004f04be0000000600f0ff2f0083
:1056e000f1ff2700f9ff3700c70ade00f107b2001b
:1056f000f50fb20008003200e1cf42000200320094
:105700000170a00024000500810f7000010032002c
:105710000408050044000500810f700002003a00f3
:10572000140005008502e9000000400081c0480027
:10573000fcff3b000170a00024000500889fbe0014
:105740008a9fbe00841f7800cfff07004f007800bb
:1057500011003300f0ff2f00838f6c0006003b0028
:10576000040565000a00a7000800370009f0a6003c
:105770001000200008003700820f5400838f5c0067
:10578000030039001000200001003e00000020004e
:1057900009f0a7000000ea004f05be004f04be005c
:1057a0000000e000000006006022b80006022000b1
:1057b0000000d0008180d2000482d2008582d20015
:1057c0000000a0000202520083825a0003003b0046
:1057d0000202420083824a000000a1000603e900a1
:1057e000f3ff3a0000000600020ab900001bb900ee
:1057f0000200b80081004200810043000000060062
:1058000014002000cdff370081037800b6ff0700a9
:105810000001be006000b8000478a30013003a0045
:105820006220e10015003e000d0039008301d10027
:105830000281d3008180d3008301d1000281d30093
:105840008180d3008301d1000281d3008180d30005
:105850000538b000c42add00f300b2008381720075
:1058600007f0a70003f0a00000000600f3ff2700e8
:10587000f2ff2f006110b900fbff370003ff270084
:10588000f7ff37008f1fd100640207008f87e90000
:105890000000e000000006001400fa00889fbe002f
:1058a0008a9fbe008c9fbe000004be000205be00a1
:1058b000680047000a90be000890be008002070002
:1058c0000070a7000bf0a100304320009e02900062
:1058d00080825200b0fe2f000028e10011003d0040
:1058e000b0fc2f000028e100150034001e099000d4
:1058f0008e0890007e0090000501b0000201d100ea
:105900008180d3000080d3008502e800fbff3a00cd
:105910000b00e000a5023b0060001000e0801800d2
:10592000a2023700f0ff2f00f1ff27000b00e0007c
:105930009e023b0001002800000020009b0237006f
:105940006000b800990237004f89de0082017800bc
:105950009b02370007f0a200d0023700809feb00c7
:105960002e0207008f87e9000000e000000006001b
:105970002800fa00889fbe008a9fbe008c9fbe0050
:1059800003866b00750207000028a30064003a003c
:105990000128a30067003a000008a30062003a0053
:1059a0000108a30065003a001e009000be089000a8
:1059b00081064000ed3fb100f4805700ee019000f9
:1059c000111ab8008e099000311bb8009e09900092
:1059d000311cb800511db800f4855700460007007f
:1059e000fe0190003a0007008b85e8003e000700aa
:1059f0008e09900040000700ee019000340007007f
:105a00008b85e800380007008e09900040000700f1
:105a10009e0990001b18b800890440000a854800c0
:105a2000fe019000340007008b85e8003800070075
:105a3000ee019000300007008e0990001b18b8009e
:105a4000890440000a8548000a98a30008003a002b
:105a50000402420085824a0006034b0087834b0004
:105a600008044c0089844c000a054d008d06e900ad
:105a700084827200850273004c3add008502720058
:105a80000100320015002000443ade001400b2008c
:105a90004538de00cb45dd000b007000c540de0060
:105aa000cb4ddd008b8070004549de00cb55dd001d
:105ab0000b017100c551de000d037800f4020700f0
:105ac00003f0a1000cf0a70003f0a000370237009c
:105ad0001b18b8008502400006834800e0834b0095
:105ae00060044c00070037001b18b8000603400094
:105af00087834800faff37001b18b800870340006f
:105b000008844800e0844c0060054d000000060059
:105b10001b18b8000804400089844800faff3700c9
:105b20000108a3001e023a005800be005801be0042
:105b3000e3ff37000008a30019023a0009047800c7
:105b4000f9ff37002800fa00889fbe008a9fbe0038
:105b50008c9fbe0003866b00000207006400e1001a
:105b6000440032006408e1004a0032006100e100b4
:105b7000460032006108e10049003200ec064700af
:105b80006000b8003d02be003d03be00f486570031
:105b90006011b8003d04be003d05be007d0320003d
:105ba0000b0037000000a0008d06e9001300320052
:105bb0000402420085824a0006034b0087834b00a3
:105bc00000004000818048000201490083814900b3
:105bd0000802520089825a000a035b008b835b0033
:105be000f0ff3b000802420089824a000a034b0092
:105bf0008b834b008d06e900edff3a008482720032
:105c000086827200f707b2008782720001003200bc
:105c1000150020001e0490003e0b90000603540067
:105c2000e63fb0000368a300070032000000a700b1
:105c30000500a0008301d1000281d3008180d30040
:105c40000080d3000603e8008301d1000281d30065
:105c50008180d3000080d3000002eb000482d200d8
:105c60008b02070003f0a1000cf0a70003f0a000d6
:105c7000ce013700640247006408e100c801320029
:105c80003400be003401be00f6ff37006108e100b9
:105c9000c30132006011b8006000b800f1ff3700a6
:105ca00003ff270002002000fbff37006000100008
:105cb000e080180060011900e08119000000060072
:105cc000881f7800000478005001be004000be002c
:105cd0000000420081804a0002014b0083814b009a
:105ce000009cbe000294be00dc00070003003100ef
:105cf000480090000000e800400498004f0478003d
:105d000000000600889fbe00000478008004eb00bd
:105d10005001be004000be00d0000700010031006d
:105d20001900200004005000858058000601590029
:105d300087815900009cbe000294be00480090007c
:105d400009005000400498004f04be000000060007
:105d50001200fa00889fbe008a9fbe008c1f780048
:105d60000205be000004be00f4b79f0085bf9f007f
:105d700096bf9f00a7bf9f000000eb00e0b79f0009
:105d8000d0b79f00c0b79f00b0b79f00a0b79f00db
:105d90000006eb005fb197006fb097008000d00065
:105da0000000e00015003d00e1b79f000100780011
:105db0000200e00001003d000000a000ac00070070
:105dc00001003d000000a000af00070001003d0001
:105dd0000000a000b200070001003d000000a0008c
:105de0008100070001003d000000a000b200070094
:105df0007c805700b2ff070014003700e1b79f0016
:105e0000010078000200e00001003d000000a00059
:105e10009700070001003d000000a0009a00070065
:105e200001003d000000a0009d00070001003d00b2
:105e30000000a0006c00070001003d000000a00071
:105e40009d0007007c805700aeff07006fb09700f1
:105e50000000e000070035001000200001002000d5
:105e60006011b80008047000898470000a05710090
:105e70008b8571000c06e800f0032000800f5600af
:105e8000c4ff34006fb097000000e00006003d0042
:105e90007fb297008fba97001fbb9700afbb9700e8
:105ea0007c80570086ff07000802be000a03be0080
:105eb0006fa897000000e00004003a002fb297009e
:105ec000bfb297004fb39700dfb397000400be0046
:105ed0000601be004f0678004f05be004f04be000d
:105ee0000080fa0000000600881f780018002000db
:105ef000881f780096ff07008f87e9004f0478001d
:105f000000000600801feb0091ff07008f87e9006b
:105f1000000006000800fa00889fbe008a9fbe00ad
:105f20008c1f78006e00070005003d00430007004d
:105f3000300007000c003d00330007000b00370065
:105f4000e00f5200e08f5a00e00f5b00e08f5b0033
:105f500006003d000400be000601be0053ff07001e
:105f60000205be000004be001c0020002c0007003b
:105f7000ddff07000c00e000010032004bff0700ce
:105f80004f0678004f05be004f04be000080fa00a7
:105f9000000006000800fa00889fbe008a9fbe002d
:105fa0008c1f78004e00070002003d001c002000fe
:105fb000220007000f00070001003d00120007004b
:105fc00017000700cfff07000c00e00001003200bf
:105fd00036ff07004f0678004f05be004f04be0095
:105fe0000080fa000000060090b79f000100d0007a
:105ff00080b79f00e00f5400e08f5c00e00f5d0071
:10600000e08f5d00000006000800be000a01be002f
:1060100026ff07000205be000004be0000000600c7
:106020000802be000a03be005fb09700efb0970001
:106030007fb197008fb99700000006001bff070093
:106040000100070000000600b0b79f00c1b79f0025
:10605000d2b79f00e3b79f00000006000400e100f4
:106060000588e1000690e1000798e10000000600c5
:10607000c0b79f000200d000b0b79f00afb097003c
:106080000100e00000000600b0b79f000100d00052
:10609000a0b79f009fb097000100e000000006003d
:1060a000a0b79f000100d00090b79f008fb097006d
:1060b0000100e0000000060080b79f000804d00047
:1060c0008984d2000a85d2008b85d2005fb2970006
:1060d000efb297007fb397008fbb970000000600d8
:1060e000d9ff07000605be000404be000006eb0051
:1060f000e00f5000e08f5800e00f5900e08f59008a
:1061000000000600889fbe008a9fbe008c9fbe00d4
:106110000404b8000506b8008904460060854e00f6
:106120000606b8000a054600e0854e000706b800de
:106130008b054600040eb800890446000a854e000f
:10614000050eb8000a0546008b854e00060eb80005
:106150008b0546000416b8000a0546008b854e00e4
:106160000516b8008b054600041eb8008b054600d6
:106170000800be000a01be004f06be004f05be006b
:106180004f04be00000006000800fa00889fbe0011
:106190008a9fbe00170007000605be000404be006b
:1061a000e00f5200e08f5a00e00f5b00e08f5b00d1
:1061b00008003d000400be000601be00bbfe070053
:1061c0000205be000004be000f000700b7fe070076
:1061d000080007000802be000a03be000a0007000c
:1061e000c8ff07004f05be004f04be000080fa0044
:1061f00000000600e0b79f00f1b79f0082bf9f003c
:1062000093bf9f00000006006fb09700ffb097009b
:106210000fb997009fb9970000000600889fbe0045
:106220008a9fbe008c9fbe000404be000605be000f
:10623000809fbe00829fbe004101070004067800d7
:106240000800be000a01be003d0107008406780078
:106250004f03be004f02be008d4f76007fb0970007
:1062600013003300f0ff2f008b8f6b0006003b0004
:106270000d0666000c00a7000a00370007f0a60014
:10628000100020000a003700880f5200898f5a0042
:106290008a0f5b008b8f5b00030039001000200029
:1062a00001003e000000200007f0a7000000ea0007
:1062b0004f06be004f05be004f04be0000000600a2
:1062c000800078005002be005003be004439de005a
:1062d000f700b200f37f20000301610009003200e3
:1062e0000218e10016003a00850172008301730074
:1062f000838173000008200015003a004000200050
:1063000013003700850172008301730083817300dd
:1063100005003a0004a8be0006a8be001000200038
:106320000b0037000201e9000402420085824a00a6
:1063300006034b0087834b000748a300f9ff320098
:106340000740a00004a8be0006a8be002000200050
:106350008000980092009800000006006804470042
:106360000294be000094be00fc0447008694be0068
:106370008494be0009007800d1ff0700080078006f
:10638000cfff070099007800814f70000b003b00a1
:106390000800be00fc0007004f00b10003003700fa
:1063a000f3ff2700f2ff2f006110b9004f06be0077
:1063b0004f05be004f04be000080fa00000006003a
:1063c000889fbe00830478000300e0002c003500a5
:1063d00003003c00008270000402710026003200bd
:1063e00036432000c50020008383cf000a00390017
:1063f0000541b1008283cf00070039000541b1009b
:106400008183cf00040039000541b1008083cf00b3
:10641000010039000541b10085c353006022b80076
:10642000120032000a003b008482720061026000a8
:106430008301d1000281d3008180d3000080d3008a
:106440000603e8008743e800f7ff3a00070037003b
:10645000000040008180480002014900838149001a
:106460000603e9008743e900f9ff3a0088000700c6
:1064700009f0a70003f0a0004f04be0000000600d2
:1064800060001000e080180060011900e081190030
:10649000d3ff3b00033e2c00f7ff37002800fa0033
:1064a000889fbe008a9fbe008c9fbe0007067800b2
:1064b000878669000c003b0003047800870478009d
:1064c00008f0a10009f0a100840f5000858f58004a
:1064d000860f5900890f5c00030033000cf0a20006
:1064e00001003a000cf0a1009cff07006400e100ed
:1064f0005f003200780147006408e100610032006b
:106500006c014700748557003200be001201be00c6
:106510003a04be001a05be001e039000be0a900099
:106520008503530006003d000004fd008104fd00ca
:106530000205fd008305fd008703ea0005037800de
:106540000df8a3000400320060041400e0841c0075
:1065500060051d00e0851d006022b8007d0320005d
:106560000d38e1008006eb000b0039004433dd00fc
:10657000f300b20083017300390037008482720097
:106580000d027800e10664008b85d1000a85d300f6
:106590008984d3000884d3008703e900f7ff3b0018
:1065a00008004000898048000a0149008b814900a9
:1065b00004003b0060001000e0801800600119003a
:1065c000e08119000358a300090032008d82720097
:1065d00084827200610260008301d1000281d300d5
:1065e0008180d3000080d3000603e8001b00370041
:1065f0000348a30017003a000600e000170034002b
:106600000603e9000d00a300000048008180480057
:1066100002014900838149000348a3000f003a00aa
:106620000600e000090034000603e9000000400015
:1066300081804800020149008381490001003a003d
:106640000003eb000348a300f5ff32006022b8000e
:106650000200370084827200618266000c0007002d
:1066600003f0a1000cf0a70003f0a0004fff3700db
:10667000640147006408e10002003a000df8a3003d
:1066800047ff3a003200be001201be0047ff37004c
:106690001800200057002000080453000d003d00a2
:1066a0000600200097fc2f000740e1001e00340088
:1066b00084827200610260008301d1000281d300f4
:1066c0008180d3000080d3000804e800f8ff3a007e
:1066d00047002000610460000504740004046400a5
:1066e0000d00320061004000e08048006001490078
:1066f000e081490003b8a500070032000603e80066
:106700006538e10004003a008301d1000281d30022
:106710008180d3000080d300f87f20000830e100a2
:1067200003003500080378006000b8006011b8006d
:106730004433dd00f300b200830173000000060063
:1067400005ff270005826100070032000428e100f0
:1067500001003200240005000600070001003a0095
:10676000440005000408050002000700f9ff3a0094
:10677000140005006f8261008102700085027100c3
:106780008502720000000600e48240001078a30039
:1067900007003200640240001178a3003400be00fc
:1067a0001401be00040032000330a7000000060000
:1067b0003500be001501be000330a0000000060039
:1067c000881f7800cdc2a900cfc2a9008025200073
:1067d000a240020000000000cdc2a800c0032000bb
:1067e000a240020000000000cfc2bf004600de0051
:1067f00061446000c0122000a240020000000000be
:106800000880fb004f04780000000600cdc2a900fc
:10681000cfc2a90020002000a2400200000000001a
:10682000cdc2a80020002000a2400200000000000d
:10683000cfc2bf004600de00610060000080fb00a8
:1068400000000600cdc2a900cfc2a900e14f500050
:1068500005003a00d0002000a24002000000000025
:10686000cdc2a80003003700d0002000a2400200e3
:1068700000000000f0032000a24002000000000021
:10688000cdc2a80050002000a2400400000000007b
:10689000889fbe008044eb000044eb00dbff070054
:1068a0000004e000040032008880fb00100020009b
:1068b0000100dd0080c4740000052000a240020039
:1068c000000000000844e800e74f5400f3ff3600e2
:1068d0000980fb004f04be0000000600889fbe0038
:1068e000804478000044eb000900fb008880fb0036
:1068f0000180de0061406000d2ff07000844e8002c
:10690000e74f5400f8ff360020082000a2400200a4
:1069100000000000100020004f04be000000060030
:1069200082a22000124068000080fb00810a2f0034
:1069300060c978001280fb0000000600881f780004
:106940000044eb009eff07000004e00006003a0050
:1069500050cab300e1ff07000004e00003003a0062
:1069600098c0b3000100370028c0b3000800fb0046
:106970004f04780000000600881f780000047800ab
:10698000cdc2a900cfc2a90080252000a2400200ec
:1069900000000000cdc2a80080252000a240020017
:1069a0000000000020c3b300004c78004f047800c2
:1069b000000006000000fb00cf80de00eb0f50005f
:1069c000e08f580026003e00006001000b003700f9
:1069d0000c0037000e0037000f00370010003700a2
:1069e0001100370012003700130037001400370081
:1069f000150037001600370017003700801a2f00e7
:106a000001003700501c2f00d407040000000000d4
:106a1000201e2f00fcff370030202f00faff370028
:106a200000242f00f8ff370030262f00f6ff370034
:106a300080282f00f4ff3700702b2f00f2ff370063
:106a4000402e2f00f0ff3700d0312f00eeff37002f
:106a500060352f00ecff370080382f00eaff370049
:106a6000103b2f00e8ff3700889fbe008a1f780088
:106a700080447800020578000044eb00e0c6b300d3
:106a800080cf54000100360038c0b3000804e00095
:106a900011003a0020c3b300914f100003003200f0
:106aa0006b404000914f100003003a00ac0007001b
:106ab000004478000100370058c0b3000804e0002b
:106ac00005003a0012c0b3008a007800094078003f
:106ad000b20007000044780039ff07000800fb00ff
:106ae0004f0578004f04be0000000600889fbe00de
:106af0008a1f780080447800024578000044eb004b
:106b0000e0c6b30080cf54000100360038c0b300a7
:106b10000804e00010003a0020c3b300914f1000b9
:106b2000030032006b404000914f100003003a0018
:106b30008b000700004478000100370058c0b30004
:106b40000804e00004003a008a80fb000980fb0092
:106b5000b30007000044780019ff07000800fb009d
:106b60004f0578004f04be0000000600889fbe005d
:106b70008a1f780080447800020578000044eb000a
:106b8000e0c6b30080cf54000100360038c0b30027
:106b90000804e00010003a0020c3b300914f100039
:106ba000030032006b404000914f100003003a0098
:106bb0006b000700004478000100370058c0b300a4
:106bc0000804e00004003a000980fb008a00780015
:106bd000ad00070000447800f9fe07000800fb0044
:106be0004f0578004f04be0000000600889fbe00dd
:106bf0008a9fbe00800478000045eb008005780085
:106c0000effe07000004e00032003a0030c3b3009a
:106c100032ff07000004e00004003a009ac0b3000d
:106c2000903d2f00d4070200000000000a04e0009d
:106c300019003a000044eb0015ff0700805c780063
:106c40000844e800e74f5400fbff3600803e2f0069
:106c5000801f78000c080200000000000044eb00d8
:106c60008f87e9002980fb00801f780010402f00eb
:106c7000801f78000c08020000000000e487570025
:106c80000844e800e74f5400f6ff360040402f006c
:106c9000d40702000000000080a220000048eb00a2
:106ca0000044eb000880fb006b4078001cff0700ed
:106cb0000844e800e64f5400faff3600fb4090001d
:106cc00080a2200090cf5000030032001ac0b30011
:106cd000010037002ac0b3000a00fb004f05be00c8
:106ce0004f04be0000000600889fbe008a1f780087
:106cf000000578008044eb00b1fe07000004e000ce
:106d000012003a0050c5b300f4fe07000004e00092
:106d100001003a0099c0b3000904e0000c003a00f9
:106d20000044eb000800fb006a407800ebfe07001f
:106d30000004e00001003a0099c0b3000844e800f4
:106d4000e74f5400f7ff34000100370029c0b300bb
:106d50000900fb004f0578004f04be00000006004c
:106d6000881f78000044eb0095fe07000004e00057
:106d700006003a00c0ccb300d8fe07000004e000d3
:106d800003003a0098c0b3000100370028c0b300e8
:106d90000800fb004f04780000000600889fbe003a
:106da0008a9fbe0000447800010578008245780083
:106db0008044eb0090c6b300c8fe07000004e0006a
:106dc00001003a0099c0b3000904e00005003a0050
:106dd00008407800c1fe07000004e00001003a000e
:106de00099c0b3000904e00008003a000044eb0039
:106df0000b04e00005003400a5fe0700005d7800ec
:106e00000844e8008b4f5400fbff3500cbfe070021
:106e10000900fb004f05be004f04be000000060045
:106e2000889fbe008a1f7800804478000145780062
:106e30000044eb00c0c6b300a8fe07000004e00059
:106e400001003a0098c0b3000804e00005003a00d1
:106e500009407800a1fe07000004e00001003a00ac
:106e600098c0b3000804e00002003a000a4078002d
:106e70009afe0700b1fe07000800fb004f057800ee
:106e80004f04be0000000600889fbe008a9fbe001f
:106e9000804478000044eb00480dde008145780016
:106ea000c0c6b3008dfe07000004e00001003a00f8
:106eb00098c0b3000804e00005003a0009407800db
:106ec00086fe07000004e00001003a0098c0b3000d
:106ed0000804e00004003a000a4078007ffe070042
:106ee0000b4078007dfe070094fe07000800fb00c1
:106ef0004f05be004f04be000000060061122000d6
:106f000000222c00da43020000000000e0430200ef
:106f1000000000000000eb00713e20000000e800cf
:106f2000810f5000fdff360000000600e462a8005b
:106f3000e442a8000422ef000622ef0007a2a90005
:106f40000782a8000762a9000742a9000722a8003b
:106f50000702a90006e2a90006c2a80006a2a9002d
:106f6000100320005010880000c7b3009a60b700db
:106f700080cfb3009b60b6008da0a8008dc0a90093
:106f800007e2a8000000060085c0a9000040060036
:106f90003600f800809fbe00829fbe00849fbe0026
:106fa000869fbe00881f7800802020004200f800e5
:106fb00042a0a80042c0a80042e0a800900f7800bc
:106fc000100078004200f900e74060000002b200c3
:106fd0004200de0080c07000eacf500020003a007e
:106fe000705080000000e0000c003a000a440200eb
:106ff000000000000080fb00d0508800a0a120000d
:1070000010c1e9009150800020912000827078002a
:107010001000200070508800050037009850800054
:107020000a440200000000002191200000f47800d2
:107030000782a8009150800000032000808f50003c
:1070400003003c000100e800905088004000370039
:1070500060402f00d4070200000000003c00370011
:10706000e2cf500007003a000a440200000000008e
:107070000000eb006050880070508800805088004d
:1070800032003700e6cf50002a003a0060508000fe
:107090000000e00009003a008e4a020000000000f3
:1070a000a459020000000000e646020000000000b3
:1070b000008e2000104078000500370060508000ee
:1070c000e10f500009003a00008e200010409000af
:1070d00018440200000000000782a80060508000f1
:1070e0000000e8006050880019003700088e20007a
:1070f00080508000080040002040900018440200aa
:10710000000000000782a800805080000000e80016
:10711000805088009800fb00810f50000c003a005e
:10712000ce22a900cc22a90010002000a050880087
:10713000070037000a440200000000000080fb0046
:10714000d05088000000eb00705088000782a80033
:1071500092508000d0508000800f510005003a000e
:1071600010002000b0508800a1c0b3002091200082
:107170000171780085a0a9004f0478004f03be007c
:107180004f02be004f01be004f00be003600f900a6
:1071900000400600881f7800004478001e4402006a
:1071a0000000000006c2bf000008a300fdff3a0077
:1071b000e043020000000000084078002244020082
:1071c0000000000008c2bf000008a300fdff3a0055
:1071d00009c2bf000080fb004700de000080fb000a
:1071e000fbff3a00e0430200000000004f0478007b
:1071f00000000600881f7800004478000080fb0033
:10720000801f780010412f00801f78000c080200ba
:107210000000000008407800224402000000000046
:10722000e487570008c2bf000008a300fdff3a0032
:1072300009c2bf000080fb004700de000080fb00a9
:10724000fbff3a00e0430200000000004f0478001a
:1072500000000600889fbe008a1f78000044780066
:1072600081447800024578001e44020000000000be
:1072700006c2bf000008a300fdff3a0008407800e6
:10728000224402000000000009c2bf000068a30001
:10729000fdff3a0009c2bf000080fb004700de008e
:1072a0000080fb00fbff3a00094078002244020006
:1072b0000000000009c2bf000068a300fdff3a0003
:1072c00009c2bf000080fb004700de000080fb0019
:1072d000fbff3a000a407800224402000000000050
:1072e00009c2bf000068a300fdff3a0009c2bf0049
:1072f0000080fb004700de000080fb00fbff3a003f
:10730000304402000000000006c2bf000028a300b5
:10731000fdff3a00e0430200000000004f05780046
:107320004f04be00000006000800fa00889fbe005f
:1073300000447800d2bf9f00e684570081ff9f0081
:107340008140e80091ff9f00c1f79f001940900025
:10735000d0f79f001e4402000000000006c2bf00dc
:107360000008a300fdff3a00084078002244020014
:107370000000000009c2bf000068a300fdff3a0042
:1073800009c2bf000080fb004700de000080fb0058
:10739000fbff3a004ff0970022440200000000007b
:1073a00009c2bf000068a300fdff3a0009c2bf0088
:1073b0000080fb004700de000080fb00fbff3a007e
:1073c0005ff09700224402000000000009c2bf00e5
:1073d0000068a300fdff3a0009c2bf000080fb0067
:1073e0004700de000080fb00fbff3a003044020053
:1073f0000000000006c2bf000028a300fdff3a0005
:10740000e0430200000000000ff89700c0f79f0063
:1074100099447800d9f79f001e4402000000000044
:1074200006c2bf000008a300fdff3a000840780034
:10743000224402000000000009c2bf000068a3004f
:10744000fdff3a0009c2bf000080fb004700de00dc
:107450000080fb00fbff3a004ff09700224402003f
:107460000000000009c2bf000068a300fdff3a0051
:1074700009c2bf000080fb004700de000080fb0067
:10748000fbff3a005ff0970022440200000000007a
:1074900009c2bf000068a300fdff3a0009c2bf0097
:1074a0000080fb004700de000080fb00fbff3a008d
:1074b000304402000000000006c2bf000028a30004
:1074c000fdff3a00e0430200000000004f04be0050
:1074d0000080fa00000006000e00fa00889fbe003f
:1074e00000447800c2bf9f00d3bf9f00e8845700cc
:1074f000c1f79f000140e800d0f79f0001c0e800fd
:10750000e0f79f00e3c04000f1f79f00e1ef9f002c
:1075100039409000f0ef9f001e4402000000000080
:1075200006c2bf000008a300fdff3a000840780033
:10753000224402000000000009c2bf000068a3004e
:10754000fdff3a0009c2bf000080fb004700de00db
:107550000080fb00fbff3a006fe897002244020026
:107560000000000009c2bf000068a300fdff3a0050
:1075700009c2bf000080fb004700de000080fb0066
:10758000fbff3a007fe89700224402000000000061
:1075900009c2bf000068a300fdff3a0009c2bf0096
:1075a0000080fb004700de000080fb00fbff3a008c
:1075b000304402000000000006c2bf000028a30003
:1075c000fdff3a00e0430200000000006ff097006a
:1075d000e0ef9f0029409000f0ef9f001e44020062
:1075e0000000000006c2bf000008a300fdff3a0033
:1075f00008407800224402000000000009c2bf00d9
:107600000068a300fdff3a0009c2bf000080fb0034
:107610004700de000080fb00fbff3a006fe89700a8
:10762000224402000000000009c2bf000068a3005d
:10763000fdff3a0009c2bf000080fb004700de00ea
:107640000080fb00fbff3a007fe897002244020025
:107650000000000009c2bf000068a300fdff3a005f
:1076600009c2bf000080fb004700de000080fb0075
:10767000fbff3a00304402000000000006c2bf00d9
:107680000028a300fdff3a00e043020000000000d4
:107690005ff09700e0ef9f0019409000f0ef9f002f
:1076a0001e4402000000000006c2bf000008a30044
:1076b000fdff3a000840780022440200000000006c
:1076c00009c2bf000068a300fdff3a0009c2bf0065
:1076d0000080fb004700de000080fb00fbff3a005b
:1076e0006fe89700224402000000000009c2bf00ba
:1076f0000068a300fdff3a0009c2bf000080fb0044
:107700004700de000080fb00fbff3a007fe89700a7
:10771000224402000000000009c2bf000068a3006c
:10772000fdff3a0009c2bf000080fb004700de00f9
:107730000080fb00fbff3a00304402000000000024
:1077400006c2bf000028a300fdff3a00e04302008c
:10775000000000004ff09700e0ef9f009944780090
:10776000f9ef9f001e4402000000000006c2bf00a7
:107770000008a300fdff3a00084078002244020000
:107780000000000009c2bf000068a300fdff3a002e
:1077900009c2bf000080fb004700de000080fb0044
:1077a000fbff3a006fe8970022440200000000004f
:1077b00009c2bf000068a300fdff3a0009c2bf0074
:1077c0000080fb004700de000080fb00fbff3a006a
:1077d0007fe89700224402000000000009c2bf00b9
:1077e0000068a300fdff3a0009c2bf000080fb0053
:1077f0004700de000080fb00fbff3a00304402003f
:107800000000000006c2bf000028a300fdff3a00f0
:10781000e0430200000000004f04be000080fa00b8
:1078200000000600881f7800004478000080fb00fc
:10783000801f780010432f00801f78000c08020082
:10784000000000003444020000000000e4875700fc
:1078500006c2bf000018a300fdff3a0008407800f0
:107860000004a000224402000000000008c2bf0083
:107870000008a300fdff3a0009c2bf000080fb0022
:107880004700de000080fb00fbff3a00e0430200ff
:1078900000000000384402000000000000447800ae
:1078a000484402000000000006c2bf000048a300d8
:1078b000fdff3a00e0430200000000000884fb00e6
:1078c000881f7800f0442f00801f78000c08020009
:1078d00000000000e4875700080078004f0478009b
:1078e00000000600889fbe008044780001447800b4
:1078f0001e4402000000000006c2bf000008a300f2
:10790000fdff3a0009407800224402000000000018
:1079100009c2bf000068a300fdff3a0009c2bf0012
:107920000080fb004700de000080fb00fbff3a0008
:1079300008407800224402000000000009c2bf0095
:107940000068a300fdff3a0009c2bf000080fb00f1
:107950004700de000080fb00fbff3a0034440200d9
:107960000000000006c2bf000018a300fdff3a009f
:107970000940e800224402000000000009c2bf00e4
:107980000068a300fdff3a0009c2bf000080fb00b1
:107990004700de000080fb00fbff3a003844020095
:1079a000000000000044780009c2bf000080fb0016
:1079b0004700de000080fb00fbff3a00304402007d
:1079c0000000000006c2bf000028a300fdff3a002f
:1079d000e0430200000000000880fb004f04be00ee
:1079e00000000600889fbe008a9fbe000005be0002
:1079f0006044b80000c2bf0008c2a90008c2bf00ae
:107a00000048a3001c003a00040037000900780079
:107a10008b0f5400190031000804e80000440200f4
:107a2000000000000004e000f8ff32000004eb005a
:107a300000c2bf00005d78008904e80006a2a9002a
:107a40000682a80006c2bf000048a300fdff3a005e
:107a500006c2bf000068a3000400320007c2bf00d6
:107a60000048a30001003a000782a80008c2bf0036
:107a70000048a300e9ff3200090078004f05be006e
:107a80004f04be0000000600f0002000a010880097
:107a900090cfb3000c62b6000c02a9008d20a800a4
:107aa00000c7b3009860b700f0c3b3000e62b60021
:107ab0008d40a90070c0b3009960b7000de2a80026
:107ac0000f42a800000006000de2a8000004e0003c
:107ad000010032000f42a800000006000004e00090
:107ae000010032000f42a9000de2a90000000600cb
:107af0003600f800809fbe00829fbe00849fbe00bb
:107b0000869fbe00881f78008520a90010003700de
:107b1000985180004e440200000000004194200073
:107b200000f478009151800020062000808f5000e2
:107b300002003c000100e80004003700e0462f008e
:107b4000d4070200000000000000eb009051880004
:107b500062440200000000000004e000ecff3a0074
:107b600090518000419420000100400070f897007f
:107b7000ea4f500002003200ed4f500008003a007a
:107b800090518000e10f500003003c000000eb002a
:107b9000905188000200370010002000a05188009a
:107ba0004f0478004f03be004f02be004f01be00dd
:107bb0004f00be003600f900004006002008980083
:107bc000300898008040eb00015898000000eb005e
:107bd0001052880000000600889fbe000004780054
:107be000801f7800a0472f00801f78000c0802003b
:107bf0000000000038089000801f7800b94a2f006c
:107c0000891f78000c08020000000000280c90007a
:107c1000881f7800891f78000c080200000000000f
:107c2000ec8757004f04be000000060000017800fa
:107c3000005890008001eb00f34f500012003c0010
:107c4000105280000000e8001052880032089000b6
:107c500001487800f300410032089000810f500085
:107c600002003a0032099800030037003208900001
:107c70000000e80030099800025890000040e80039
:107c8000005998001300200003007800000006004f
:107c900000017800005890008000eb000004e00034
:107ca00013003200105280000000e90010528800da
:107cb000a2089000a09d2000114878000258900072
:107cc0000040e90000599800f300410022089000ac
:107cd000810f500002003a0022099800030037008b
:107ce000220890000000e800200998001100200000
:107cf0000100780000000600800078000058900025
:107d00000001eb000004e00004003200a108900034
:107d1000a09d200011487800120020000200780089
:107d200000000600800178002009900030089000d3
:107d3000800f51000c00320092cf100001003a0079
:107d40001000050073804100800f510002003a00ce
:107d500003017800010037000201e80033089000b9
:107d6000800f5100f4ff3a00000005008000780009
:107d7000005890000001eb00f34f50000f003c0052
:107d8000105280000000e800105288003109900075
:107d900073804000800f510002003a00b108980043
:107da00003003700310890000000e800b008980098
:107db000015890000040e8008058980002007800c8
:107dc0000000060000017800014278008041eb00cd
:107dd000005890000004e000130032000104e000ad
:107de00011003400f300410022089000810f500080
:107df00002003a0022099800030037002208900090
:107e00000000e80020099800025890000040e900b6
:107e1000005998008341e8000004e00002003200ad
:107e200084cf5100efff350000000600e5c2a90035
:107e3000614060004600dd00712e20009140780016
:107e40000164a10080c0700001007800e7e2b70083
:107e500000000600e5e2a9004700dd00712e2000c9
:107e6000914078000174a10080c07000010078008a
:107e7000e7e2b70000000600e5c2a900e5e2a900bc
:107e80000000060041c7bf0001cfb3000140600001
:107e9000c040b30041e7b7009140a9004187a80066
:107ea00041c7bf000058a300fdff32008940a90070
:107eb00070c0b300a960b7009140a80000000600a0
:107ec000801f7800c04f8000e40f500004003c0089
:107ed0000000e800c04f88000000eb0003003700fe
:107ee0000000eb00c04f880010002000d04f880039
:107ef0008940a9004f007800004006000080fb0088
:107f000051302c00e10f50000c00320004003c0006
:107f10008100e9000000e0000800320006003700a0
:107f200061302c00e20f5000040032008100e800b4
:107f3000e30f50000100320041302c0080cfb3002d
:107f400032e0b7000000eb000108bb008000240015
:107f5000003b88004200f800000e20004220b700dd
:107f600050052000303b8800a00a2000303b8800ec
:107f700061e7a80000000000000000004200f900d6
:107f800061c7bf000078a300fdff3a0000000600b3
:107f9000c9c2bf004600de006100600000000600ac
:107fa000c9c2bf000080fb004700de000080fb006c
:107fb00000000600000178000080fb00e1cf5000c7
:107fc000010032004810de00000006008001780049
:107fd000e14f5100030032004008de0001002000a4
:107fe000800178000300780000000600889fbe0032
:107ff0000004be0011c0b30009007800edff0700c7
:10800000004c78008040eb0009007800e9ff070091
:10801000104498000884e800080078004f04be006f
:1080200000000600889fbe008a9fbe000004780002
:108030000205be0012c0b3000a00be00e3ff070045
:108040008004780011c0b300daff0700004c78000c
:108050008040eb0009007800d6ff0700104498002c
:108060000041eb000a00be00d8ff07008004780042
:1080700011c0b300cfff0700204498008040eb0000
:1080800009007800cbff07003044980064044400e6
:10809000080078004f05be004f04be000000060037
:1080a0008180fb00c29f2000e14079000140600018
:1080b0000080fb000000ea004f00de000000060028
:1080c0008180fb0042a02000e140790010c86000e0
:1080d0001080fb00000006008180fb00c29f200092
:1080e000e140790010c870001080fb00000006001d
:1080f0000000000000000000000000000000000080
:10810000000000000000000000000000000000006f
:10811000000000000000000000000000000000005f
:10812000000000000000000000000000000000004f
:10813000000000000000000000000000000000003f
:1081400000000600881f7800000478000000eb00a3
:1081500020528800e00f140006003d00e4ff0700f5
:10816000205280000000e80020528800880f500054
:10817000faff35004f04780000000600889fbe001b
:108180000004780049c0b300a00f2000edff0700f5
:108190008944e900fcff3a000804e900f9ff3a00cd
:1081a0004f04be00000006001008880005e1a90089
:1081b00005a1a90004c1a900f0ccb3000461b60078
:1081c0000441a9000421a90095c0bf000054a100ea
:1081d0000045b30095e0b7008460a9008c60a90059
:1081e000000006006008880011e1a90011a1a900a3
:1081f00010c1a90010c1bf000054a1000044a0009c
:1082000010e1b7001021a9001061a90097c0bf00bc
:1082100081cfb300014060000024a00097e0b700c8
:1082200084c0a9008cc0a900000006007008880066
:1082300013e1a90013a1a90012c1a900f0ccb30059
:108240001261b6001221a90097c0bf000064a1000e
:108250000043b30097e0b70084e0a9008ce0a900d8
:1082600000000600d00888001fe1a9001fa1a90096
:108270001ec1a900f0ccb3001e61b6001e61a900aa
:108280001e21a9009ec0bf000064a1000043b300ee
:108290009ee0b70086a0a9008ea0a90000000600fd
:1082a000e008880021e1a90021a1a90020c1a900be
:1082b00000c3b3002061b7002021a9009fc0bf0008
:1082c00081cfb300014060000014a0009fe0b70020
:1082d00086c0a9008ec0a900000006000080fb0037
:1082e000e30f50000f00320005003c00e10f50008a
:1082f00008003200e20f5000080032000f00370083
:10830000e40f500009003200e50f50000900320070
:108310000a00370005e1a9000100370011e1a900ba
:108320001000050013e1a900fdff37001fe1a900bf
:10833000fbff370021e1a900f9ff3700000005002d
:108340000080fb00e30f50000f00320005003c00ee
:10835000e10f500008003200e20f50000800320028
:108360000f003700e40f500009003200e50f500005
:10837000090032000a00370005e1a80001003700bb
:1083800011e1a8001000050013e1a800fdff37006f
:108390001fe1a800fbff370021e1a800f9ff37002b
:1083a000000005000080fb00e30f500011003200c8
:1083b00005003c00e10f500008003200e20f5000c1
:1083c0000900320014003700e40f50000c003200a6
:1083d000e50f50000d0032000f0037008460a90047
:1083e0008c60a9000200370084c0a9008cc0a900dd
:1083f0001000050084e0a9008ce0a900fcff370014
:1084000086a0a9008ea0a900f9ff370086c0a900a8
:108410008ec0a900f6ff3700000005000080fb00b9
:10842000e30f50001100320005003c00e10f500046
:1084300008003200e20f500009003200140037003b
:10844000e40f50000c003200e50f50000d00320028
:108450000f0037008460a9008c60a800020037007c
:1084600084c0a9008cc0a8001000050084e0a90009
:108470008ce0a800fcff370086a0a9008ea0a80011
:10848000f9ff370086c0a9008ec0a800f6ff3700ac
:10849000000005000080fb00e30f50000f003200d9
:1084a00005003c00e10f500008003200e20f5000d0
:1084b000080032000f003700e40f500009003200be
:1084c000e50f5000090032000a0037000021ef00dc
:1084d000010037000621ef00100005000a21ef001f
:1084e000fdff37001421ef00fbff37001821ef00dc
:1084f000f9ff370000000500c602a800c622a80048
:10850000c642a800c662a800c682a800c6a2a800eb
:10851000c702a800c722a800c742a800c762a800d7
:10852000c782a800a1e2a900a802a900a822a90068
:10853000a842a900a862a900a882a900a8a2a9002f
:10854000a8c2a800a8e2a800a902a900a922a9001f
:10855000a942a900a962a900a982a900a9a2a9000b
:10856000a9c2a900a9e2a800a2c2bf000044a100bc
:10857000c042b300a2e2b700a222a900a202a90051
:10858000a682a900a342a800f0f32100501588009c
:10859000a4e2a900a4c2bf0001ccb3000140600066
:1085a0006041b300a4e2b700a5c2bf0001ceb30092
:1085b00001406000c040b300a5e2b700f0c1b300c5
:1085c000a362b600a382a900a202a900014078001c
:1085d000a062b700a042a80000000600c602a800e2
:1085e000c622a800c642a800c662a800c682a8008b
:1085f000c6a2a800c702a800c722a800c742a800b8
:10860000c762a800c782a800c7a2a800a1e2a9006b
:10861000a802a900a822a900a842a900a862a9004e
:10862000a882a900a8a2a900a8c2a800a8e2a80040
:10863000a902a900a922a900a942a900a962a9002a
:10864000a982a900a9a2a900a9c2a800a9e2a8001c
:10865000f0c8b3009960b600aa22ef00a4e2a90016
:10866000a4c2bf0001ccb300014060006041b30070
:10867000a4e2b700a5c2bf0001ceb3000140600074
:10868000c040b300a5e2b700f0c1b300a362b600da
:10869000a382a900a202a900a342a90030ccb30082
:1086a000a262b600a222a900c0cfb300a162b600a8
:1086b00001407800a062b700a042a90000000600b7
:1086c000a1e2a80000000600a1e2a9000000060047
:1086d0006f406000622a20001241780003cfb3008f
:1086e000034161000041710002007800a6e2b7007a
:1086f000e1c06000c408dd00a6c2bf000044a100c4
:1087000001407000a6e2b70000000600800078007b
:10871000030009008018eb000114800001087800b4
:10872000111480001100980021148000210098008d
:1087300031148000310098004114800041009800fd
:10874000511480005100980061148000610098006d
:108750007114800071009800811480000108980055
:108760009114800011089800a1148000210898003d
:1087700000000600a022a800a0c2bf000008a300bd
:10878000fdff320000148000f1ff200001006000b6
:10879000a002a900a022a900000006008560a9008f
:1087a0008d60a800000006008560a9008d60a9000a
:1087b000000006002110880030108800000006002c
:1087c00006c2bf000008a300fdff3a0006c2bf00ba
:1087d0000028a300faff3a0006c2bf000038a30039
:1087e000f7ff3a0006c2bf000048a300f4ff3a00ba
:1087f00009c2bf000068a300f1ff3a0000000600b4
:1088000008c2bf000000d100610060000000fb0052
:108810000000060008c2bf000018a300fdff3200e0
:1088200008c2a90000c2bf000080fb0000000600d3
:1088300002e2b7000782a800000006000602a800b6
:108840000000060002e2b70008c2bf000080fb0083
:108850004700de000000a2000000e9000000060062
:108860000642a800000006000622a800000006003c
:108870000662a80006c2bf000038a300fdff3a0050
:1088800008c2a90000c2bf000080fb000000060073
:1088900006a2a9000682a800000006000cc2bf00c4
:1088a0000000d10063006000e30f500002003a00b6
:1088b0009010800000000600901080000080fb00f7
:1088c000000006000ec2bf00610060000000fb0057
:1088d0000000060000a22000c4f807000000e0002d
:1088e0000e003a000041eb0053c0b300a51f210069
:1088f00014a220008300fb000200fb0060407a000d
:1089000080f07a000241e8008341e900a01f2100c5
:10891000e54f510004003c00f6ff3700c0dc2e009c
:10892000a1e1070090ff2f00000006000200fa00fe
:10893000889fbe000044eb0009cab300668157005f
:1089400001a22000c0c0b30047f807000000fb00f0
:108950000844e800ea4f540003003e00aff89700d7
:1089600089cf5000f5ff3e008080eb000000e00062
:108970000d003a006581570001a22000d0c0b3006d
:1089800039f807000000fb00e1ff2f0006003a0065
:108990002ff897008080fb00c808dd003ff89700a3
:1089a0000080fb0080807000010078004f04be0052
:1089b0000080fa00000006004400de00cf80de00e8
:1089c000bcf1070082862e00f3b92300e4f1070012
:1089d000000006000200fa00889fbe000044eb0081
:1089e00089ccb3006681570001a22000a0c0b3006b
:1089f0001df807008000fb000844e800ea4f54001f
:108a000003003e002ff89700894f5000f5ff3e000d
:108a1000d0ff2f000100e00015003a000044eb00f9
:108a20006581570001a22000b0c0b3000ef8070016
:108a30008000fb000844e800ea4f540003003e00b9
:108a40003ff89700e64f4000f5ff3e00c0ff2f00c3
:108a50000100e00006003a002ff897008080fb003c
:108a6000c808dd003ff897000080fb000080700020
:108a70004f04be000080fa00000006004800de003f
:108a8000000006000200fa000f81e90001a22000a8
:108a9000e0c0b300f4f707000000fb00b1ff2f00b7
:108aa0000d003a000f01e90001a22000f0c0b30060
:108ab000edf707000000fb00a1ff2f0006003a00c1
:108ac0006ff897008080fb00c808dd007ff89700f2
:108ad0000080fb0080807000010078000080fa00b8
:108ae00000000600881f78008a9fbe007aee2300ef
:108af000bb8323000000e00005003500cf80de00ce
:108b00006cf107000a01be0095f107000d00370067
:108b10000004ea006140b90066f107000800e000c7
:108b200003003d000200200003782400c1f107008b
:108b30000a01be008af107000001be006000b80013
:108b4000bbf107004f05be004f047800000006008f
:108b50000200fa000f81e90001a2200080c0b300ea
:108b6000c1f707000000fb00b1ff2f000d003a0025
:108b70000f01e90001a2200090c0b300baf707007e
:108b80000000fb00a1ff2f0006003a006ff89700dd
:108b90008080fb00c808dd007ff897000080fb00a4
:108ba00080807000010078000080fa00000006005c
:108bb000881f78008a9fbe007aee2300bb832300c3
:108bc0000000e00005003500cf80de0039f107002d
:108bd0000a01be0062f107000d0037000004ea0040
:108be0006140b90033f107000800e00003003d00d8
:108bf00002002000037824008ef107000a01be0065
:108c000057f107000001be006000b80088f10700be
:108c10004f05be004f047800000006000200fa0075
:108c20000f81e90001a2200020c0b3008ef70700e9
:108c30000000fb00b1ff2f000d003a000f01e9001a
:108c400001a2200030c0b30087f707000000fb003e
:108c5000a1ff2f0006003a006ff897008080fb000c
:108c6000c808dd007ff897000080fb00808070005e
:108c7000010078000080fa00000006000200fa00ff
:108c80000f81e90001a2200060c0b30076f7070061
:108c90000000fb00b10f200002003a006ff89700bf
:108ca0008080fb00010078000080fa0000000600d0
:108cb00000a2200030f7070000a22000cbf7070039
:108cc0000000cf000000e9004f00de000000e900d6
:108cd000000006000200fa00881f780000447800b7
:108ce0006481570001a220005ff707000000fb002d
:108cf000b1ff2f000d003a000840e80063815700e3
:108d000001a2200058f707000000fb00b1ff2f0070
:108d100006003a004ff897008080fb00c808dd008d
:108d20005ff897000080fb008080700001007800f1
:108d30004f0478000080fa00000006000200fa00ec
:108d40000f81e90001a2200047f707000000fb00a7
:108d5000b10f200002003a006ff897008080fb00fe
:108d6000010078000080fa0000000600881f7800eb
:108d70000181fb000080fb0001a220005bf70700df
:108d8000b10f20000000e00001003a008880fb00e5
:108d9000010078004f04780000000600881f78006a
:108da000010178000080fb0001a220006ff707009e
:108db000b10f20000000e00001003a008880fb00b5
:108dc000010078004f04780000000600e048e2004f
:108dd00003003200ce22a800cc22a9000782a800fe
:108de00000000600889fbe008a9fbe008c9fbe00c8
:108df000098e2000994478000904e00085013200c2
:108e0000e2c8bf000000fb0073e00700e2c8bf003b
:108e10008000fb00f0062000808f50000a003c001c
:108e20000000e900808f500013003d0069005000f1
:108e3000808f50001a0132000080e800808f5000bf
:108e4000850032005301370060072000808f5000fa
:108e5000e300320004003c0064005000808f5000aa
:108e6000460032004b01370080072000808f500001
:108e700037013200470137000044eb000980fb0056
:108e800065005000e00f100015003d00fa0f2000b3
:108e90000980fb00e50450000881fb00408e2000a3
:108ea000e240780081006500c808dd00308e2000b7
:108eb000624078000000fb000a006000809f7000a4
:108ec00060de2e00801f780053e00700e487570023
:108ed00008c4e8000880fb00890f5000eeff350051
:108ee000fcc8bf000003fb00cfb3de00c833dd00c9
:108ef00006002000fbc8bf000000fb00cf80de00a2
:108f0000c000dd000000200002002000f30f200060
:108f1000020060008380600000037300818373009f
:108f2000fac8bf000000fb00cf80de00c808dd00eb
:108f30000080fd00804078000040eb0002f02f0030
:108f400003002000020060008380600000037300c3
:108f500081837300f9c8bf000080fb00010020007e
:108f6000801f7300819f7300a0de2e00801f780099
:108f700029e00700e6875700200137000044eb0096
:108f80000980fb000000e900e00f10001b013d001c
:108f90000980fb008004e9000882fb00608e20004d
:108fa000644078000000fb00cf80de00c803dd00d5
:108fb00006002000508e2000644078000000fb0076
:108fc000cf80de00c000dd00000020000200200095
:108fd000f30f200002006000838060000003730034
:108fe00081837300408e2000644078000000fb0005
:108ff000cf80de00c808dd000080fd0080407800e2
:109000000040eb0002f02f0003002000020060008f
:10901000838060000003730081837300308e200022
:10902000644078000080fb0001002000801f730076
:10903000819f7300f0de2e00801f7800f6df0700ae
:10904000e6875700644444000880fb00890f500005
:10905000d1ff3500e9003700e3c8bf000000fb0086
:10906000801f780060de2e00801f7800eadf070096
:1090700028c0b300e48757000980fb00640050005b
:10908000e20f5000490034004c8e2000fa0f2000ff
:109090003b8e20006dde2e000880fb00e0407e004d
:1090a00081006500c808dd0060c07d000000fb0095
:1090b0000a006000809f70008d1f7800d6df0700d7
:1090c00008c4e8000880fb00e0407e0081006500e5
:1090d000c808dd0060c07d000000fb000a006000e1
:1090e000809f70008d1f7800cbdf070008c4e80068
:1090f0000882fb00608e2000644078000003fb00c3
:10910000cfb3de00c833dd0006002000508e200003
:10911000644078000000fb00cf80de00c000dd006e
:109120000000200002002000f30f20000200600079
:1091300083806000000373008183730064407e00bd
:109140000000fb00cf80de00c808dd000080fd00cd
:10915000804078000040eb0002f02f000300200068
:10916000020060008380600000037300818373004d
:1091700064c07d000080fb0001002000801f7300a0
:10918000819f7300f0de2e00801f7800a2df0700b1
:1091900064444400ee8757008880fb000980fb0090
:1091a00064005000808f5000bbff35000881fb0039
:1091b000408e2000e2407800c808dd00308e20009c
:1091c000624078000080fb00809f700060de2e000f
:1091d000801f780090df0700e48757008700370082
:1091e000e448e20008003500418e200091407800fc
:1091f000c808dd00e3c8bf000080fb00809f70004e
:1092000040df2e0008003700418e2000914078009a
:10921000f107b200c808dd00e3c8bf000080fb0012
:10922000809f700080df2e00801f78007adf0700ab
:10923000e487570028c0b3000980fb000000e90064
:10924000e20f50006d003400fa0f20000980fb008f
:109250008004e9000881fb00408e2000e240780095
:1092600081006500c808dd00308e20006240780073
:109270000000fb000a006000809f700040df2e00ad
:10928000801f780064df0700e487570008c4e80007
:109290000880fb00890f5000eeff350057003700b3
:1092a000648e200014427800c822dd0004002000f3
:1092b000e5c8bf008080fb000000200000027200b3
:1092c00081827200e4c8bf004800dd000100200078
:1092d0000002720081827200368e200016437800f0
:1092e0000683fb0007002000a28e200012417800b8
:1092f000c811dd0002002000e9c8bf008080fb002b
:10930000000020000001710081817100e8c8bf00e9
:109310004800dd0001002000000171008181710022
:10932000e7c8bf000080fb0001002000801f710023
:10933000819f7100861f7200879f7200d0df2e0010
:10934000801f780034df0700ea8757002b003700c2
:1093500038c0b3000980fb000080e800e30f500034
:10936000260034000a8e20000980fb008084e8007b
:109370000880fb0060407d000000fb0016df070056
:109380000844e8000880fb00890f5000f8ff350012
:109390001a0037000044eb000980fb000000e900e0
:1093a000e00f100015003d00fa0f20000980fb00bf
:1093b0008004e9000881fb00408e2000e240780034
:1093c00081006500c808dd00308e20006240780012
:1093d0000000fb000a006000809f700060de2e002d
:1093e000801f78000cdf0700e487570008c4e800fe
:1093f0000880fb00890f5000eeff350060e02e0072
:10940000801f780004df070010002000c051880092
:109410008f87e9004f06be004f05be004f04be0017
:109420000000060040942000630009000058eb0093
:10943000c0ff2f00362ab60000000600409420002e
:10944000630009000058eb00360aa900342aef0037
:109450000000060020912000310009000058eb00b8
:10946000180aa900162aef00000006000002780082
:109470008001eb0010417800ed4f510025003200d3
:10948000ea4f510023003200ed4f5100110032002d
:10949000ea4f51000f003200c0c2b300804f5100ac
:1094a0000c00320000417800f18f510001003c00b7
:1094b000e4f079008301e80064c07900ed4f5000ca
:1094c00004003200ea4f500002003200824f500088
:1094d000f5ff3a000040eb0080f0790064c07900ad
:1094e000ed4f500002003200ea4f500002003a00f7
:1094f0000300420008003700e4c07900c0c2b30096
:1095000080cf500003003a00030042000000e80052
:10951000010037000000eb00000006001400fa0014
:10952000889fbe008a9fbe008044eb00160ae200be
:1095300020003200162aef0031912000914078007f
:10954000c09d2000b9f907000004e00003003a00c4
:10955000a0e02e0094de070018003700c09d200018
:1095600002fa0700800578000000e00013003200d6
:109570001249e2000d0032000004eb001249e20043
:109580000a0034004a912000e8407d00c09d200080
:10959000a6f907008944e8000804e80012c9bf00e2
:1095a0000000fb00800f5400f7ff3500894d780064
:1095b000122aef001000200002003700a5ff07006c
:1095c0000000eb004f05be004f04be000080fa0013
:1095d000000006001400fa00889fbe008a9fbe00ab
:1095e0008c1f78008045eb00340ae20076003200e0
:1095f000342aef004194200091407800c09d200063
:109600008af907000004e00003003a00a0e02e0001
:1096100065de07006e003700c09d2000d3f907000b
:10962000000678000000e00069003200509420003d
:10963000d1c0b30090cf100061003200a2c0b300cf
:10964000904f11005e003200c0c2b3004549e300f4
:109650000b0032000040eb0070fe9f006a94200077
:10966000fe8057000a00780080ff070000057800a0
:109670008045eb000000e00051003200f8ff3700a9
:109680006a942000480037002fe097008000fb001c
:1096900060062000808f50001f00320004003c0054
:1096a0000080e900808f500005003200360037004e
:1096b000c0062000808f50001200320032003700b8
:1096c000a20020008000eb007d8057005ade0700da
:1096d0006104b9004849dd004840de000000710027
:1096e000c8c8de0080407800c09d20004ff9070008
:1096f00088407800c09d20004cf907008bc5e80029
:1097000029003700a20020008000eb007d80570078
:1097100049de0700050037006011b8008000eb004b
:109720007d805700d7de07001fef07000004be0052
:109730004888de00cf80de0080407800c09d200099
:109740003af9070040c8de00cf80de008040780094
:10975000c09d200035f907004849dd004840de0083
:1097600000007100c8c8de0080407800c09d200065
:109770002ef9070088407800c09d20002bf90700d3
:10978000e4c5450008003700a20020008000eb007f
:109790007e80570028de070080407800c09d2000b2
:1097a00022f907008b45e800fe8057000a00780088
:1097b0002eff0700000578000000e000b2ff3a002d
:1097c0000b4e7800322aef00100020000200370014
:1097d0001aff07000000eb004f0678004f05be009f
:1097e0004f04be000080fa0000000600881f7800c9
:1097f00000447800c09d200025f90700084078004b
:10980000da49e300020032000000eb0001003700fb
:10981000100020004f04780000000600881f780028
:1098200000447800140ae20002003a00380ae2001c
:1098300005003200142aef00382aef00008e2000c5
:10984000310009000058eb0010c0b300e7ff07002b
:10985000110020000000e00036003200c09d200012
:109860000bf90700da49e20009003a002005200060
:109870007e0d0700400520007c0d0700a4a8ef0026
:109880003f71ef0020c0b3003ef1b7001f0037006a
:10989000a09d200011c0b30090cf10000c003a0032
:1098a000f0012000e044880050002000f0448800cf
:1098b000a428ef00200520006c0d070040052000c3
:1098c0006a0d070010c0b3003ff1b7001300370066
:1098d000a09d200021c0b30090cf10000d003a00e1
:1098e000f0012000e044880050002000f04488008f
:1098f000a4a8ef00010078003ff1b7002005200088
:109900005a0d070040052000580d070010c0b30095
:10991000020037001100200006003700e0e8b70021
:10992000e168ef0001c2b30001404400e2e8b70083
:109930008000eb00010078004f0478000000060072
:10994000140ae20002003a00380ae2000500320080
:10995000142aef00382aef00008e200031000900a1
:109960000058eb000040eb00a0ff070011002000b2
:109970000000e0000600320040e12e008add070012
:10998000a6db0700b0e32e0087dd07008000eb00b8
:109990000100780000000600889fbe008a9fbe007c
:1099a0008c1f780000447800140ae20002003a009c
:1099b000380ae20005003200142aef00382aef00ce
:1099c000008e2000310009000058eb0010c0b300e9
:1099d00086ff0700110020000000e0006e0032004a
:1099e00050c0b300e0e8b700e168ef00ffc04000fe
:1099f00001404400e2e8b700c09d2000a4f8070041
:109a0000dac9bf000000fb00e20f50001600320070
:109a100005003c000000e0000a003200e10f5000a9
:109a20000d00320052003700e40f500046003200b3
:109a3000e30f500041003400e50f500047003200b2
:109a40004b003700d083800010007800dafb07005d
:109a50000005be000d003700d0838000100090008c
:109a600020fc070003003700d08380002000900016
:109a70004ffc07000005be006011b8006bee070048
:109a80000000e000140035000a00be0069ee070087
:109a90000004be0000067800cf80de0085ed0700e0
:109aa0000800e00003003d000200200003782400cd
:109ab000e0ed07000001be000a00be00dced07007b
:109ac00002002400c3612400a5ed070059ee070041
:109ad00000047800280037000a01be006000b800ca
:109ae000d3ed07000005be0052ee07000004be00e3
:109af00000067800cf80de006eed07000800e00071
:109b000003003d000200200003782400c9ed070097
:109b10000001be000a00be00c5ed070002002400df
:109b2000c36124008eed070042ee070000047800b8
:109b300000002800000676000f003700d083800068
:109b40003006900008003700d0838000400090006d
:109b5000cafb07000006780003003700d0838000ae
:109b6000204890000086fb000004eb000200370054
:109b700011002000080037008c007800308e200093
:109b80001af9070088007800508e200017f90700a6
:109b9000e768ef008000eb00010078004f067800d6
:109ba0004f05be004f04be0000000600881f78006d
:109bb00000447800140ae20002003a00380ae20089
:109bc00005003200142aef00382aef00008e200032
:109bd000310009000058eb000040eb0003ff0700d4
:109be000110020000000e0003e003200b0c1b300d0
:109bf000e0e8b700e168ef00ffc04000014044002a
:109c0000e2e8b700b083800090007800308e20003a
:109c1000f6f80700b083800090009000508e20007e
:109c2000f2f80700b0838000a0009000708e200042
:109c3000eef80700b0838000b0009000908e200006
:109c4000eaf80700b0838000c0009000b08e2000ca
:109c5000e6f80700b0838000d0009000d08e20008e
:109c6000e2f80700b0838000e0009000f08e200052
:109c7000def80700b0838000f0009000108f200015
:109c8000daf80700b083800080089000308f200051
:109c9000d6f80700b083800090089000508f200015
:109ca000d2f80700b0838000a0089000708f2000d9
:109cb000cef80700b0838000b008900061468800ad
:109cc0004008900050468800908f2000c7f8070099
:109cd00051468000b08f2000c4f80700fd68ef00f7
:109ce0008000eb00010078004f04780000000600bf
:109cf000881f780000447800140ae20002003a004d
:109d0000380ae20005003200142aef00382aef007a
:109d1000008e2000310009000058eb000040eb00ed
:109d2000b2fe0700110020000000e0003e003200fb
:109d3000b0c1b300e0e8b700e168ef00ffc0400049
:109d400001404400e2e8b700c08380009000780042
:109d5000308e2000a5f80700c0838000900090009e
:109d6000508e2000a1f80700c0838000a000900062
:109d7000708e20009df80700c0838000b000900026
:109d8000908e200099f80700c0838000c0009000ea
:109d9000b08e200095f80700c0838000d0009000ae
:109da000d08e200091f80700c0838000e000900072
:109db000f08e20008df80700c0838000f000900036
:109dc000108f200089f80700c08380008008900071
:109dd000308f200085f80700c08380009008900035
:109de000508f200081f80700c0838000a0089000f9
:109df000708f20007df80700c0838000b0089000bd
:109e0000614688004008900050468800908f2000ee
:109e100076f8070051468000b08f200073f80700e5
:109e2000fd68ef008000eb00010078004f0478002f
:109e300000000600881f780000447800140ae20041
:109e400002003a00380ae20005003200142aef004e
:109e5000382aef00008e2000310009000058eb0086
:109e60000040eb0061fe0700110020000000e00050
:109e70000e00320050c0b300e0e8b700e168ef0028
:109e8000ffc0400001404400e2e8b70020c0b3003a
:109e9000e3e8b700e468ef0070c0b300e5e8b7009e
:109ea000e668ef00e768ef008000eb000100780053
:109eb0004f04780000000600889fbe008a1f7800cb
:109ec00000457800140ae20002003a00380ae20075
:109ed00005003200142aef00382aef00008e20001f
:109ee000310009000058eb0030c0b3003ffe07000e
:109ef000110020000000e0001b003200c09d200087
:109f000063f70700dac9bf008084fb00c09d200012
:109f10005ff70700a89d200018447800c09d20002e
:109f20005bf70700c840dd00dac9bf000080fb0016
:109f300080807000e78f540004003e000900d000cc
:109f4000c2892000020040000108780010c0b30060
:109f5000e0e8b700e168ef0001c2b300014045004e
:109f6000e2e8b7008000eb00010078004f057800c0
:109f70004f04be0000000600889fbe008a9fbe00fe
:109f800080457800140ae20002003a00380ae20034
:109f900005003200142aef00382aef00008e20005e
:109fa000310009000058eb0080c0b3000ffe07002d
:109fb000110020000000e00033003200c09d2000ae
:109fc00033f70700aa9d20001a457800c09d2000a5
:109fd0002ff70700a99d200099447800c09d20001c
:109fe0002bf70700a89d200018447800c09d200092
:109ff00027f70700a29d2000124178008a427800ce
:10a00000094278008841780031c0b30020c5b30010
:10a01000de0a0700c09d20001df70700aa9d200052
:10a020001a457800c09d200019f70700a99d20005f
:10a0300099447800c09d200015f70700a89d2000d6
:10a0400018447800c09d200011f70700a29d200051
:10a05000124178008a4278000942780088417800ed
:10a0600031c0b30040c5b300c80a070010c0b30038
:10a07000e0e8b700e168ef0001c2b30001c04500ad
:10a08000e2e8b7008000eb00010078004f05be0059
:10a090004f04be0000000600889fbe008044780088
:10a0a000140ae20002003a00380ae2000500320019
:10a0b000142aef00382aef00008e2000310009003a
:10a0c0000058eb0020c0b300c8fd070012002000bc
:10a0d0000000e00042003200c09d2000ecf60700c6
:10a0e000a89d200018447800c09d2000e8f60700d5
:10a0f000a19d2000914078000880fb000300320001
:10a10000e10f5000150032002c003700e5c2a90015
:10a11000e1cf500005003e00e1c06000c608dd0050
:10a12000e7c2bf000064a100120037001200200047
:10a13000e2cf50002a003a00e7c2bf004600de002e
:10a14000020060000000a2004600dd00712e200029
:10a15000914078000164a10014003700e5e2a900f5
:10a16000e1cf500006003e00c708dd00e7c2bf0097
:10a170000074a10001407000e7e2b7001100370051
:10a1800012002000e2cf500015003a00e7c2bf00e5
:10a190000080fb004700de000000a2004700dd0059
:10a1a000712e2000914078000174a10080c07000e1
:10a1b00001007800e7e2b70002003700120020003b
:10a1c0000700370010c0b300e0e8b700e168ef0017
:10a1d00001c2b30001c04400e2e8b7000001eb0097
:10a1e000020078004f04be0000000600889fbe00f9
:10a1f0008a9fbe0080457800140ae20002003a00ff
:10a20000380ae20005003200142aef00382aef0075
:10a21000008e2000310009000058eb0080c0b30020
:10a2200072fd0700110020000000e0003300320042
:10a23000c09d200096f60700aa9d20001a457800d0
:10a24000c09d200092f60700a99d20009944780047
:10a25000c09d20008ef60700a89d200018447800bd
:10a26000c09d20008af60700a29d200012417800c0
:10a270008a42780009427800884178008040eb00eb
:10a2800020c5b300410a0700c09d200080f60700ea
:10a29000aa9d20001a457800c09d20007cf607008a
:10a2a000a99d200099447800c09d200078f6070001
:10a2b000a89d200018447800c09d200074f6070077
:10a2c000a29d2000124178008a427800094278005d
:10a2d000884178008040eb0040c5b3002b0a07009e
:10a2e00010c0b300e0e8b700e168ef0001c2b300be
:10a2f00001c04500e2e8b7008000eb0001007800f3
:10a300004f05be004f04be0000000600889fbe003f
:10a310008a9fbe0080457800140ae20002003a00dd
:10a32000380ae20005003200142aef00382aef0054
:10a33000008e2000310009000058eb0080c0b300ff
:10a340002afd0700110020000000e0003300320069
:10a35000c09d20004ef60700aa9d20001a457800f7
:10a36000c09d20004af60700a99d2000994478006e
:10a37000c09d200046f60700a89d200018447800e4
:10a38000c09d200042f60700a29d200012417800e7
:10a390008a427800094278008841780021c0b300e1
:10a3a00020c5b300f9090700c09d200038f607005a
:10a3b000aa9d20001a457800c09d200034f60700b1
:10a3c000a99d200099447800c09d200030f6070028
:10a3d000a89d200018447800c09d20002cf607009e
:10a3e000a29d2000124178008a427800094278003c
:10a3f0008841780021c0b30040c5b300e3090700dd
:10a4000010c0b300e0e8b700e168ef0001c2b3009c
:10a4100001c04500e2e8b7008000eb0001007800d1
:10a420004f05be004f04be0000000600881f7800e4
:10a4300000447800140ae20002003a00380ae20000
:10a4400005003200142aef00382aef00008e2000a9
:10a45000310009000058eb000040eb00e3fc07006e
:10a46000110020000000e0000b0032002005200059
:10a470007e0a0700400520007c0a070010c0b300d8
:10a48000e0e8b700e168ef0001c2b300014044001a
:10a49000e2e8b7008000eb00010078004f0478008c
:10a4a000000006000800fa00881f780000447800c9
:10a4b000140ae20002003a00380ae2000500320005
:10a4c000142aef00382aef00008e20003100090026
:10a4d0000058eb000040eb00c4fc07001100200016
:10a4e0000000e00026003200ea825700698257002f
:10a4f000e88157006781570031c0b30020c5b30021
:10a50000f6090700e682570065825700e48157008c
:10a510006381570031c0b30040c5b300ef090700a5
:10a5200090c0b300e0e8b700e168ef0001c2b300fb
:10a5300001404400e2e8b7001ff89700e3e8b700e5
:10a540000ff89700e4e8b7007ff09700e5e8b70060
:10a550006ff09700e6e8b7005ff89700e7e8b7000c
:10a560004ff89700e8e8b7003ff89700e9e8b70030
:10a570002ff89700eae8b700eb68ef008000eb00e7
:10a58000010078004f0478000080fa000000060007
:10a590000400fa00881f780000447800140ae200e2
:10a5a00002003a00380ae20005003200142aef00e7
:10a5b000382aef00008e2000310009000058eb001f
:10a5c0000040eb0089fc0700110020000000e000c3
:10a5d00025003200e682570065825700e48157006b
:10a5e0006381570020c5b300bc09070090c0b300c9
:10a5f000e0e8b700e168ef0001c2b30001404400a9
:10a60000e2e8b7005ff89700e3e8b7004ff897007b
:10a61000e4e8b7003ff89700e5e8b7002ff89700a7
:10a62000e6e8b700e682570065825700e4815700ec
:10a630006381570011c0b30040c5b300a7090700ec
:10a640005ff89700e7e8b7004ff89700e8e8b70031
:10a650003ff89700e9e8b7002ff89700eae8b7005d
:10a66000eb68ef008000eb00010078004f047800f9
:10a670000080fa0000000600889fbe008a9fbe008e
:10a6800080457800140ae20002003a00380ae2002d
:10a6900005003200142aef00382aef00008e200057
:10a6a000310009000058eb0080c0b3004ffc0700e8
:10a6b000110020000000e00031003200c09d2000a9
:10a6c00073f50700aa9d20001a457800c09d200060
:10a6d0006ff50700a99d200099447800c09d2000d7
:10a6e0006bf50700a89d200018447800c09d20004d
:10a6f00067f50700dac9bf000a82fb008981fb0009
:10a700000881fb008080fb0020052000cd080700a9
:10a71000c09d20005ef50700aa9d20001a45780024
:10a72000c09d20005af50700a99d2000994478009b
:10a73000c09d200056f50700a89d20001844780011
:10a74000c09d200052f50700dac9bf000a82fb0055
:10a750008981fb000881fb008080fb004005200010
:10a76000b808070010c0b300e0e8b700e168ef00e8
:10a7700001c2b30001c04500e2e8b7008000eb0071
:10a78000010078004f05be004f04be000000060027
:10a79000889fbe008a9fbe0080457800140ae200b0
:10a7a00002003a00380ae20005003200142aef00e5
:10a7b000382aef00008e2000310009000058eb001d
:10a7c00080c0b30009fc0700110020000000e00079
:10a7d00033003200c09d20002df50700aa9d200007
:10a7e0001a457800c09d200029f50700a99d20008a
:10a7f00099447800c09d200025f50700a89d200001
:10a8000018447800c09d200021f50700a29d20007b
:10a81000124178008a427800094278008841780025
:10a8200011c0b30020c5b300d8080700c09d2000a8
:10a8300017f50700aa9d20001a457800c09d20004a
:10a8400013f50700a99d200099447800c09d2000c1
:10a850000ff50700a89d200018447800c09d200037
:10a860000bf50700a29d2000124178008a42780073
:10a87000094278008841780011c0b30040c5b30098
:10a88000c208070010c0b300e0e8b700e168ef00bd
:10a8900001c2b30001c04500e2e8b7008000eb0050
:10a8a000010078004f05be004f04be000000060006
:10a8b000e4874700889fbe008a9fbe008c9fbe0031
:10a8c0008e1f780000447800140ae20002003a006b
:10a8d000380ae20005003200142aef00382aef009f
:10a8e000008e2000310009000058eb0010c0b300ba
:10a8f000befb0700110020000000e000470032000e
:10a90000c09d2000e2f40700dac9bf0080f79f0075
:10a910000040e90011002000e44f50003f003e00dd
:10a92000d0c2b300e0e8b700e168ef00ffc040002c
:10a9300001404400e2e8b7000ff197000280fb00fd
:10a940000000d000a11e210001004000100078008e
:10a9500090007800308e2000a4f507000047eb003f
:10a960000ff197000280fb000000d000a11e210023
:10a97000810540000e84fb000805d0009b004500c7
:10a980006846b900528e200002004600b1009000d7
:10a9900096f507001b054500718e2000010046005a
:10a9a0008a08900091f507006444b8001b04440035
:10a9b0007a04440018017800624688001804900068
:10a9c00058468800918e20000100460082007800e1
:10a9d00086f50700b28e2000020046005146800036
:10a9e00082f507000e47e800e44f5700e1ff36000c
:10a9f0008ff097000180fb000000d000a21e210014
:10aa00000200400010007800a0009000d0902000cc
:10aa100076f507000f69ef008000eb000100780079
:10aa20004f0778004f06be004f05be004f04be0022
:10aa30004f00b10000000600881f78000044780035
:10aa4000140ae20002003a00380ae200050032006f
:10aa5000142aef00382aef00008e20003100090090
:10aa60000058eb000040eb0060fb070011002000e5
:10aa70000000e0000a00320010c0b300e0e8b700b8
:10aa8000e168ef00ffc0400001404400e2e8b70089
:10aa9000e368ef00c028ef00c228ef008000eb0061
:10aaa000010078004f04780000000600889fbe0077
:10aab0008a9fbe0080457800140ae20002003a0036
:10aac000380ae20005003200142aef00382aef00ad
:10aad000008e2000310009000058eb0030c0b300a8
:10aae00042fb0700110020000000e0001d003200c2
:10aaf000c09d200066f40700aa9d20001a4578003a
:10ab0000c09d200062f40700a99d200099447800b0
:10ab1000c09d20005ef40700a89d20001844780026
:10ab2000884178000a4178008940780020c5b30048
:10ab3000dc070700884178000a41780089407800e6
:10ab400040c5b300d707070010c0b300e0e8b70066
:10ab5000e168ef0001c2b30001c04500e2e8b700c0
:10ab60008000eb00010078004f05be004f04be00de
:10ab700000000600889fbe008a9fbe008c9fbe001a
:10ab800000447800140ae20002003a00380ae200a9
:10ab900005003200142aef00382aef00008e200052
:10aba000310009000058eb0080c0b3000ffb070024
:10abb000110020000000e0003c0032001cc0b30087
:10abc0000c007800e0e8b700e168ef0000c2b300d5
:10abd000804544000b007800e2e8b700e368ef002e
:10abe000c09d20002af40700dac9bf00c806dd00b6
:10abf000c09d200026f40700dac9bf000000fb005a
:10ac000080867600c09d200021f40700aa9d2000c8
:10ac10001a4578004855dd00c09d20001cf407004f
:10ac2000dac9bf000000fb0000057500c09d2000d0
:10ac300017f40700a99d200099447800c84cdd0056
:10ac4000c09d200012f40700dac9bf000000fb001d
:10ac500080847400c09d20000df40700a89d200092
:10ac6000184478004844dd00c09d200008f4070027
:10ac7000dac9bf000000fb00000474000802be0037
:10ac80008a0178000d01780041c5b30020c5b300ea
:10ac9000b70807000c007800e0e8b700e168ef00b3
:10aca0000b007800e2e8b7008000eb0001007800bc
:10acb0004f06be004f05be004f04be000000060058
:10acc000881f7800140ae20002003a00380ae20005
:10acd00005003200142aef00382aef00008e200011
:10ace000310009000058eb0020c0b300bffa070094
:10acf000110020000000e00026003200c09d20006e
:10ad0000e3f30700a89d2000184478000804fb0026
:10ad1000c09d2000def307004844dd00dac9bf0013
:10ad20000080fb0000047400d0e42e009ed80700d1
:10ad3000803e200011f5070000e52e00801f7800fe
:10ad4000b5d80700803e20000cf50700881f78006a
:10ad500040e52e00801f7800afd80700a0e62e0047
:10ad600091d80700e0e72e008fd8070010e92e00e9
:10ad70008dd8070040ea2e008bd80700c05d200068
:10ad8000fef40700d0ea2e0087d807008000eb0011
:10ad9000e6875700010078004f04780000000600a5
:10ada0000800fa00889fbe0000447800140ae20000
:10adb00002003a00380ae20005003200142aef00cf
:10adc000382aef00008e2000310009000058eb0007
:10add0000040eb0085fa0700110020000000e000b1
:10ade000a600320010c4b300e0e8b700e168ef004d
:10adf000ffc0400001404400e2e8b700c08380008b
:10ae000090007800308e200078f40700c083800026
:10ae100090009000508e200074f40700c0838000e2
:10ae2000a0009000708e200070f40700c0838000a6
:10ae3000b0009000908e20006cf40700c08380006a
:10ae4000c0009000b08e200068f40700c08380002e
:10ae5000d0009000d08e200064f40700c0838000f2
:10ae6000e0009000f08e200060f40700c0838000b6
:10ae7000f0009000108f20005cf40700c083800079
:10ae800080089000308f200058f40700c0838000b5
:10ae900090089000508f200054f40700c083800079
:10aea000a0089000708f200050f40700b08380004d
:10aeb00090007800908f20004cf40700b083800051
:10aec00090009000b08f200048f40700b08380000d
:10aed000a0009000d08f200044f40700b0838000d1
:10aee000b0009000f08f200040f40700b083800095
:10aef000c0009000109020003cf40700b083800058
:10af0000d00090003090200038f40700b08380001b
:10af1000e00090005090200034f40700b0838000df
:10af2000f00090007090200030f40700b0838000a3
:10af300080089000909020002cf40700b0838000df
:10af400090089000b090200028f40700b0838000a3
:10af5000a0089000d090200024f40700ec82570055
:10af60006b825700ea8157006981570031c0b300f6
:10af700020c5b30059070700e882570067825700d1
:10af8000e68157006581570031c0b30040c5b3006a
:10af9000520707007ff097000fe9b7006ff09700a6
:10afa00010e9b7005ff0970011e9b7004ff0970084
:10afb00012e9b7003ff8970013e9b7002ff89700a0
:10afc00014e9b7001ff8970015e9b7000ff89700cc
:10afd00016e9b700ec8257006b825700ea815700f0
:10afe0006981570011c0b30020c5b3003b070700bb
:10aff000e882570067825700e68157006581570055
:10b0000011c0b30040c5b300340707007ff09700bc
:10b0100017e9b7006ff0970018e9b7005ff09700e5
:10b0200019e9b7004ff097001ae9b7003ff8970009
:10b030001be9b7002ff897001ce9b7001ff897002d
:10b040001de9b7000ff897001ee9b7000146800020
:10b050000846800019468000404cde0009002000b0
:10b06000f0912000e1f307008800780010922000a2
:10b07000def307002369ef008000eb000100780099
:10b080004f04be000080fa0000000600889fbe004a
:10b0900000447800140ae20002003a00380ae20094
:10b0a00005003200142aef00382aef00008e20003d
:10b0b000310009000058eb0010c0b300cbf90700c5
:10b0c000110020000000e0001500320020c0b30095
:10b0d000e0e8b700e168ef00ffc040000140440035
:10b0e000e2e8b700c09d2000e9f20700a99d20001a
:10b0f000994478000044eb000844e8000980fb0014
:10b100000ef70700e14f400002003a00fd4f5400e7
:10b11000f9ff3600e3e8b700e568ef008000eb00d8
:10b12000010078004f04be0000000600881f780070
:10b1300000447800140ae20002003a00380ae200f3
:10b1400005003200142aef00382aef00008e20009c
:10b15000310009000058eb0020c0b300a3f907003c
:10b16000110020000000e0001300320010c0b30006
:10b17000e0e8b700e168ef00ffc040000140440094
:10b18000e2e8b700c09d2000c1f20700a89d2000a2
:10b1900018447800c09d2000bdf20700a19d20004a
:10b1a000914078008180fb000880fb00eff60700eb
:10b1b000e568ef008000eb00010078004f047800a4
:10b1c00000000600889fbe0000447800140ae200d8
:10b1d00002003a00380ae20005003200142aef00ab
:10b1e000382aef00008e2000310009000058eb00e3
:10b1f0000040eb007df90700110020000000e00096
:10b200004300320010c0b300e0e8b700e168ef008f
:10b21000ffc0400001404400e2e8b70020c0b30096
:10b2200060f4070020c0b3002cf407000044eb00da
:10b230000844e80010002000c0f60700e14f40007d
:10b2400002003a00fd4f5400f9ff36000044eb00c5
:10b250000844e800e101200000012000c3f60700d7
:10b26000a0002000c5f3070000012000b3f607008e
:10b27000fe4f500002003200fd4f5400f4ff360034
:10b280000044eb0009cab3000844e800010a2000aa
:10b2900010012000b5f60700a0002000b7f307005a
:10b2a00010012000a5f6070080cf540002003200f4
:10b2b000fd4f5400f4ff36000044eb0039c7b300e3
:10b2c0000844e8003107200000022000a7f607002c
:10b2d000a0002000a9f307000002200097f6070055
:10b2e00080cf540002003200fd4f5400f4ff3600be
:10b2f000b0eb2e002cd7070020c0b30047f40700a6
:10b3000020c0b3000ef40700e568ef008000eb00fa
:10b31000010078004f04be0000000600c09d200020
:10b320005bf207000004e000fcff3a0010c0b3002d
:10b33000e0e8b700e168ef0040c2b300e2e8b70020
:10b34000e368ef0000000600140ae20002003a0081
:10b35000380ae20005003200142aef00382aef0014
:10b36000008e2000310009000058eb00c09d200035
:10b3700047f207000004e000ba003200dac9bf005b
:10b380000000fb00cf80de00a2052000820f5000ed
:10b39000e08f5800a9003e0000600100a5003700c2
:10b3a000a6003700a5003700a4003700a30037002f
:10b3b000a2003700a1003700a00037009f0037002f
:10b3c0009e0037009d0037009c0037009b0037002f
:10b3d0009a0037009900370098003700970037002f
:10b3e000960037009500370094003700930037002f
:10b3f0009200370091003700900037008f0037002f
:10b400008e0037008d0037008c0037008b0037002e
:10b410008a0037008900370088003700870037002e
:10b42000860037008500370084003700830037002e
:10b430008200370081003700800037007f0037002e
:10b440007e0037007d0037007c0037007b0037002e
:10b450007a0037007900370078003700770037002e
:10b46000760037007500370074003700730037002e
:10b470007200370071003700700037006f0037002e
:10b480006e0037006d0037006c0037006b0037002e
:10b490006a0037006900370068003700670037002e
:10b4a000190037001b0037001d0037001f00370050
:10b4b0002100370023003700250037002700370020
:10b4c000290037002b0037002d0037002f003700f0
:10b4d00031003700330037003500370037003700c0
:10b4e000390037003b0037003d0037003f00370090
:10b4f0004d003700430037003f003700440037005d
:10b500004e0037004500370010c4b300c3f80700f1
:10b510004b00370020c4b30046fa0700480037004c
:10b5200030c4b30064fa07004500370040c4b300dc
:10b5300091fa07004200370050c4b300d9fb07005e
:10b540003f00370060c4b30070fb07003c003700c9
:10b5500070c4b300d6fc07003900370080c4b300c4
:10b5600084fd07003600370090c4b30042fc07009a
:10b5700033003700a0c4b3004cfd07003000370093
:10b58000b0c4b300c4fa07002d003700c0c4b30034
:10b5900016fb07002a003700d0c4b300a3fb070046
:10b5a00027003700e0c4b300d1f9070024003700ba
:10b5b000f0c4b3007df907002100370000c5b300d7
:10b5c00073fc07001e00370010c5b300bcfd070068
:10b5d0001b00370020c5b300edfb07001800370043
:10b5e00030c5b300a9fe07001500370040c5b30001
:10b5f000cefe07001200370070c5b300f1fe070051
:10b600000f00370060c5b300e3f807000c003700f7
:10b6100080c5b300e2fd070009003700a0c5b300f4
:10b6200005fd07000600370050c5b300c4f8070049
:10b63000030037000040eb000100370010c0b300ea
:10b640000004e0000300320034ff0700010037006f
:10b6500000000000c09d20008df107000004e00004
:10b66000fbff3a00000006001a00fa00889fbe00a7
:10b670008a9fbe008c9fbe003f71ef00e013210047
:10b6800011c0b30090cf100009003a00c1838000c0
:10b6900031009000b2122000820f500071013e0074
:10b6a00041009000820f50006e013e000400370000
:10b6b000e013210021c0b30090cf10003d003a00fc
:10b6c0003e71ef004031ef00f48257007382570063
:10b6d000f28157007181570011c0b30020c5b3003b
:10b6e0007e0507004fe99700c811dd000200200029
:10b6f0005fe897008080fb000000200000017100df
:10b70000818171006fe897004800dd000100200092
:10b7100000017100818171007fe897000080fb00cb
:10b72000010020000001710081817100a2458800a4
:10b73000b3458800f482570073825700f2815700a6
:10b740007181570011c0b30040c5b3006305070005
:10b750004fe99700c811dd00020020005fe8970064
:10b760008080fb00000020000001710081817100d9
:10b770006fe897004800dd00010020000001710023
:10b78000818171007fe897000080fb0001002000ac
:10b790000001710081817100c2458800d345880095
:10b7a000a0458000b1458000604588007145880053
:10b7b0002a0137006033b80086bf9f0097bf9f0003
:10b7c0000002eb00c3838000853e2000e8152000c6
:10b7d0008400d00003804000908f120004003600e7
:10b7e000a2fd2f000101410008b17f0012003700c7
:10b7f0000401d00083004100b0122000910f10001e
:10b8000005003e00a1fd2f008f8040000100410097
:10b810000008eb00080037008400d00003804000df
:10b8200042ed2f00100041000000d100a9fd2f00c3
:10b830008184440080b47f000402e800e80f5200d5
:10b84000e3ff34000002eb0068102100450f2100e7
:10b850000401d000a9fd2f008f844400890141001c
:10b8600062007c001380b900cf80de000603400038
:10b870008783480062807a001380b900cf80de00a1
:10b880000fb997009fb997000201400083814800db
:10b8900082bf9f0093bf9f000402e800e80f5200a0
:10b8a000ebff3400304580006106b8000c01be009b
:10b8b0000600be00fae60700e8898000cfc4de007b
:10b8c0000005440081854c000c01be000fb89700b4
:10b8d0009fb89700f2e607000006440081864c00fe
:10b8e00061005500e0805d00e80f5000e08f5800d7
:10b8f00002003e00aa0020000b002000e00f5500cf
:10b90000e08f5d0006003d0060ff2f00f1ff2f007b
:10b91000800f5500818f5d00010034000005be00de
:10b9200061005600e0805e00e80f5000e08f580094
:10b9300002003e00ac0020000d002000e00f560089
:10b94000e08f5e0006003d0060ff2f00f1ff2f003a
:10b95000800f5600818f5e00010034000006be009b
:10b96000021020000250b80002dab90084804000c2
:10b970000005be000260b80002e9b9008280400004
:10b980000006be00faef9f0002f02f000300200027
:10b990000200650083806500c809dd004800de0004
:10b9a00000807100c888de00e0ef9f00dbef9f00a1
:10b9b0004858de0001002000c0ef9f008042780060
:10b9c0000b427800efe997000a41780031c0b300dc
:10b9d00020c5b3006d040700fcef9f0002f02f00ac
:10b9e000030020000200660083806600c809dd00b5
:10b9f0004800de0000807100c888de00e0ef9f0094
:10ba0000ddef9f004868de0001002000c0ef9f00ce
:10ba1000804278000d427800efe997000c417800f1
:10ba200031c0b30040c5b30058040700f48257008a
:10ba300073825700f28157007181570011c0b30023
:10ba400020c5b300a50407004fe99700c811dd0029
:10ba5000020020005fe897008080fb0000002000cb
:10ba600000017100818171006fe897004800dd00de
:10ba70000100200000017100818171007fe89700c2
:10ba80000080fb0001002000000171008181710035
:10ba9000a2458800b3458800f4825700738257009e
:10baa000f28157007181570011c0b30040c5b30047
:10bab0008a0407004fe99700c811dd00020020004a
:10bac0005fe897008080fb0000002000000171000b
:10bad000818171006fe897004800dd0001002000bf
:10bae00000017100818171007fe897000080fb00f8
:10baf000010020000001710081817100c2458800b1
:10bb0000d34588003e71ef0060458000b408b50061
:10bb1000301fb000613e2000810f500048003e0001
:10bb200080458000b808b500301fb000810f50007c
:10bb300043003e004011ec00008a8800e70f5000ef
:10bb40004800360000e02c00f10f20000084eb00dc
:10bb5000880078000005be000c2023000d002000a6
:10bb600000406400f0ef9f0002f02f00030020006f
:10bb70000200650083806500c809dd004800de0022
:10bb800000807100c888de00e0ef9f000000200008
:10bb9000f10f200000006500818065004088de0014
:10bba000cf80de00d0ef9f000000200001f02f00ca
:10bbb00000006500818065004808de00010020006b
:10bbc000c0ef9f00804278005fea9700efe997009e
:10bbd0007fe9970031c0b30020c5b300eb03070035
:10bbe0000c446400f8ef9f0002f02f0003002000d7
:10bbf0000200660083806600c809dd004800de00a0
:10bc000000807100c888de00e0ef9f006000b8008f
:10bc1000d0ef9f00c0ef9f00804278005fea97005e
:10bc2000efe997000841780031c0b30040c5b30088
:10bc3000d603070010c0b3003ef1b700090037007b
:10bc40004031ef00a0458000b1458000604588008c
:10bc500071458800c2458000d34580008245880038
:10bc6000934588004f06be004f05be004f04be003e
:10bc70000080fa00000006000e00fa00889fbe0057
:10bc80008a9fbe008c9fbe0010c0b3003ff1b7007a
:10bc90006033b80086bf9f0097bf9f000002eb0093
:10bca000c51e2100388320004a0620008001eb00d9
:10bcb0000400d0008000780060807a0070004000ae
:10bcc000900f140009003e00e1807a008301e80033
:10bcd0000300d0000100400070004000900f1400ed
:10bce00002003e00e48f5100f8ff34000400d00051
:10bcf000e0807a000300d0000100400066004000b0
:10bd0000900f150002003e00e48f51000500340042
:10bd10000400d000fa805700010040000008eb004a
:10bd2000080037000401d000e2807a000300d00050
:10bd30000100400066004000100055007a015100eb
:10bd400000b17f000402e800e40f5200d7ff340086
:10bd50000002eb00a8122100851121000401d0008f
:10bd60007a8057008001410062007c001380b90096
:10bd7000cf80de00060340008783480062807a009f
:10bd80001380b900cf80de000fb997009fb99700ec
:10bd9000020140008381480082bf9f0093bf9f0043
:10bda0000402e800e40f5200ecff3400504580002c
:10bdb0006106b8000c01be000600be00b8e5070031
:10bdc000e8898000cfc4de000005440081854c0076
:10bdd0000c01be000fb897009fb89700b0e50700b0
:10bde0000006440081864c0061005500e0805d0043
:10bdf000e80f5000e08f580002003e00aa0020002b
:10be00000b002000e00f5500e08f5d0006003d00b4
:10be100060ff2f00f1ff2f00800f5500818f5d0024
:10be2000010034000005be0061005600e0805e00a5
:10be3000e80f5000e08f580002003e00ac002000e8
:10be40000d002000e00f5600e08f5e0006003d0070
:10be500060ff2f00f1ff2f00800f5600818f5e00e2
:10be6000010034000006be00021020000250b8009d
:10be700002dab900848040000005be000260b8000c
:10be800002e9b900828040000006be0008f02f00e1
:10be90000900200008016500898165004818dd005f
:10bea0004811de0002017000c899de000b83fb0020
:10beb000070020004858de00010020008042780082
:10bec00006427800824178000a41780031c0b30010
:10bed00020c5b3002d0307000804660089846600ae
:10bee000c848dd004844de0008847000c8ccde008d
:10bef0000d81fb00030020004868de0001002000e7
:10bf00008042780002427800884178000c41780035
:10bf100031c0b30040c5b3001c0307004f06be008c
:10bf20004f05be004f04be000080fa00000006006e
:10bf30000001fb00cf91de00ea0f5100e08f5900b5
:10bf40004e003e00026001000a0037000e0037007c
:10bf500013003700180037001d003700220037009b
:10bf6000270037002c00370032003700360037003a
:10bf70003b003700d202a900e1c06000d4c2bf007c
:10bf80000004a10028003700d222a900e1c060000f
:10bf90008140d000d4c2bf000014a10022003700ad
:10bfa000d242a900e1c06000c208dd00d4c2bf00d7
:10bfb0000024a1001c003700d262a900e1c060008b
:10bfc000c308dd00d4c2bf000034a1001600370052
:10bfd000d282a900e1c06000c408dd00d4c2bf0065
:10bfe0000044a10010003700d2a2a900e1c0600007
:10bff000c508dd00d4c2bf000054a1000a0037000c
:10c00000d2c2a900e1c06000c608dd00d4c2bf00f2
:10c010000064a10004003700d2e2a900c708dd00d7
:10c02000d4c2bf000074a10001407000d4e2b70088
:10c0300012003700d302a900e1c06000d5c2bf00e2
:10c040000004a1000b003700d322a900e1c060006a
:10c050008140d000d5c2bf000014a1000500370008
:10c06000d342a900e1c06000c208dd00d5c2bf0014
:10c070000024a10001407000d5e2b70000000600d6
:10c08000881f78000004eb0011c0b300084078005e
:10c09000a7ff0700100020002af007000804e800ae
:10c0a000ea0f5400f8ff34004f0478000000060047
:10c0b000c00721000c0009000018eb0060092100f6
:10c0c0000c0009000018eb00000b21000c00090017
:10c0d0000018eb00a00c21000c0009000018eb0078
:10c0e000800e2100050009000018eb00e4ff0700a6
:10c0f000f000200013f0070000000600889fbe003b
:10c100008a9fbe008c1f780000457800810578006a
:10c110000206780097f107008a80fb0010002000db
:10c120000100dd00a408b60002003a000100d000c2
:10c1300009003700e84f55000c003600c9c2bf00a7
:10c140000080fb004700de000080fb0007003a0093
:10c150000a80fb000000d0008c0040008008eb004b
:10c160000b0040000008eb003400370011c0b300a2
:10c170000a4078006eff070040c0b30089f0070056
:10c180008c00a9000a80fb00e54f55000200360034
:10c190000a80fb000080e8008000eb004cf1070003
:10c1a00010002000e7ef07000044eb008004eb00e4
:10c1b00070f10700808444000844e800e34f540015
:10c1c000fbff36000a80fb000000d000c248de0002
:10c1d00001b07d008040eb000a40780054ff07006a
:10c1e00020032000d7ef07000044eb008004eb00a1
:10c1f00060f10700808444000844e800e34f5400e5
:10c20000fbff360040c0b30084f007000a80fb004b
:10c210000000d0000c0140000b004000c248de00ce
:10c220001080100001003b000000ea0000097800c7
:10c2300011c0b3000a4078003dff07004f067800a8
:10c240004f05be004f04be0000000600c028ef00ee
:10c25000c228ef0040ea2000e2ef070020c0b30050
:10c260008cf0070020c0b3006cf0070020c0b300c2
:10c2700033f007000000eb00000006008000eb0038
:10c28000d000200012f10700a1e2a900a342a800fb
:10c29000a042a800c0c3b300a262b70010002000f3
:10c2a000a8ef0700a1e2a8008560a9008d60a800a2
:10c2b0000000eb0000000600a1e2a9008560a900d3
:10c2c0008d60a900a342a900a042a90030ccb30010
:10c2d000a262b600100020009aef0700a1e2a800b9
:10c2e000000006003600f800809fbe00829fbe005e
:10c2f000849fbe00869fbe00881f78000046800095
:10c300001146800061004000e0804800004688003f
:10c310001146880032002000030020006fe407006f
:10c32000e00f5000e08f580031003a00e2ff0700b4
:10c33000c408e2000b003a00c007210020878800f3
:10c34000000b21003087880060092100b08388003d
:10c35000a00c2100c0838800100020002046880027
:10c3600009003700c428ef006009210020878800f9
:10c37000a00c210030878800c0072100b08388000e
:10c38000000b2100c0838800328780002187800055
:10c39000bcc8bf0059ff0700bcc8bf008040780080
:10c3a0000040e800bce8b700e9cf50000b003600c1
:10c3b000bc68ef0030878000024680001346800092
:10c3c00032089800430898002087800002468000c9
:10c3d000134680003208980043089800b01e2100e0
:10c3e00013c0b30090cf110001003a00a3ff070073
:10c3f000420120000300200000468000114680001a
:10c4000036e40700e00f5000e08f580042003a0089
:10c41000a9ff0700eb71ef00de82a900e082a8000f
:10c42000800e2100d0838800bec8bf008080fb0042
:10c430000040e800bee8b700ef8f50001700320060
:10c4400005003c00e58f50000c003200ea8f5000e0
:10c450000e00320021003700f98f50001700320023
:10c4600003003c00f48f5000100032001b00370026
:10c47000fe8f50001500320018003700d88380006e
:10c480002af10700000c780014003700d8838000e0
:10c490007cf107001004980010003700d88380005a
:10c4a000abf10700200498000c003700d88380000f
:10c4b000daf107003004980008003700d8838000c4
:10c4c00044f107004004980004003700d88380003e
:10c4d000eaf10700204c9800be68ef00d8d1bf00f9
:10c4e000804078000040e800d8f1b700e3cf50006a
:10c4f00001003600d871ef00e1448000d8d1bf00c0
:10c500009e0307000004e00003003200d8d1bf0002
:10c510000080fb00690307002203200003002000c5
:10c520000046800011468000ece30700e00f500059
:10c53000e08f580004003a003f51e20002003a0048
:10c5400030c0b3003ff1b700c20820000300200054
:10c550000046800011468000e0e30700e00f500035
:10c56000e08f580006003a00f013210011c0b3001c
:10c5700090cf100002003a0040c0b3003ff1b70076
:10c5800084c0a9004f0478004f03be004f02be00d4
:10c590004f01be004f00be003600f900004006000b
:10c5a000881f780081e0a900c09d200083ed07006e
:10c5b00035ed070010c0b30043ed07007000200008
:10c5c000801f780020002000801f780000ed2e00e2
:10c5d000801f780090d207002a05070038f0070076
:10c5e00022030700b2f1070018ff07006cee0700f6
:10c5f000e68757000000e00002003200f0ef2e0056
:10c600000100370090f12e0067d20700a8fe070056
:10c61000c7c2a8005eee07000000e0001200320072
:10c6200060f32e0060d2070040ea070010c0b3009c
:10c630002aed0700f8182000ce42a800418f8000a4
:10c64000308f8000808f5000fbff3200d003070046
:10c65000e811ec00408f8800880f5000f6ff36008c
:10c66000e831ef00f4ff370060f52e004ed20700ee
:10c6700040062000c1ee070020ea070050f72e0018
:10c6800049d2070040052000f801070040052000be
:10c69000320007000080fb00ef1f60004400de0056
:10c6a000801f7800b0f92e00801f78005ad2070052
:10c6b00020052000ed0107002005200027000700cd
:10c6c0000080fb00ef1f60004400de00801f780048
:10c6d000c0fc2e00801f78004fd20700d0ff2e0034
:10c6e00031d2070020c0b3003ff1b700ec875700fc
:10c6f000f8132100ce42a800b6f3070012fb070092
:10c70000b8f1070030c0b300984f100002003a00a3
:10c71000d5fb07000400370040c0b300984f10005d
:10c7200001003a0054fd0700418f8000308f8000e7
:10c73000808f5000efff320095030700418f80008b
:10c740008100e800418f8800f0182000808f5000a1
:10c75000e8ff3600e831ef00e6ff37008040eb00ed
:10c7600060ec07000080fb0000000600889fbe0010
:10c770008a1f780000457800810478000204780060
:10c78000811f7800c0012f00801f780022d207008f
:10c79000881f780010032f00801f78001ed207002a
:10c7a000e88757000900e00004003200e1c2b3004e
:10c7b0000a4078004bec0700804c78000800e0004d
:10c7c00004003200d1c2b3000a40780045ec0700f3
:10c7d000004c78001880fb00801f78001980fb0057
:10c7e000801f780050042f00801f78000ad20700b5
:10c7f000e68757004f0578004f04be000000060092
:10c80000889fbe008a1f78000044780001057800e8
:10c8100082047800b1c2b30032ec0700004d78000a
:10c82000a1c2b300084078002eec0700804c7800cd
:10c830000080fb00801f78001a80fb00801f7800ba
:10c8400050062f00801f7800f3d10700e6875700bd
:10c850004f0578004f04be00000006000400fa00f7
:10c86000889fbe008a9fbe008c1f7800804478009d
:10c870000205be0004067800e48f500005003e006b
:10c88000e0c3b300e18f500008003e000400320016
:10c890000b003700e58f500003003200080037001e
:10c8a00010c6b3000100370070c6b300a0f79f00a8
:10c8b00000c0e800b0f79f0000c0e800c0f79f008c
:10c8c000aff097000940780006ec070000447800bc
:10c8d0002ff097008040e8000940780001ec070045
:10c8e0004800dd00000d78000880fb001a0d700084
:10c8f000bff0970009407800faeb07000044780089
:10c90000bff097008140e80009407800f5eb070090
:10c910004800dd00800d78000880fb009b0d700052
:10c92000cff0970009407800eeeb07000044780054
:10c93000cff097008140e80009407800e9eb07005c
:10c940004800dd00000e78000880fb001c0e70001f
:10c950004f0678004f05be004f04be000080fa006d
:10c96000000006000400fa00889fbe008a9fbe00f7
:10c97000004478008204780083057800040578007c
:10c98000e48f500005003e00e0c3b300e18f50008b
:10c9900008003e00040032000b003700e58f500015
:10c9a000030032000800370010c6b3000100370052
:10c9b00070c6b300c0f79f0000c0e800d0f79f002a
:10c9c00000c0e800e0f79f0048c9de004ff0970084
:10c9d0008040e800084078001eea0700094178001e
:10c9e000cff09700084078001aea070048d1de002f
:10c9f000dff097008140e8000840780015ea070062
:10ca00000a417800dff097000840780011ea07003b
:10ca100048d9de00eff097008140e8000840780038
:10ca20000cea07000b417800eff09700084078000f
:10ca300008ea07004f05be004f04be000080fa0060
:10ca400000000600889fbe008a9fbe000044780058
:10ca500081457800024578008344780004417800dd
:10ca600071c3b300fbe907000941780061c3b3005b
:10ca700008407800f7e907000a41780051c3b30085
:10ca800008407800f3e907000b41780041c3b30088
:10ca900008407800efe907004f05be004f04be00d4
:10caa00000000600889fbe008a1f780000447800be
:10cab0008144780003457800e1c6b300e5e907004a
:10cac00009417800d1c6b30008407800e1e90700c9
:10cad0000a41780021c5b30008407800dde907006d
:10cae0004f0578004f04be0000000600889fbe007e
:10caf0008a1f7800004578000404be000100fb0096
:10cb0000e10f500011003500e20f50000300340027
:10cb1000e50f5000090032000c003700a1c4b3003b
:10cb20000a4078006cea07000801be00e1c4b300c7
:10cb30000a40780068ea0700040037000401780022
:10cb400061c5b3000a407800f7e907004f05780097
:10cb50004f04be0000000600889fbe00004478001d
:10cb60008244780001417800a1c2b30008407800f7
:10cb7000b8e9070009417800b1c2b3000840780065
:10cb8000b4e907004f04be0000000600889fbe0005
:10cb90008a9fbe008c9fbe000044780081447800cc
:10cba0008246780003467800844578000545780081
:10cbb00081c2b3004beb0700e14f5000040032008c
:10cbc00012c0b30081c2b30008407800a1e9070099
:10cbd00009417800c1c2b300084078009de9070010
:10cbe0000a41780021c3b3000840780099e90700a2
:10cbf0000b41780011c3b3000840780095e90700a5
:10cc00000c41780001c3b3000840780091e90700a7
:10cc10000d417800f1c2b300084078008de90700ab
:10cc20000041eb0091c2b3000840780089e9070099
:10cc30004f06be004f05be004f04be0000000600b8
:10cc4000889fbe008a9fbe008c1f780080447800b9
:10cc500001047800f1c2b30022eb0700004678001f
:10cc600001c3b300094078001eeb0700804578003f
:10cc700011c3b300094078001aeb070000457800a3
:10cc800021c3b3000940780016eb0700c800dd009f
:10cc900000002000008cbe008a80fb000000200005
:10cca000181c7000189470004858dd000100200026
:10ccb000181c7000189470000c80fb00010020000c
:10ccc000181c7000189470000000eb004f067800ec
:10ccd0004f05be004f04be0000000600889fbe0046
:10cce0008a9fbe008c1f78000044780002067800fe
:10ccf0008305780004057800850478000100fb00b6
:10cd0000e20f500003003c000000e0000a003c007d
:10cd100004003700e40f500015003400e50f500008
:10cd200021003200004eeb00804deb00004deb0087
:10cd3000804ceb002400370071c3b300084078003a
:10cd4000e8ea0700804c780061c3b300084078002f
:10cd5000e4ea0700004d780051c3b30008407800b2
:10cd6000e0ea0700804d780041c3b30013003700ac
:10cd7000b1c3b30008407800daea0700804c7800bd
:10cd8000a1c3b30008407800d6ea0700004d780040
:10cd900091c3b30008407800d2ea0700804d7800c4
:10cda00081c3b30005003700b1c5b3000840780067
:10cdb000ccea0700804d7800a1c5b3000840780098
:10cdc000c8ea0700004e78000000eb004f0678002c
:10cdd0004f05be004f04be00000006000041eb00fe
:10cde000d1c2b3001be90700000006000141780032
:10cdf00061c4b30017e9070000000600889fbe0069
:10ce000080447800010478004809de0051c4b30072
:10ce100010e907000841780041c4b30009407800d8
:10ce20000ce907004f04be00000006000141780035
:10ce300081c2b30007e90700000006000141780045
:10ce400001c6b30003e907000000060001417800b5
:10ce500031c7b300ffe80700000006000141780079
:10ce600001c7b300fbe8070000000600889fbe0072
:10ce7000804478000004e000380032000084fb00a9
:10ce80008000eb0008007800e8ff0700e160200068
:10ce900008007800d9ff0700610020000800780032
:10cea000e6ff070020c5b30080cf540004003a001d
:10ceb000220a20008000eb00080078000300370001
:10cec0000980fb00220220008000eb0022ff070007
:10ced0000984fb0008007800c0ff0700a1002000c3
:10cee00008007800c1ff0700431f20000001eb008d
:10cef0005100200008007800fcfe070003712200aa
:10cf0000028f2d001100200008007800f7fe0700b6
:10cf100034002000a3002000c226200084007800f6
:10cf2000094078008ffe070044012000e301200043
:10cf300082252000110020000940780089fe0700aa
:10cf4000e3c1b30072c2b30001c1b300094078006d
:10cf5000d4fe07001000200003003700c0072f0098
:10cf600011d007000000eb004f04be0000000600d7
:10cf7000889fbe008a9fbe00814578000305780027
:10cf800084047800050478000200e0000a00320002
:10cf900005027800890178000a017800110020005c
:10cfa00070fe070008027800890178000a01780005
:10cfb000110020000900370005027800890178007f
:10cfc0000a0178003100200066fe070008027800a0
:10cfd000890178000a017800310020000b407800b8
:10cfe00060fe07004f05be004f04be0000000600b3
:10cff000881f7800014478000080fb002100200099
:10d000008aff07000880fb002100200087ff07003f
:10d010004f04780000000600d562a900d362a90081
:10d0200000000600d562a800d362a9000000060037
:10d03000e522a900e582a900e5a2a9000080fb0085
:10d04000e20f50001800320005003c000000e00034
:10d0500008003200e10f50000b00320020003700c2
:10d06000e30f500015003200e40f500015003200ad
:10d070001b003700e722a8001000200031ec070059
:10d08000e782a80004003700e722a9001000200072
:10d090002cec0700e782a9001000200029ec070013
:10d0a000e7a2a9000e003700e722a9001000200027
:10d0b00024ec0700e782a80006003700e722a90059
:10d0c00001003700e722a800100020001dec070037
:10d0d000e782a900100020001aec0700e7a2a800d0
:10d0e00000000600881f7800dea2a900e0a2a800c8
:10d0f0001000200013ec0700de82a900e082a900e6
:10d100000044eb00100020000eec0700e0a2a90094
:10d11000dea2a900100020000aec0700dea2a90090
:10d12000e0a2a8000844e800ff4f5400f5ff3400d7
:10d13000de82a900e082a8001000200001ec0700b8
:10d14000e0a2a900dea2a90010002000fdeb07006c
:10d15000de82a900e082a9004f04780000000600ea
:10d16000dea2a900e0a2a80050002000f5eb070015
:10d17000dea2a900e0a2a90050002000f1eb070008
:10d1800000000600881f780000047800e402a9006f
:10d19000e422a900e4c2a900e4e2a900e502a90092
:10d1a000401720002fec070040c0b3009bec0700a5
:10d1b000e20f54000e00320006003c001000200078
:10d1c0000800e0000f003200e10f540006003200ba
:10d1d0000f003700e30f540007003200e40f540043
:10d1e000070032000a003700200020000500370049
:10d1f0000004200003003700000820000100370071
:10d2000000102000108f8800602e2000208f8800e2
:10d2100040c0b3004aec07004f047800000006004d
:10d22000160009003118780000000600881f7800f9
:10d230008000eb00d000200025ed0700100020004a
:10d24000c0eb07004bed070000047800200320002e
:10d25000bceb070047ed0700000444000804d100c0
:10d26000080078004f04780000000600881f78004e
:10d2700069ff07008000eb00c21e21000100d00002
:10d2800060007900160009000018eb0020712100f1
:10d29000160009000018eb008100e800e48f500040
:10d2a000f6ff3400e1ff0700000478005aff070092
:10d2b000080078004f04780000000600889fbe0038
:10d2c000800478005aff070086ff07002576ef00ec
:10d2d0002676ef002036ef002236ef00dc71ef00fb
:10d2e0002776ef002476ef00d631ef00db71ef00f8
:10d2f000da71ef00de31ef00e631ef00e831ef00e8
:10d3000040c0b300f5eb070040c0b30025ec0700b8
:10d310008c00a9008000eb00d0002000ecec07009e
:10d320001000200087eb070012ed0700010020002d
:10d3300040b1880051b18800b08f8000160009000c
:10d340000018eb00b88f8000b8ff07002004980099
:10d35000b08f80001900980020c0b300dfeb0700f9
:10d360000900780087ff0700d971ef0010c0b300f3
:10d37000ddf1b7004f04be00000006006109b800ef
:10d38000ff0f5100e08f590044003e000260010091
:10d390003e003700250037001d0037002c00370005
:10d3a0001d0037003d003700240037002f003700f4
:10d3b0001b003700390037003800370037003700ce
:10d3c0002000370035003700250037002c003700db
:10d3d0001500370031003700300037002f003700cc
:10d3e0002e0037002d0037002c0037002b003700af
:10d3f00016003700290037002800370027003700c3
:10d4000019003700250037001c00370021003700c5
:10d410000004a200050037000014a200030037003a
:10d4200030c0b200010037000024a2000080fb00e1
:10d430000000e900cf00de00180037000040e900de
:10d440000300370000c0e9000100370063405000ce
:10d4500011002000e14f5000100036000b00370093
:10d460000040e9000100370000c0e9001100200081
:10d47000e24f500009003600040037000040e90088
:10d4800011002000e34f5000040036008000eb0044
:10d490000200370011002000000037000100780072
:10d4a00000000600000178008001eb0001b180005f
:10d4b00080072000808f5000330036008001eb0091
:10d4c00001b1800000642000808f50002e003e00db
:10d4d0008001eb0030832000800f51002a003600cd
:10d4e000a808e2002700320000b1800071f82f0088
:10d4f0000100400001032000810f500004003e00a5
:10d500008001eb00b0c12000800f51001e003600ea
:10d5100000b1800061f52f0001004000fd0f5000b8
:10d5200004003e008001eb00309c2000800f510081
:10d530001500360000b1800081f32f00010040008b
:10d5400011032000810f500004003e008001eb0019
:10d55000b08f2000800f51000b00360000b180001a
:10d5600061f02f0001004000710c2000810f50007d
:10d5700004003e008001eb0070892000800f510004
:10d5800001003600130020000300780000000600b0
:10d59000889fbe002756e2002c003a002556ec007a
:10d5a00025f6b7000084fb00f0448000800f540093
:10d5b00024003e0009302100e811d40060807c0086
:10d5c000b8ff07000004e0001e00320010c0b300e6
:10d5d00027f6b7000800d000b18f8000010040009e
:10d5e00001b18000210098005262210012417800b0
:10d5f0000281fb006411b800b08f8000000141007f
:10d6000000468000114680003009980041099800ca
:10d61000e811d40060807c000100200040b1880047
:10d6200051b1880025d6bf000080fb000000d0006b
:10d63000b18f80000100400041b18000710098006e
:10d640008e0037002576ed008c003700a01d2100ec
:10d6500041c0b30090cf10003c003e0025d6bf0073
:10d660000080fb000000d000b18f8000010440006a
:10d67000ee00440009302100e811d4000900400008
:10d6800091007800908f50001f003100100078004a
:10d6900084ff07000004e0001b00320000b180009e
:10d6a0002004980052622100124178000281fb00a0
:10d6b0006411b800b18f8000010141000046800074
:10d6c00011468000300998004109980025d6bf0016
:10d6d0000080fb000000d000b18f800001004000fe
:10d6e000418f80008100d000e1807c0071009800b3
:10d6f000e811d40060807c000100200040b1880067
:10d7000051b18800da71ef00e811d4000130210036
:10d7100001004000100078006101b80040b18000b5
:10d7200051b18000800f5100818f590053003100aa
:10d73000da51ec00daf1b700e44f50004f00360048
:10d7400042b1880053b188004c003700a41d21006d
:10d750001442780065405200e24f500015003e0030
:10d76000e811d400013021000100400010007800d1
:10d770000100200042b1800053b18000820f5000b0
:10d78000838f5800030036000440e800daf1b70048
:10d790003a003700e811d4000130210001004000b8
:10d7a000100078003fff07000004e00033003a005b
:10d7b00030003700a01d210071c0b30090cf1000d1
:10d7c0002e0036002556ec0025f6b7000084fb003d
:10d7d000f0448000800f540025003e0009302100f5
:10d7e000e811d40060807c002eff07000004e000f8
:10d7f0001f003200da71ef000800d000b18f800006
:10d800000100400001b18000210098005262210017
:10d81000124178000281fb006411b800b08f8000d3
:10d820000001410000468000114680003009980048
:10d830004109980025d6bf000080fb000000d00001
:10d84000b18f800001004000418f80008100d00036
:10d85000e1807c0071009800e811d40060807c00b9
:10d860000100200040b1880051b18800030037005a
:10d870002576ed00da71ef002776ef0040002000fa
:10d880002036b4004f04be00000006003600f80049
:10d89000809fbe00829fbe00849fbe00869fbe0008
:10d8a000b18e80008100e800b18e88001002200057
:10d8b000808f50000a003a0010c0b300ebf1b700af
:10d8c0006efa070020c0b3009dea070040c0b30015
:10d8d00082ea070040c0b300b2ea07000700370041
:10d8e000b18e800000022000808f500003003c00b9
:10d8f000218f8000108f80009108680086a0a90009
:10d900004f03be004f02be004f01be004f00be00dd
:10d910003600f900004006003600f800809fbe0087
:10d92000829fbe00849fbe00869fbe00889fbe006f
:10d930008a1f78008044eb00022820000530210077
:10d94000f4182000338f800032007800320040004d
:10d9500032004000320040008300d0004200de0070
:10d9600080b07a008301e800848f51000100360006
:10d970008001eb008944e800e3cf5400f2ff360059
:10d98000338f88002216ec0010b188000008a30035
:10d9900006003a004062210091c1b30090cf100010
:10d9a00002003e00eefd07002476ec0011b180007d
:10d9b000d0062000808f500029003600eb71ef0068
:10d9c0003dfa070025d6bf000080fb00b18f800024
:10d9d000800878008044eb0025d6bf00004ce100b1
:10d9e000160031000980fb000000d000b18f8000dc
:10d9f00001004000660540001a0478006140b9004b
:10da0000acdd07000800e00003003d00020020003c
:10da10000378240007de0700c2f52800a30b2400ca
:10da2000b1de070083de0700000d78008944e800be
:10da300025d6bf00004ce100eaff3900b18f80001d
:10da4000110090000000d000c21e21000200400022
:10da500010007800f2fd070010c0b300eaf1b70033
:10da60008560a9004f0578004f04be004f03be003b
:10da70004f02be004f01be004f00be003600f9004d
:10da800000400600c602a800c622a800c642a800a0
:10da9000c662a800c682a800c6a2a800c702a80045
:10daa000c722a800c742a800c762a800c782a80072
:10dab000c7a2a800a802a900a822a900a842a900fc
:10dac000a862a900a882a900a8a2a900a8c2a800cb
:10dad000a8e2a800a902a900a922a900a942a900b8
:10dae000a962a900a982a900a9a2a900a9c2a800a7
:10daf000a9e2a800aa02a900aa22a900aa42a90094
:10db0000aa62a900aa82a900aaa2a900aac2a90081
:10db1000aae2a900ab02a900ab22a900ab42a9006e
:10db2000ab62a900ab82a900aba2a800abc2a9005e
:10db3000abe2a900a1e2a900c0cfb300a162b60088
:10db4000a042a90001ceb30001407800a062b70056
:10db50007dc05000a262b600a342a900f0c1b3008c
:10db6000a362b600a382a900a5c2bf000140600065
:10db7000c040b300a5e2b700a4c2bf0001ccb3000f
:10db8000014060003041b300a4e2b700000006008d
:08db90000000fe000040060049
:020000040000fa
:0200000401f009
:04000000f7ff000006
:020000040000fa
:0200000401f009
:04000400ff7f00007a
:020000040000fa
:0200000401f009
:04000800efff000006
:020000040000fa
:0200000401f009
:04001400ffff0000ea
:020000040000fa
:10000800c86d0000c86d0000c86d0000c86d000014
:10001800c86d0000c86d0000c86d0000c86d000004
:10002800c86d0000c86d0000c86d0000c86d0000f4
:10003800c86d0000c86d000072610000c86d000046
:10004800c86d0000783d0000c86d00008c6c000091
:10005800c86d0000c8370000c4370000c86d000034
:10006800c86d0000c86d0000c86d0000c86d0000b4
:10007800c86d0000466c0000c86d0000c86d000027
:10008800c86d0000c86d0000c86d0000c86d000094
:10009800c86d0000c86d0000c86d0000c86d000084
:1000a800c86d0000c86d0000c86d0000c86d000074
:1000b800c86d0000c86d0000c86d0000c86d000064
:1000c800c86d0000c86d0000603f0000c86d0000ea
:1000d800c86d0000c86d0000c86d0000c86d000044
:1000e800c86d0000c86d0000c86d0000c86d000034
:0800f800c86d0000c86d000096
:020000040000fa
:10010800c86d0000c86d0000c86d0000c86d000013
:10011800c86d0000c86d0000c86d0000c86d000003
:10012800c86d0000c86d0000c86d0000c86d0000f3
:10013800c86d0000c86d000072610000c86d000045
:10014800c86d0000783d0000c86d00008c6c000090
:10015800c86d0000c8370000c4370000c86d000033
:10016800c86d0000c86d0000c86d0000c86d0000b3
:10017800c86d0000466c0000c86d0000c86d000026
:10018800c86d0000c86d0000c86d0000c86d000093
:10019800c86d0000c86d0000c86d0000c86d000083
:1001a800c86d0000c86d0000c86d0000c86d000073
:1001b800c86d0000c86d0000c86d0000c86d000063
:1001c800c86d0000c86d0000603f0000c86d0000e9
:1001d800c86d0000c86d0000c86d0000c86d000043
:1001e800c86d0000c86d0000c86d0000c86d000033
:0801f800c86d0000c86d000095
:020000040000fa
:10db98004261000074740000657200007920000082
:10dba800534e0000203d0000205200006561000037
:10dbb8006420000045520000524f0000520d000042
:10dbc800000000002c250000640000002c25000047
:10dbd8006c750000002c0000256c0000640000003b
:10dbe8002c250000750000002c2d00002575000074
:10dbf800002c0000256c0000642c0000256c00003f
:10dc0800640000000a0d0000000000004f560000ec
:10dc180045520000464c00004f5700000d00000020
:10dc28004f53000020750000706c00006f61000009
:10dc380064650000722000006d6f000064650000dc
:10dc48002c2000007761000069740000696e0000f4
:10dc580067200000666f0000722000006461000009
:10dc6800746100002e2e00002e0d000000540000ec
:10dc7800696d0000656f0000757400002061000088
:10dc8800626f000072740000696e0000670d00008a
:10dc9800007100000d0000002b2b00002b0000007d
:10dca800534500005420000042540000204e00005c
:10dcb800414d0000452000004b4800004949000044
:10dcc80049200000257500000a00000053450000a7
:10dcd8005420000042540000204300004c41000042
:10dce8005353000020300000303000003131000074
:10dcf800300000005345000054200000425400004a
:10dd08002041000055540000482000002a2000004f
:10dd1800303000003030000000530000455400004f
:10dd2800204300004f4e0000545200004f4c0000aa
:10dd380020450000434800004f200000300000004c
:10dd4800534500004c4500004354000020300000bb
:10dd5800004300006f6e0000666900006720000045
:10dd680042540000204f00004b0d0000004200000c
:10dd7800617400007465000072690000652000008d
:10dd8800707200006f670000726100006d6d000026
:10dd9800e96500000d0000000d0a00004b68000056
:10dda800657000006572000061330000204f0000bc
:10ddb8005320000028630000292000004b2d00009c
:10ddc80054650000616d0000205300002e410000e2
:10ddd8002e2000003230000030370000207600008e
:10dde8006572000020250000642e000025640000f4
:10ddf8000d0a000000460000726f00006e740000fb
:10de08002065000078740000656e000073690000ea
:10de18006f6e0000206400006574000065630000f8
:10de280074650000640d0000004e00006f200000c3
:10de3800467200006f6e00007420000065780000d4
:10de4800746500006e730000696f00006e200000aa
:10de58006465000074650000637400006564000078
:10de68000d000000536c0000617600006520000082
:10de78004f530000206d00006f6400006520000013
:10de88002877000069740000682000006b6f0000ac
:10de980072650000626f0000742900000d0a00001e
:10dea8000d0000004d6100007374000065720000f1
:10deb800204f0000532000006d6f000064650000d3
:10dec8002028000073740000616e00006461000087
:10ded8006c6f00006e650000290d00000a0d00003f
:10dee8000049000032430000204800006173000030
:10def80020620000656500006e200000696e000069
:10df080069740000696100006c69000073650000b5
:10df1800642000006173000020610000206d000093
:10df28006173000074650000720d0000005200006b
:10df38006967000068740000206d00006f740000bd
:10df48006f720000206900006e69000074690000ab
:10df5800616c00006973000061740000696f000063
:10df68006e200000636f00006d7000006c6500009b
:10df780074650000642000007665000072200000cf
:10df8800256400002e250000640d00000a00000032
:10df98004c65000066740000202000006d6f0000d2
:10dfa800746f000072200000696e00006974000040
:10dfb800696100006c690000736100007469000009
:10dfc8006f6e0000206300006f6d0000706c000031
:10dfd800657400006564000020760000657200002a
:10dfe80020250000642e0000256400000d0a0000b2
:10dff8000053000065720000696100006c20000099
:10e00800436f00006d6d0000756e000069630000cd
:10e0180061740000696f00006e20000050720000fb
:10e028006f7400006f6300006f6c00000d0000004b
:10e03800537400006174000075640000206f0000d4
:10e048006666000073650000742000003d20000033
:10e05800255800000d0a00000045000072720000fb
:10e068006f720000206f0000666600007365000094
:10e07800742000003d200000255800000d0a000013
:10e0880000730000746100007475000073200000c4
:10e098003d200000253200002e320000582c0000e0
:10e0a80020650000727200006f720000203d0000c1
:10e0b80020250000322e0000325800000d0a000012
:10e0c80000730000772000003d2000003078000039
:10e0d800257800002c20000068770000203d000013
:10e0e8002030000078250000780d00000a000000ac
:10e0f800696e0000697400004d6f00007420000014
:10e1080065720000726f0000722c00002069000028
:10e118003263000020610000646400007265000042
:10e128007373000020630000616e00006e6f0000d2
:10e138007420000062650000206e0000756c00000d
:10e148006c0d000000000000005e0000bce2000052
:10e15800613f0000dd830000c29c00007e200000bb
:10e16800a3fd00001f4100009dc30000217f0000a7
:10e17800fca20000401e00005f010000e3bd00009b
:10e188003e60000082dc0000237d00009fc100008b
:10e19800421c0000fea00000e1bf00005d0300007b
:10e1a80080de00003c620000bee00000025c00006f
:10e1b800df810000633d00007c220000c09e00005b
:10e1c8001d430000a1ff000046180000faa400004b
:10e1d800277900009bc5000084da0000386600003b
:10e1e800e5bb000059070000db8500006739000027
:10e1f800bae400000658000019470000a5fb00001b
:10e2080078260000c49a0000653b0000d98700000a
:10e21800045a0000b8e60000a7f900001b450000fa
:10e22800c69800007a240000f8a60000441a0000ee
:10e2380099c70000257b00003a64000086d80000da
:10e248005b050000e7b900008cd20000306e0000ca
:10e25800edb30000510f00004e100000f2ac0000ba
:10e268002f71000093cd0000114f0000adf30000a6
:10e27800702e0000cc920000d38d00006f3100009a
:10e28800b2ec00000e500000aff10000134d00008a
:10e29800ce900000722c00006d330000d18f00007a
:10e2a8000c520000b0ee0000326c00008ed000006e
:10e2b800530d0000efb10000f0ae00004c1200005a
:10e2c80091cf00002d730000ca940000762800004a
:10e2d800abf500001749000008560000b4ea00003a
:10e2e80069370000d58b000057090000ebb5000026
:10e2f800366800008ad4000095cb0000297700001a
:10e30800f4aa000048160000e9b70000550b000009
:10e3180088d60000346a00002b75000097c90000f9
:10e328004a140000f6a80000742a0000c8960000ed
:10e33800154b0000a9f70000b6e800000a540000d9
:10e34800d78900006b35000045720000726f00002d
:10e35800722000003a20000053750000636300003b
:10e368006573000073200000282000006e6f000015
:10e3780020650000727200006f720000290d000015
:10e3880000450000727200006f720000203a000021
:10e39800204300006f6d00006d7500006e6900007d
:10e3a80063610000746900006f6e0000206900005e
:10e3b80073730000756500000d00000045720000d1
:10e3c800726f0000722000003a2000004e6f0000bb
:10e3d800207400006f75000063680000206400006e
:10e3e8006576000069630000652000007072000017
:10e3f80065730000656e0000740d000000450000a4
:10e40800727200006f720000203a00002054000071
:10e4180072790000696e000067200000746f0000c8
:10e428002061000063630000657300007320000032
:10e43800612000006279000074650000206e000011
:10e448006f740000206100006c6c00006f770000a2
:10e4580065640000206200007920000074680000f4
:10e4680065200000667500006e6300007469000096
:10e478006f6e00000d00000045720000726f000012
:10e48800722000003a2000005472000079690000f0
:10e498006e670000207400006f20000072650000a5
:10e4a80061640000207400006865000020730000ab
:10e4b8006563000072650000740d000000450000ef
:10e4c800727200006f720000203a0000204e0000b7
:10e4d8006f20000064650000766900006365000035
:10e4e80020630000686f0000736500006e20000064
:10e4f800746f000020720000656100006420000055
:10e50800746f00000d00000045720000726f00007b
:10e51800722000003a200000496d0000706f000072
:10e5280073730000696200006c65000020740000cd
:10e538006f2000006f76000065720000777200009f
:10e548006974000065200000612000007365000008
:10e558006372000065740000206200007974000096
:10e56800650d000000450000727200006f72000027
:10e57800203a000020540000686500007220000066
:10e588006279000074650000207700006173000064
:10e598006e74000020770000726900007474000037
:10e5a800656e00002073000075630000636500005d
:10e5b80073660000756c00006c7900000d000000a7
:10e5c80045720000726f0000722000003a200000bf
:10e5d8005468000065200000617500007468000040
:10e5e8006f720000697a000061740000696f0000b2
:10e5f8006e2000006279000074650000732000003e
:10e6080064690000642000006e6f00007420000040
:10e618006d610000746300006820000074680000e9
:10e62800652000006368000069700000730d000039
:10e6380000450000727200006f720000203a00006e
:10e64800204400006174000061200000636f000036
:10e658006c6c000069730000696f00006e20000098
:10e6680064750000726900006e6700002063000096
:10e678006f6d00006d7500006e6900006361000039
:10e68800746900006f6e0000207700006974000054
:10e69800682000006465000076690000636500007a
:10e6a8000d00000045720000726f0000722000002b
:10e6b8003a200000417200006561000020620000fd
:10e6c800656900006e67000020770000726900002d
:10e6d80074740000656e0000207400006f20000054
:10e6e80069730000207700007269000074650000fb
:10e6f80020700000726f00007465000063740000f1
:10e70800656400000d00000045720000726f000093
:10e71800722000003a20000047690000766500007a
:10e728006e2000007061000067650000206e000028
:10e73800756d00006265000072200000646f0000c3
:10e74800657300006e2700007420000065780000e3
:10e7580069730000740d000000450000727200002b
:10e768006f720000203a0000205500006e72000011
:10e77800656300006f6700006e6900007a6500003d
:10e788006420000065720000726f0000722e0000a5
:10e798002e2e0000206f000075700000732e000000
:10e7a8002e2e00002e0d0000006500007272000081
:10e7b800206300006f6c00006c6900007369000042
:10e7c8006f6e00000d0000004261000074740000cc
:10e7d800657200007920000050610000636b000042
:10e7e800204600006f7500006e640000203a0000ab
:10e7f800205300004e2000000025000058000000b3
:10e808000d00000042750000664f000076660000ab
:10e818006c6f0000770d0000006d00006932000089
:10e82800635f000077720000697400006562000091
:10e8380079740000652000003a200000646100003f
:10e8480074610000203d000020250000322e0000e9
:10e85800325800000d0a0000006d00006932000007
:10e86800635f000072650000616400006279000067
:10e8780074650000203a0000206100006464000014
:10e88800203d000020250000322e000032580000f4
:10e898000d0a0000006d000069320000635f00008f
:10e8a8007265000061640000627900007465000010
:10e8b800203a000020760000616c0000203d000036
:10e8c80020250000322e0000325800000d0a0000fa
:10e8d8000000000042750000664f000076660000e8
:10e8e8006c6f0000770d00000000000070720000df
:10e8f800696e0000745f000066690000666f0000c2
:10e908005f700000747200003a200000706c000014
:10e9180061630000652000007768000065720000f0
:10e928006520000077650000206400006174000025
:10e938006120000069730000202000003a200000d8
:10e9480030780000255800000d0a00000070000013
:10e95800726900006e7400005f660000696600005e
:10e968006f5f000070740000723a000020700000b1
:10e978006c61000063650000207700006865000096
:10e9880072650000207700006520000073740000a5
:10e998006f7200006520000069730000203a0000d3
:10e9a8002030000078250000580d00000a00000003
:020000040000fa
:10e9b800f81100000800000002000000000000003c
:10e9c8000000000000000000c8170000320000002e
:10e9d80000000000d2080000020000000200000051
:10e9e80000000000c608000004000000000000004d
:10e9f800ca08000004000000000000009c08000095
:10ea080010000000020000000400030000050000e0
:10ea18000000ff00ff0f00000100070000000000d9
:10ea2800f41000004e000000020000000200fe008a
:10ea3800fffcff00f4ff05000002000002000200d6
:10ea48000004000002000200000200000500f400bb
:10ea5800fffcff00feff0200000400000200fe00b1
:10ea6800fffaff000400040000000000000000009e
:10ea7800000000000400040000faff00feff02008e
:10ea8800000000000000000000000000320000004c
:10ea980002000000ac0800001000000000000000a8
:10eaa800bc0800000a00000002000000000000008e
:10eab80000000000000000000000000076100000c8
:10eac8007e00000000000000d408000002000000e2
:10ead8000200000000000000d41100002400000023
:10eae8000200000004000000000000000000000018
:10eaf800000000000000000000000000000000000e
:10eb0800000000002c165a0016881600b616e400fd
:10eb18001612170000130000400400000000000057
:10eb280000100000020000000200000000000000c9
:10eb380002100000020000000200000000000000b7
:10eb480004100000020000000200000000000000a5
:10eb58000610000002000000020000000000000093
:10eb68000810000002000000020000000000000081
:10eb78000a1000000200000002000000000000006f
:10eb88000c1000000200000002000000000000005d
:10eb98000e1000000200000002000000000000004b
:10eba8001010000002000000020000000000000039
:10ebb80012100000640000000200000000000000c5
:10ebc800000000000000000000000000000000003d
:10ebd800000000000000000000000000000000002d
:10ebe800000000000000000000000000000000001d
:10ebf800000000000000000000000000000000000d
:10ec080000000000000000000000000000000000fc
:10ec180000000000000000000000000000000000ec
:10ec280000000000000000000000000000000000dc
:10ec380000000000000000000000000000000000cc
:10ec480000000000001200000001000002000000a7
:10ec580000000000000000000000000000000000ac
:10ec6800000000000000000000000000000000009c
:10ec7800000000000000000000000000000000008c
:10ec8800000000000000000000000000000000007c
:10ec9800000000000000000000000000000000006c
:10eca800000000000000000000000000000000005c
:10ecb800000000000000000000000000000000004c
:10ecc800000000000000000000000000000000003c
:10ecd800000000000000000000000000000000002c
:10ece800000000000000000000000000000000001c
:10ecf800000000000000000000000000000000000c
:10ed080000000000000000000000000000000000fb
:10ed180000000000000000000000000000000000eb
:10ed280000000000000000000000000000000000db
:10ed380000000000000000000000000000000000cb
:10ed480000000000000000000000000000000000bb
:10ed580000000000000000000000000000000000ab
:10ed6800000000000000000000000000000000009b
:10ed7800000000000000000000000000000000008b
:10ed8800000000000000000000000000000000007b
:10ed9800000000000000000000000000000000006b
:10eda80000000000000000001c0a00000c00000029
:10edb8000200000000000000000000000000000049
:10edc80000000000280a00000a00000000000000ff
:10edd8000c0a000010000000020000000000000003
:10ede8000000000000000000000000000000ff001c
:10edf80000000000e00800006400000000000000bf
:10ee0800320a0000080000000200000000000000b4
:10ee18000000000000000000440900006400000039
:10ee280000000000420a000002000000020000008a
:10ee380000000000da0900001e00000000000000c9
:10ee4800f8090000140000000200000000000000a3
:10ee5800000102000408100020408000fefdfb00b5
:10ee6800f7efdf00bf7f0000440a00000200000047
:10ee780000000000421100004a00000002000000eb
:10ee880030313200333435003637380039616200aa
:10ee98006364650066676800696a6b006c6d6e0084
:10eea8006f707100727374007576770078797a00e4
:10eeb80000000000211511000e0d0c000b0b0a00bc
:10eec8000a090900090909000808080008080800d3
:10eed80008070700070707000707070007070700d5
:10eee800070700004017000088000000020000002b
:10eef8000100000000661700671766001766170014
:10ef08006617660017561700000000000000000092
:10ef180000000000000000000000000000000000e9
:10ef2800000000000002080001018e00178f170082
:10ef38008e178e00178e17008e177e0017000000a0
:10ef480000000000000000000000000000000000b9
:10ef5800000000000000000000000200080202009b
:10ef6800b617b70017b61700b617b60017b61700ca
:10ef7800a6170000000000000000000000000000cc
:10ef88000000000000000000000000000000000079
:10ef980040176800179017000000000000000000ec
:10efa80000000000000000008a08000012000000b5
:10efb80002000000202b2d00233000000100020079
:10efc8000004000008001000000000003a0a0000d9
:10efd8000800000002000000686a6c00747a4c00a7
:10efe80000000000ce08000004000000020000003d
:10eff8000000000000000000500800002000000091
:10f00800020000000a000000006400000000e800a0
:10f01800030000001027000000a086000100400047
:10f02800420f0000809698000000e100f5050000fe
:10f03800000800002e0000000200000030313200fd
:10f04800333435003637380039616200636465004f
:10f0580066414200434445004600000001020300a7
:10f0680004050600070809000a0b0c000d0e0f0026
:10f078000a0b0c000d0e0f000000000070080000c5
:10f088001a000000020000000000200041000000fb
:10f09800c8420000401c460020bcbe004cca1b00f1
:10f0a8000e5aae00c59d740005000000fa17000056
:10f0b800060000000200000000000000000002003e
:10f0c800d608000002000000000000008c110000bb
:10f0d80048000000020000000000000000000000de
:10f0e800244000000000000000005900400000001b
:10f0f8000000000088c34000000000000084d70022
:10f108009741000080e0370079c3410043176e0043
:10f1180005b5b500b8934600f5f93f00e9034f007f
:10f12800384d32001d30f900487782005a3cbf0044
:10f13800737fdd004f157500a8090000320000003c
:10f14800020000004e414e00006e61006e00490052
:10f158004e460000696e66000030310032333400dc
:10f16800353637003839610062636400656600002f
:10f1780030313200333435003637380039414200f7
:10f1880043444500460000002e080000220000000d
:10f198000200000030313200333435003637380091
:10f1a8003961620063646500660030003132330003
:10f1b800343536003738390041424300444546006b
:10f1c80000000000d8080000020000000200000053
:10f1d80000000000460a00000200000002000000d3
:10f1e80030000000da080000020000000200000001
:10f1f80000000000dc08000002000000020000001f
:10f2080001000000de08000002000000000000000d
:04f2180000000000f2
:00000001FF
